:020000040800F2
:100000000020001045BC0208951F02086902010883
:10001000911F02088D1F0208891F020800000000BE
:10002000000000000000000000000000851F020822
:10003000811F0208000000007D1F0208B5C90008EA
:10004000ADBC0208ADBC0208ADBC0208ADBC0208E4
:10005000ADBC0208ADBC020891110008BD12000839
:1000600081120008451200080912000851280008F2
:10007000412800083128000821280008112800081C
:10008000FD270008E9270008ADBC0208ADBC020846
:10009000C9230208ADBC0208ADBC0208CD1100089E
:1000A000A1BE0008D1BE000891BE0008F9BE00083C
:1000B000C1BE0008B1BE0008ADBC0208ADBC02085C
:1000C000ADBC0208ADBC0208ADBC0208ADBC020864
:1000D000ADBC020839CB0008BDCA000841CA0008FF
:1000E00057110008ADBC02086D1F0208ADBC020824
:1000F000ADBC0208ADBC0208ADBC0208ADBC020834
:10010000000000000000000000000000ADBC02087C
:10011000ADBC0208ADBC0208ED850208D18502081D
:10012000D5270008C1270008AD2700089927000837
:1001300085270008ADBC0208000000000000000098
:10014000ADBC0208ADBC0208ADBC02080000000056
:10015000000000000000000000000000000000009F
:100160000000000000000000ADBC0208ADBC0208A9
:10017000ADBC02080000000000000000000000000C
:0801800000000000ADBC020804
:10018800152303701623C370172383712D2343701F
:100198002E2303712F23C3717047F0B484894FF65F
:1001A800FF764FF47A743BB3002937D00F780131CA
:1001B80001E0B44219D00589013C15F00205A4B24A
:1001C800F7D007734FF47A7402E0BCB2B4420CD093
:1001D800058915F0010504F1FF37F6D0057BEDB26E
:1001E8000AB115700132013BDDE70D4B984207D08B
:1001F800A3F57843984202D00120F0BC704701254E
:10020800084B03EB05156B8901339BB26B81688939
:1002180080B2003018BF0120F0BC7047FF27CAE742
:10022800003001405C67002040F2E93300E09BB1F8
:100238000289013B12F0020F9BB2F8D0017340F221
:10024800E93300E043B10289013B12F0010F9BB290
:10025800F8D0007BC0B27047094A904205D0094BDC
:10026800984201D0FF2070470123074A02EB03138D
:100278005A89013292B25A815889C0B2704700BF78
:1002880000300140003800405C670020002870B54D
:100298001EDB0928044620DD012303EB83035B00F2
:1002A800B0FBF3F2092AF8D87BB10E4EB4FBF3F099
:1002B8000928CCBF57223022A6FB03E5024403FBE2
:1002C8001044EB0801F8012BF0D100230B7070BD2E
:1002D8002D230B7040420131DBE7303001F8010B70
:1002E800F3E700BFCDCCCCCC884230B44FF001044A
:1002F8002ED301FB04F4B0FBF4F58D42F9D284B19E
:10030800AAB901E0B0FBF4F5092DCCBF5722302281
:100318002A4404FB150003F8012BB4FBF1F4002C6C
:10032800F0D100221A7030BC7047B0FBF4F5092DEB
:10033800CCBF372230222A4404FB150003F8012BD6
:10034800B4FBF1F4002CF0D100221A7030BC7047D5
:100358000546002AEBD1D7E703685A1C02601970DA
:1003680070472DE9F047089C2578002B8046894680
:100378000CBF4FF0200A4FF0300A661C35B3002A34
:1003880029DD334601E0024698B113F8011B501EDF
:100398000029F8D1971E60B13D46013D51464046BF
:1003A800C8476B1C002BF8DC257827EAE77001307A
:1003B80055B1041B29464046C847301916F8015B59
:1003C800002DF7D1BDE8F087BDE8F087002A04DCEE
:1003D8002846BDE8F0870020EBE7571EDCE7836876
:1003E8004268D0ED037A00EB83010133934281ED3B
:1003F800040A836004BF0023836000EB830393ED4A
:10040800047A036870EE277A9A42C0ED037A77EE91
:10041800C77AC0ED037A0CDA013307EE103AF8EE2A
:10042800C76AB7EE007A87EEA60A036030EE070ABD
:10043800704707EE102AB8EEC77A87EE870A70472A
:1004480090ED057A90ED004AD0ED066AD0ED014AAC
:10045800D0ED047A90ED035AD0ED025AA4EE007A5A
:10046800B0EE406AB0EE470AB0EE667AA6EE247A9D
:1004780067EEC07AA0EE457AE6EE257A80ED057A39
:10048800C0ED067A7047D0ED057A90ED013AD0EDCF
:10049800003AD0ED064A90ED024A90ED077A90EDC9
:1004A800035A90ED086AD0ED045AC0ED067AF0EED2
:1004B800406A27EE830AC0ED056AA3EEA60A80ED1E
:1004C800087AA4EE240AA5EE470AA5EEC60A80ED2E
:1004D800070A7047D0ED007A90ED017A30EE670A8E
:1004E800E7EE007AB0EE670AC0ED007A7047704711
:1004F8000A44914214D030B40139551E41F2210208
:1005080011F8014F082380EA042004044CBF82EA52
:1005180040004000013B80B2F7D18D42F0D130BCA1
:10052800704750F8043C012280F84520103803B188
:100538001847704790F8203033B1012B03D14FF49E
:1005480000638382704770474FF4806383827047EB
:1005580070B5044682B01430E56D06236A4643211F
:10056800A847B0B19DF804009DF800609DF80110FF
:100578009DF802509DF803209DF8053041EA0621B8
:1005880043EA002342EA0522A187E287A4F8403023
:10059800012002B070BD70B5044682B00830656AAB
:1005A80006236A463B21A847A8B19DF804009DF898
:1005B80000609DF801109DF802509DF803209DF8F9
:1005C800053041EA062143EA002342EA0522E18296
:1005D80022836383012002B070BD70B40468037B7A
:1005E8002268022101FA03F31A4213D042690A4928
:1005F800582000FB02124FF6FE7650685289C568F3
:100608000068296831402960C168D24392B20A4023
:10061800C260636070BC7047F061002030B4094B61
:100628001C7864B1084B002503EBC4041A68998848
:100638005562D06808330143A342D160F6D130BC7B
:10064800704700BFB0640020B464002010B4026892
:10065800047B11680223A340194209D00649406867
:1006680000240C7001684FF6FE742140016053604D
:100678005DF8044B704700BF5B380020F0B4334C82
:1006880000EB800004EB80046468002C5BD0304EE3
:1006980049004FF42040CDB23060A169090444D428
:1006A80060682C4F45F08071384041F49031014327
:1006B8004FF420406160306003E0411E002838D0CC
:1006C8000846A1698F07F8D54FF42040A262306030
:1006D80002E0421E68B31046A2691106F9D56268A5
:1006E8001C4945F0007545F480350A4015434FF420
:1006F80020406560306002E0421ED0B11046A26919
:100708009207F9D5A362A3694FF420409B06306095
:1007180005D4431E68B11846A3699B06F9D5202362
:100728003060E3610120F0BC7047411E08B1084603
:10073800B3E7094A138801339BB24FF0FF313160A8
:100748001380F0BC70472046F0BC70478C580020DE
:10075800B4580020009800FCB85800201346002028
:100768000A4668218AE700232622036002702722AE
:100778008270012243600271837170472DE9F34151
:10078800056906460F467DBBD0F80080C8F30A030A
:1007980023B30023D6F80080019323F0B1F804288E
:1007A80019D1224C236943F001032361BBB2A8F895
:1007B800003023F0A5F804282ED108F10203019394
:1007C800019B3F0C1F8023F09BF82369042823F02A
:1007D8000103236125D06FF0010505E023F090F8AF
:1007E800042805D04FF0FF35284602B0BDE8F08157
:1007F8000E4C236943F002032361C4F81480236973
:1008080043F04003236123F07BF82369042823F095
:1008180002032361BDD0E5E7236923F001032361C7
:10082800D9E7336804333360DEE700BF00200240B5
:10083800F8B504460D468E180027B54201D1206947
:10084800F8BDE368591CE160234415F8012B1A72BE
:100858000429F2D1A1682046FFF790FFE7602061E4
:10086800EBE7024B18680CF011BA00BFE8570020FC
:100878000846194624F040BD10B490E80600047BF1
:1008880040690223A3404B6013685DF8044B4FF6A0
:10089800FE710B4013600CF089B9002867D003681B
:1008A8002DE9F04F03F138445B4EA40A0125345D6D
:1008B80004F01F066409022C05FA06F558D0032C2B
:1008C80000F0A580012C58D08088B0FA80F4C4F1DB
:1008D8001F04A4B2E50803EB850504F007042E6A9B
:1008E800A4000F27A74026EA07062E622E6A01F009
:1008F8000307A2407C1E3243012CC1F3810CC1F3D3
:1009080000182A62C1F341113CD9C60700F188805A
:10091800850700F19480440700F1A280020700F1E6
:10092800B080C60600F1BE80850600F1CC80440682
:1009380000F1DA80020600F1E880C60500F1F680D1
:10094800850500F10481440500F11281020500F1DA
:100958002081C60400F12E81850400F13C81440405
:1009680000F14A81020400F15881BDE8F08F704718
:100978002A4CA6693543A561A6E7284C6669354324
:100988006561A1E7002422464FF0010E4FF00309EC
:1009980004E00132102A04F10204E6D00EFA02F64D
:1009A80036EA0005F5D1D3F808A009FA04F5ED43B5
:1009B8000AEA050AC3F808A0D3F808B00CFA04FA42
:1009C8004AEA0B0AC3F808A0B3F804A01FFA8AFA87
:1009D8002AEA06069E80B3F804A008FA02F646EA58
:1009E8000A06B6B29E801E682E401E60D3F800A08C
:1009F80007FA04F646EA0A061E60D3F80CA001FAC4
:100A080004F605EA0A0A46EA0A05DD60C1E7034C6E
:100A1800E6693543E56157E7240D030800100240F5
:100A28001A6822F003021A601A683A431A60DA68F0
:100A380022F003020A438507DA607FF56CAF1A6873
:100A480022F00C021A601A6842EA87021A60DA6811
:100A580022F00C0242EA81024407DA607FF55EAFB9
:100A68001A6822F030021A601A6842EA07121A60FD
:100A7800DA6822F0300242EA0112DA6002077FF5F2
:100A880050AF1A6822F0C0021A601A6842EA871248
:100A98001A60DA6822F0C00242EA8112C606DA60F9
:100AA8007FF542AF1A6822F440721A601A6842EA67
:100AB80007221A60DA6822F4407242EA01228506A7
:100AC800DA607FF534AF1A6822F440621A601A6857
:100AD80042EA87221A60DA6822F4406242EA8122F6
:100AE8004406DA607FF526AF1A6822F440521A608D
:100AF8001A6842EA07321A60DA6822F4405242EA77
:100B08000132DA6002067FF518AF1A6822F4404213
:100B18001A601A6842EA87321A60DA6822F4404298
:100B280042EA8132C605DA607FF50AAF1A6822F414
:100B380040321A601A6842EA07421A60DA6822F4F8
:100B4800403242EA01428505DA607FF5FCAE1A6858
:100B580022F440221A601A6842EA87421A60DA6868
:100B680022F4402242EA81424405DA607FF5EEAE83
:100B78001A6822F440121A601A6842EA07521A6088
:100B8800DA6822F4401242EA0152DA6002057FF57F
:100B9800E0AE1A6822F440021A601A6842EA8752E4
:100BA8001A60DA6822F4400242EA8152C604DA6026
:100BB8007FF5D2AE1A6822F040721A601A6842EACB
:100BC80007621A60DA6822F0407242EA016285041C
:100BD800DA607FF5C4AE1A6822F040621A601A68BB
:100BE80042EA87621A60DA6822F0406242EA816269
:100BF8004404DA607FF5B6AE1A6822F040521A60F3
:100C08001A6842EA07721A60DA6822F0405242EA29
:100C18000172DA6002047FF5A8AE1A6822F0404239
:100C28001A601A6842EA87771F60DA6822F0404241
:100C380042EA8171D960BDE8F08F002852D003687C
:100C480003F138422DE9F04F920A514DAA5C02F0A7
:100C58001F0552090124022A04FA05F443D0032A85
:100C680000F09080012A43D001F003077A1E012A80
:100C7800C1F3810CC1F300188088C1F341113CD93C
:100C8800C60700F18980850700F19580440700F1C7
:100C9800A380020700F1B180C60600F1BF80850677
:100CA80000F1CD80440600F1DB80020600F1E98006
:100CB800C60500F1F780850500F10581440500F1BE
:100CC8001381020500F12181C60400F12F818504FA
:100CD80000F13D81440400F14B81020400F1598187
:100CE800BDE8F08F70472B4A95692C439461BBE7A8
:100CF800284A55692C435461B6E7002422464FF030
:100D0800010E4FF0030904E00132102A04F1020435
:100D1800E6D00EFA02F636EA0005F5D1D3F808A0B7
:100D280009FA04F5ED430AEA050AC3F808A0D3F85E
:100D380008B00CFA04FA4AEA0B0AC3F808A0B3F898
:100D480004A01FFA8AFA2AEA06069E80B3F804A0CD
:100D580008FA02F646EA0A06B6B29E801E682E40D7
:100D68001E60D3F800A007FA04F646EA0A061E60D9
:100D7800D3F80CA001FA04F605EA0A0A46EA0A05BD
:100D8800DD60C1E7034AD5692C43D4616CE700BF35
:100D9800240D0308001002401A6822F003021A60AA
:100DA8001A683A431A60DA6822F003020A43850790
:100DB800DA607FF56BAF1A6822F00C021A601A68C5
:100DC80042EA87021A60DA6822F00C0242EA8102DB
:100DD8004407DA607FF55DAF1A6822F030021A60C6
:100DE8001A6842EA07121A60DA6822F0300242EA08
:100DF8000112DA6002077FF54FAF1A6822F0C002CD
:100E08001A601A6842EA87121A60DA6822F0C00289
:100E180042EA8112C606DA607FF541AF1A6822F409
:100E280040721A601A6842EA07221A60DA6822F4E5
:100E3800407242EA01228506DA607FF533AF1A680C
:100E480022F440621A601A6842EA87221A60DA6855
:100E580022F4406242EA81224406DA607FF525AF37
:100E68001A6822F440521A601A6842EA07321A6075
:100E7800DA6822F4405242EA0132DA6002067FF56B
:100E880017AF1A6822F440421A601A6842EA873299
:100E98001A60DA6822F4404242EA8132C605DA6012
:100EA8007FF509AF1A6822F440321A601A6842EADC
:100EB80007421A60DA6822F4403242EA01428505A4
:100EC800DA607FF5FBAE1A6822F440221A601A68CD
:100ED80042EA87421A60DA6822F4402242EA8142F2
:100EE8004405DA607FF5EDAE1A6822F440121A6004
:100EF8001A6842EA07521A60DA6822F4401242EA93
:100F08000152DA6002057FF5DFAE1A6822F440026A
:100F18001A601A6842EA87521A60DA6822F44002B4
:100F280042EA8152C604DA607FF5D1AE1A6822F02F
:100F380040721A601A6842EA07621A60DA6822F098
:100F4800407242EA01628504DA607FF5C3AE1A682E
:100F580022F040621A601A6842EA87621A60DA6808
:100F680022F0406242EA81624404DA607FF5B5AE5D
:100F78001A6822F040521A601A6842EA07721A6028
:100F8800DA6822F0405242EA0172DA6002047FF520
:100F9800A7AE1A6822F040421A601A6842EA8777B8
:100FA8001F60DA6822F0404242EA8171D960BDE8E8
:100FB800F08F70B5044690F85900002833D104F139
:100FC8001405236E80226B212846984764200BF075
:100FD8004FFC236E284603226B219847236E94F812
:100FE80054201921284698470F200BF041FC236E06
:100FF80094F8522028461A219847236E284618222A
:101008001B219847236E284618221C219847236ED7
:1010180028460222372198472846236E0122382184
:10102800BDE8704018470AF009FF0546D0B12023F3
:1010380000218371C171FFF700FE21460F4B41F873
:10104800103F284629F0EAF9AB88B3FA83F3C3F1D5
:101058001F035A1CB3D001229A4009490B68134355
:101068000B60ACE70146FFF7E8FD2146034B41F86A
:10107800103F284629F0D2F90122EEE72B05000897
:101088000004014010B1036882881A85704710B1C6
:10109800036882889A61704710B5014600BF074C03
:1010A80023689868FFF7EEFF23685868FFF7BCF8D5
:1010B80023689868FFF7EBFF00BF10BDC45D0020F0
:1010C80038B500231C4620FA03F2C3F11F0102F0D1
:1010D800010201338A40202B44EA0204F3D1104D67
:1010E8002868FFF7CFFF210E0E48FFF79DF8C4F3DD
:1010F80007410C48FFF798F8C4F307210948FFF7A0
:1011080093F8E1B20748FFF78FF802200BF056FB7F
:101118002868FFF7BCFF0220BDE838400BF04EBB43
:10112800B02400200030014038B1002983880268CB
:1011380014BF002110218B409361704730B10368C0
:1011480082881B8A1A4214BF0120002070472DE9AB
:10115800F0410B4E346873691C400FD0DFF82480CF
:101168000127B4FA84F3C3F11F0307FA03F558F80B
:10117800230003689847AC437561F2D1BDE8F0815C
:1011880000040140146700202DE9F0410B4E34683B
:1011980073691C400FD0DFF828800127B4FA84F364
:1011A800C3F11F0307FA03F558F8230003689847AB
:1011B800AC437561F2D1BDE8F08100BF0004014085
:1011C800146700202DE9F0410B4E346873691C4008
:1011D8000FD0DFF828800127B4FA84F3C3F11F0386
:1011E80007FA03F558F8230003689847AC4375617C
:1011F800F2D1BDE8F08100BF00040140146700206F
:101208002DE9F0410B4E346873691C400FD0DFF8AC
:1012180028800127B4FA84F3C3F11F0307FA03F502
:1012280058F8230003689847AC437561F2D1BDE8CC
:10123800F08100BF00040140146700202DE9F0414F
:101248000B4E346873691C400FD0DFF828800127E3
:10125800B4FA84F3C3F11F0307FA03F558F823001F
:1012680003689847AC437561F2D1BDE8F08100BFCF
:1012780000040140146700202DE9F0410B4E34684A
:1012880073691C400FD0DFF828800127B4FA84F373
:10129800C3F11F0307FA03F558F8230003689847BA
:1012A800AC437561F2D1BDE8F08100BF0004014094
:1012B800146700202DE9F0410B4E346873691C4017
:1012C8000FD0DFF828800127B4FA84F3C3F11F0395
:1012D80007FA03F558F8230003689847AC4375618B
:1012E800F2D1BDE8F08100BF00040140146700207E
:1012F800084A094808B5936943F00103936100213E
:1013080040222DF08EF9054B4FF0FF321A60C3F8DA
:10131800032008BD00100240146700205467002015
:1013280003685B6A18472DE9F041044618460D46E4
:101338001646984629F0C4FF2768E6722844A0722A
:1013480029467D69434632462046AC46BDE8F04111
:101358006047036810B504461B6898472368204611
:101368009B689847A37B0133A37310BD10B503682E
:1013780004469B689847FF2301226373227310BDBC
:1013880008B50AF05BFD38B12C2282710022C271C7
:101398002021BDE8084050E408BDF8B5574C0601C7
:1013A800A7190546387A23F0ADFD3B7A03F01F01F3
:1013B8005B090122022B02FA01F278D0032B71D0CB
:1013C800012B67D0A319013518790AF037FDEDB262
:1013D800074610B11223C5718371A31958790AF011
:1013E8002DFD10B11323C5718371A31998790AF0E3
:1013F80025FD10B11423C5718371A5190E21EA7951
:101408003846FFF74AFA68790AF018FDEA790E219A
:10141800FFF743FAA8790AF011FDEA790E21FFF7E0
:101428003CFAA359364A934251D0364A934259D08E
:10143800354A934240D03444227B002A2FD10120E0
:1014480002249A8822F480521204120C9A809988F5
:1014580089B241F4805199801A8802F4415242F4C9
:101468004572024322431A809A8822F47062120459
:10147800120C42F4E0629A809A8B22F40062120401
:10148800120C07219A8319821A8892B242F04002FC
:101498001A80F8BD1D4B996A0A439A6292E70020A8
:1014A8000446CEE7194B19690A431A618AE7174BB4
:1014B800D9680A43DA6085E702F5EA32116941F42E
:1014C80000411161116921F400411161B3E702F58E
:1014D8006042D16841F48051D160D16821F48051D3
:1014E800D160A8E702F5EC32116941F4804111613D
:1014F800116921F4804111619DE700BF5C670020FC
:101508000030014000380040003C0040001002401C
:10151800427A02B9704710B504460368406804F17E
:101528000A0198470023637210BD437A5A1C03448A
:10153800D2B242729972037A934200D802B97047C4
:1015480010B504460368406804F10A01984700236F
:10155800637210BD10B40B49002301E0272B0CD097
:1015680011F8132082424FEA430403F10103F5D135
:1015780021445DF8044B4878704700205DF8044B1F
:10158800704700BF94E7020870B5448806460D46C8
:10159800C4F30B042246002128462DF042F8336993
:1015A800094A934209D3094A934206D22246284659
:1015B8001946BDE870402AF0B5BD23B1214628463A
:1015C800BDE87040184770BD1C490308104A03085D
:1015D800064B07498B4202D30023184670471A88E6
:1015E800C2F30B029042F8D01433F3E7D044030857
:1015F8001C490308024A136823EA00001060704778
:1016080028420020F8B5174D2B78A32B28D16B78EA
:10161800BE2B25D1022229464FF6FF70FEF768FF40
:10162800114FAC1C22884AB1A618BE4218D2052A0E
:1016380016D92146FEF75CFF3446F3E7214602221D
:10164800FEF756FF0222A118FEF752FF0634074B99
:10165800641B1C8041F60F53C31A58425841F8BD09
:101668000020F8BD00F0030800000408AC2C00209E
:101678002DE9F04FDFF848914C4F8BB00326A7EBCC
:1016880009071822002104A82CF0CBFF484BCDF8FD
:10169800109005971A69120604D5464A5A6002F155
:1016A80088325A6001228DF824203422DA60424BB5
:1016B800424C1B88ADF800300222694604A8FFF7A7
:1016C800B7F8022269464FF6FF70FEF711FFDFF800
:1016D800F4A080464FF0000B544536D30AAC0025E1
:1016E80024F8245D0222214604A8FFF7A1F802226B
:1016F80021464046FEF7FCFE40BAC043ADF808005C
:10170800022202A904A8FFF793F8079860B106AB74
:10171800C0F10402294618442CF083FF069904A856
:10172800FFF72CF8079508909DF82430089A23B104
:101738001F490B6943F080030B61013E2DD0002A3D
:101748009FD1FFF75FFF50B32CE065888DF80DB08F
:10175800C5F30B05AB1DADF808302388C3F30B02A6
:10176800ADF80A201B0B062202A904A88DF80C303C
:10177800FFF75EF8062202A94046FEF7B9FE616847
:1017880080462A4604A8FFF753F8616840462A466F
:10179800FEF7AEFE143480469EE7002AD1D005201D
:1017A8000AF062FD0BB0BDE8F08F00BF000004082E
:1017B8000020024023016745E2E70208D0440308FD
:1017C80000F003081C4903080378202B024600F1A7
:1017D8000100F9D0092BF7D02D2B2CD02B2B03BFD0
:1017E8005378B7EE000A0246B7EE000AA3F13001BB
:1017F800C8B209289FED467A10D8F2EE046A07EEBF
:10180800901AF8EEE77A12F8013FE7EE267AA3F18C
:101818003001C8B20928B0EE677AF0D92E2B4CD027
:1018280003F0DF03452B0BD0F7EE007A67EE276A4B
:1018380020EE260A70475378BFEE000A0246D5E725
:1018480010B451782D2959D02B290ABF9178501CF2
:10185800901C0024A1F13003092B53D8002303EB7B
:10186800830301EB430310F8011FA1F13002092A99
:10187800A3F13003F3D9B3F59A7F28BF4FF49A73D5
:10188800072B42D9DFED236A1A46F7EE007A083AA9
:10189800072A67EEA67AFAD803F007032BB1F2EE0F
:1018A800046A013B67EEA67AFBD124B3C7EE276A28
:1018B8005DF8044B20EE260A70475378A3F13001F7
:1018C800C8B2092802F10102AAD8F2EE046AF0EEC1
:1018D800665A07EE901AF8EEE77A12F8013F87EE9B
:1018E800A66AA3F13001C8B2092866EEA56A37EEE8
:1018F800067AEED994E767EE276AD9E7901C9178C3
:101908000124A7E7F7EE007ACFE7F7EE007AC5E7FC
:101918000000000020BCBE4CB5EEC00ADFED317AF5
:10192800F1EE10FACCBF30EE270A30EE670ADFED91
:101938002E7A20EE270A30B5FDEEC07A87B017EE72
:10194800904A054684EAE470002303A9A0EBE470FA
:1019580001930093029322F0DBF9002CACBF202303
:101968002D2303A88DF8003029F0AAFC012803A92B
:1019780024D002282DD0032805BF302368466846A6
:101988008DF801302CF073FE684629F099FC033875
:10199800C4B22246694628462CF0C7FE00232B55C0
:1019A800284629F08DFC2E22431C2A540DEB0401F5
:1019B800E8182CF079FE284607B030BD3023684679
:1019C8008DF801308DF802308DF803302CF04FFE81
:1019D800DAE7302368468DF801308DF802302CF0B4
:1019E80046FED1E76F12033A00007A442DE9F04130
:1019F800064615460846B6FBF2F43CB905FB1464E6
:101A0800124B1B5D00F8013BBDE8F081B4FBF2F717
:101A180067B90E4B05FB174705FB1464DA5D00F840
:101A2800012B1B5D00F8013BBDE8F081B7FBF2F824
:101A3800B8F1000F02D04046FFF7D8FF05FB187831
:101A4800024B13F8082000F8012BE3E754130308AE
:101A580030B402681146531C036011F8024B016050
:101A6800D31C517803609378151D05601B0443EA65
:101A78000123D078234343EA006030BC70470368F1
:101A8800591C1A46016012F8021B0260587841EA94
:101A98000020704703685A1C02601878704738B5F0
:101AA8000446006815462AF03DFB22682A44226055
:101AB80038BD036810B40A0A5C1C04601A70036815
:101AC8005A1C026019705DF8044B704703685A1C71
:101AD800026010B4197003680A0A5C1C04601A706A
:101AE80003680A0C5C1C04601A700368090E5A1C0F
:101AF800026019705DF8044B704703685A1C026055
:101B080019700368090A5A1C0260197070472DE998
:101B1800F047002488B080460F461E46A14605AD12
:101B2800531C0393117839B3252933D1931CCDF86D
:101B380010900393507830284ED04FF0000AA0F14F
:101B48003003DBB2092B42D96C2819D0642800F085
:101B5800938024D825281CD063D9582876D06328A8
:101B68001BD131784046B847039A531C0393117828
:101B7800043601340029D7D1204608B0BDE8F087E3
:101B8800039B5A1C03921B78642B7CD02AD8252BE4
:101B980054D1252140460134B847039AC0E7732839
:101BA80033D044D975284FD106F1040E30682B463E
:101BB80000220A217646FEF797FB049A00955346C1
:101BC80039464046FEF7CDFB039A0444A8E704AA29
:101BD80003A922F079F8B7E7D31C039390784FF064
:101BE800010AACE7732B10D05BD9752B3AD0782B50
:101BF80096D1A3F15802B2FA82F2306852092B4604
:101C080010210436FEF770FBD7E73368049A009377
:101C1800394600234046FEF7A4FB04360444039AE1
:101C28007EE70028B9D1204608B0BDE8F0876E28C5
:101C3800B3D1039A336804361C6071E72AD9582B4C
:101C4800D7D0632B8DD06BE77828A6D1A0F15802A6
:101C5800B2FA82F2306852092B461021FEF744FB93
:101C68000436AAE706F1040E30682B4600220A2142
:101C78007646FEF739FBA0E7331D306829461E4635
:101C8800FEF704FB99E7331D306829461E46FEF728
:101C9800FDFA92E7002B7FF443AF204608B0BDE879
:101CA800F0876E2BC6D03BE70EB400B584B005AB09
:101CB800019053F8042B0649039301A8FFF727FF67
:101CC800019B00221A7004B05DF804EB03B0704762
:101CD800610300080FB430B583B006AB0A490B485E
:101CE80053F8042B096800680193FFF710FF084CAC
:101CF800054620680AF0BAFF0028FAD0284603B043
:101D0800BDE8304004B07047782400207C240020CF
:101D1800E8570020DFED2B7AB4EEE70AF1EE10FA6F
:101D28004ADDDFED296A9FED297A01E0B0EE670A06
:101D3800B4EEC70AF1EE10FA70EE667AF6DC9FEDA3
:101D4800247AF4EEC77AF1EE10FA38D5DFED1E6A80
:101D58009FED207A01E0F0EE407AF4EEC77AF1EEDA
:101D680010FA37EEA60AF6D4DFED1B7AB4EEE70ACE
:101D7800F1EE10FA14DDDFED137A37EEC00A60EEEB
:101D8800006A9FED166A9FED167ADFED167AA6EEC9
:101D9800867A20EE266AE6EE877AA6EE270A70474C
:101DA800DFED117AB4EEE70AF1EE10FA44BFDFED89
:101DB800087A37EEC00AE2E7F0EE407ABFE7B0EE05
:101DC800670AD1E7DB0F4940DB0FC940E4CB164176
:101DD800DB0F49C0E4CB16C1DB0FC93F92E741B91D
:101DE8009730083C15A82ABEDB0FC9BF09B909E01E
:101DF800194690FBF1F301FB13030846002BF7D1BA
:101E0800084670470146FBE710B507EE901A2DED1E
:101E1800028BB8EE678ADFED217A28EE008A044645
:101E280028EE278AB0EE480A2AF03CFBF0EE408AFA
:101E3800B0EE480A2AF098FAF7EE007A9FED187A81
:101E4800F0EE675AE8EE875A0023A361B0EE676A9E
:101E5800C7EEA56A63612362E361A8EEC76ABDECB9
:101E6800028B77EEC07AB6EE007AF8EE005A27EECB
:101E7800877A20EE250A27EE267A26EE266A67EE6E
:101E8800A67A20EE260A84ED046AC4ED017A84ED70
:101E9800007A84ED027A84ED030A10BD27D4D23685
:101EA800F304353F10B44C09012250F8243001F0F6
:101EB8001F0102FA01F10B4340F824305DF8044B8E
:101EC80070474B0901F01F0150F82320012303FA42
:101ED80001F1114214BF184600207047074A084B09
:101EE80010781B78074A834296BFC31AC3F1800350
:101EF8000020126818441044704700BF6C68002026
:101F0800E967002038360020064A074B10781B780E
:101F180083428ABFC3F18003C01AC018C0F17F0092
:101F2800704700BF6C680020E967002030B5144C8A
:101F3800237883B01BB90120237003B030BD05227C
:101F480000238DF800208DF8013000BF0D4D2B685F
:101F58009868FFF797F82B6801AA6946586828F02F
:101F6800E7FD2B689868FFF792F800BF9DF80530E9
:101F780003F0010383F00100237003B030BD00BFFC
:101F8800D65D0020C45D002070B5064C0646256865
:101F980003E023685B1BB34203D8FFF7C7FF0028A1
:101FA800F7D070BDF05800202DE9F04F89B0B2F19C
:101FB800000A02900491039340F3B0800B4600227C
:101FC80001EB8A0153F8040B8B420244FAD1039BBC
:101FD8000592002B00F09A80059B002B6AD0544B89
:101FE800059A1B68DFF85C9100920099DAB25118E3
:101FF800B1F5807F8CBFC2F58072009A01924D4A7C
:1020080092689A426DD9190C1A0A4FF002040620F8
:102018008DF81F308DF81E208DF81D108DF81C408E
:10202800FFF7B2FF0620FFF737F8434A0123137082
:1020380000BFD9F800309868FFF724F8D9F80030C5
:1020480007A95868002228F029FD0024049D029E53
:10205800019FA34629684FEA840800220B460134F1
:1020680071B1B9422AD2D9F8000031684068FEF748
:1020780094F82A68336813443360BF1AC5F800B06F
:10208800A24505F1040506F10406E3D1D9F80030AC
:102098009868FEF7FCFF00BF254B019900981B6864
:1020A800421A0092224A0B441360039A32B3009AF0
:1020B800002A9AD1059809B0BDE8F08F029CD9F89A
:1020C800003054F80810586800223B46FEF765F8BF
:1020D80054F808202B683A44DF1B44F808202F6086
:1020E800D4E70598009C1549154A001B05900598EA
:1020F80000230B70137009B0BDE8F08F059B009AA0
:102108009B1A0593059809B0BDE8F08FFFF70EFFFD
:1021180000287FF461AF039B0593CBE7039C1CB9B0
:10212800FFF704FF0594C5E700230593C2E700BF46
:102138003836002078140020D65D00206C68002016
:10214800E9670020C45D002070B5104D104E2B7853
:1021580031788B4284B016D00E4A03921A44029208
:102168008CBF0C46CA1A04A98CBFC3F18002002494
:10217800012341F8102D02A802220194FFF714FF51
:10218800002333702B7004B070BD00BFE9670020D6
:102198006C680020EC67002070B5194C194D237845
:1021A8002978994284B027D0174A03921A44029298
:1021B80034BF0E46CA1A04A934BFC3F180020026F0
:1021C800002341F8102D02A802220196FFF7ECFE29
:1021D80023781844C0B203062B7848BF80F08000EB
:1021E8008342207002D0002004B070BD002301207B
:1021F8002B70237004B070BD012004B070BD00BF07
:10220800E96700206C680020EC67002008B545F2FB
:102218000820FFF7B9FE0620FEF73EFF064B012215
:10222800C7201A70FEF738FF04480549054A0023FD
:1022380003700B70136008BDD65D00206C68002029
:10224800E9670020383600202DE9F04182B00346C6
:10225800060C050A032406208DF807308846174621
:102268008DF805608DF806508DF80440FFF78CFE58
:10227800C0B100BF0D4C23689868FEF703FF2368C0
:1022880001A95868002228F009FC23684246002169
:1022980058683B46FDF781FF23689868FEF7F7FE0C
:1022A80000BF384602B0BDE8F08100BFC45D002021
:1022B800F0B5124B9D6885B00DB905B0F0BDED0ABB
:1022C80014D0002704AE7C196410E002102269467D
:1022D800FFF7BAFF0F2809DD6B4653F8042B0132CC
:1022E8000AD1B342F9D12546AF42ECDBFFF72CFF08
:1022F800034BED021D60E0E7671CF5E7781400204A
:10230800383600200F4A138823F040031B041B0CA7
:10231800138013889BB223F0380343F030031380F3
:1023280013889BB243F04003138044F6BD7244F215
:102338007D0300280CBF18461046400140F01700E6
:10234800FEF7BEBE00300140144A38B5138823F0AA
:1023580040031B041B0C138013889BB223F0380323
:1023680043F03003138013889BB243F040030446C4
:10237800138043F210200D46FEF7A2FE042CA8BFDE
:102388000424E400072DD4BF6119E11D044C04EBBB
:102398008101BDE83840086DFEF792BE003001406B
:1023A80094E70208B0F1FF3F0AD0022810B403DC1A
:1023B8005DF8044BFEF762B900205DF8044B7047E6
:1023C80000207047F0B55B4B5B4A97B019689142A3
:1023D80000AF00F0A3805949594A00234FF4700018
:1023E800C1F888003B607B60136843F48033136056
:1023F80003E03B68B3F5A04F09D0136803F400333A
:102408007B603B6801333B607B68002BF1D04C4B11
:102418001B6813F4003318BF01237B607B68012B12
:1024280052D0464C464B474AE260474A596A1160C7
:102438005A6A42F080725A625A6942F4FC025A613E
:102448000025032207F10801012341F6FF764FF02A
:102458009040FD60BE603A73BB7316F0CBFD4FF63B
:10246800FF7307F108013948BB6016F0C3FD07F197
:1024780008013748374E16F0BDFD07F10801364808
:1024880016F0B8FD07F10801344816F0B3FD07F15E
:102498000801334816F0AEFD07F1080016F0BAFB44
:1024A800BB683049304AA1FB031330499B0CF0202C
:1024B8004FF0070E5C370B60566084F82300956078
:1024C800C2F800E0BD46F0BD294A1D4B122111603B
:1024D8005A685A605A685A605A6842F480625A6068
:1024E8005A6822F47C125A605A6842F4E8125A6018
:1024F8001A6842F080721A601A689201FCD559680D
:102508000F4A21F003015960596841F002015960EE
:10251800536803F00C03082BFAD182E700221A60F3
:1025280062B6144B1B6883F30888134B1B689847E3
:10253800FEE700BFFC9F0020EFBEADDE00ED00E02F
:10254800001002400005FA05044F0020000400486E
:10255800000800483F190100000C0048001000481E
:102568000014004883DE1B4310E000E0F45800200C
:102578000020024000D8FF1F04D8FF1F70B50F4C81
:102588000F4DC0EBC00004EB800468692669304336
:10259800686182B09209667BA1600025012101A8CB
:1025A80063618DF804608DF805208DF806508DF86C
:1025B80007101FF0AFFE02B070BD00BFA4120020CC
:1025C80000100240074BC0EBC00030B403EB8000A2
:1025D800054C056963692B4363610176427630BC1B
:1025E800704700BFA4120020001002402DE9F04FF0
:1025F8005E4C54F8204083B0002C71D0666D98462C
:1026080091465B4B7268E264A160236004F15A0151
:102618004FF4807304F5AD726161A261E3602361D8
:102628000746307E22F06EFCF068A8B1514B0021BD
:102638005A68904203F11C0300F0928001310C2982
:10264800F6D100207A1CD2B20C21FFF7BBFFE36C55
:10265800F26822632433A364B068D8B1454B0021E3
:102668005A68904203F11C0378D001310C29F7D144
:1026780000257A1CD2B20B212846FFF7A3FF234678
:10268800F27E3D492846FFF779FFE36CB268626342
:102698002833636494F8590009F0D0FB054694F890
:1026A800580009F0CBFB18F0080F824696F819B0CD
:1026B8001AD0CDB118F0110F4FF00B0307F1010735
:1026C80014BF4E213E21EF715A46AB712846FEF7E2
:1026D800E4F818F0010F45D0236B5BB3636B4BB381
:1026E800204603B0BDE8F08F18F0010F0CBF4FF083
:1026F8002E084FF04E0819F0020F09D045B10B22F1
:102708007B1CAA71EB7128465A464146FEF7C5F86C
:1027180019F0010FE0D0BAF1000FDDD001370C231A
:102728008AF807705A4641468AF806305046FEF73E
:10273800B4F8D1E7337FB27E8DF804209B090021DD
:10274800012201A88DF805308DF806108DF80720B4
:102758001FF0E0FD204603B0BDE8F08FCDB288E75A
:10276800C8B26FE72846FEF78DFCB5E78424002041
:1027780084E80208A4120020810800080348D0F861
:102788003C3113B100F59A7018477047A412002025
:102798000348D0F8203113B100F58C701847704702
:1027A800A41200200348D0F804310BB1FC301847BC
:1027B800704700BFA41200200348D0F8E8300BB1DE
:1027C800E0301847704700BFA41200200348D0F833
:1027D800CC300BB1C4301847704700BFA41200209A
:1027E8000348D0F8B0300BB1A8301847704700BF85
:1027F800A41200200348D0F894300BB18C3018474D
:10280800704700BFA41200200248836F0BB17030DC
:1028180018477047A41200200248C36D0BB154300A
:1028280018477047A41200200248036C0BB13830D7
:1028380018477047A41200200248436A0BB11C30A5
:1028480018477047A41200200248836803B118474C
:10285800704700BFA41200201749184B184A19489E
:1028680010B4D1F8884044F47004C1F888401C685A
:1028780044F001041C605C6822405A601A6822F027
:10288800847222F480321A601A6822F480221A6054
:102898005A6822F4FE025A60DA6A22F00F02DA62FB
:1028A8001A6B002410404FF0006218639C608A6025
:1028B8005DF8044B704700BF00ED00E000100240D7
:1028C8000CC07FF8CCFC00FF2DE9F04F2DED028BFA
:1028D80093B0834618F06EFFB54B1D7825B113B041
:1028E800BDEC028BBDE8F08FB24B1B685C05F6D5DA
:1028F800B14FB24E3B68002B56D0B14C3168D4F87A
:1029080010218A1A7C2A4FD994F81421DFF8FC8206
:102918009FEDAC8AC4F81011013284F814214FF0ED
:10292800240A5E20984750463B689847A64BF8EC27
:10293800016A9B8A07EE103AF8EEE66AB8EEC77AA3
:102948000AF1010AC6EE877A5FFA8AFA67EE887A90
:10295800FDEEE77ACDED027ABDF908905FFA89F0CD
:1029680016F03CFFC9F3072016F038FFBAF1270F1D
:102978003B68D6D15E2098473B68302098470020B6
:1029880016F02CFF002016F029FF3B685E209847C0
:1029980094F8143113F0030800F08481580701F00B
:1029A8003682282B01F03283884B1B78002B72D09B
:1029B800834C874AD4F81831ABEB0303934200F2F7
:1029C8007B8794F82091B9F1000F35D1DFF8408268
:1029D800D8F800000AF056F9C0B201280FD9022829
:1029E8007C4F41F0A5833B78002B41F02A86D4F830
:1029F8002431ABEB0303B3F57A6F81F09D87D4F8EC
:102A08002831002B47D094F82031C3B9724B1B688A
:102A18009B7801211E3B00228B4284F8201184F808
:102A2800342141F22E87D8F800000221043016F034
:102A38004BFE94F82C3111E0D4F828315BB3D4F86C
:102A4800303140F6B732ABEB0303934223D994F805
:102A58002C31002B01F0C382DFF8B481013BDBB2DB
:102A680084F82C31002B00F08287D4F8287194F870
:102A7800342117F8011B94F83531D8F80000C4F850
:102A880028710A44013384F8342184F835310AF076
:102A9800FDF8C4F830B1514BD6F800801B7843B12B
:102AA8004F4F386828B14F4B1B78013B012B40F240
:102AB8006E874D4B1B7863B14C4F3B684BB1404C14
:102AC800D6F80090D4F84C31A9EB0303632B00F23D
:102AD8001C81DFF8408198F80030022B01F05E82FB
:102AE8003C4F97F87430032B00F02B87404B1B7832
:102AF80073B1404D2B685BB1314C09F013FED4F82B
:102B08005831029044F61F62C31A934200F258816A
:102B1800394B1B78002B7FD1384B1B7843B1284C9D
:102B2800D4F8A83203F5C333A0339B4580F07286EE
:102B3800334B1B78002B3FF4D2AE214E314C324D33
:102B480006F2C92720680AF09DF800283FF4C7AEAE
:102B580020680AF08FF82B7880465A1E33B1206817
:102B68002A700AF08FF80028F2D1B8E60322394615
:102B7800781E2BF03CFD96F8C83296F8C92286F8E4
:102B8800CB8283F47F4383F0FF039B1A1FFA88F8F4
:102B98009BB2B8EB132FD5D196F8CA22DBB29A4272
:102BA800D0D1781E16F00EFB2B7818442870C9E790
:102BB80091650020444D0020F0330020F05800209B
:102BC8009816002000007A44E46500201A39002095
:102BD8003F0D030000000020EC3300201C390020CA
:102BE8009C310020243900202C390020A0590020D5
:102BF80034390020383900207839002089390020FC
:102C08003E39002044390020483900201C66002045
:102C1800E8330020764400205B4C2278A2B15B4B5D
:102C28009B7A53B109F07EFD594B1B68C31AA3F573
:102C38007A73B3F5FA6F07D82278564B5649186855
:102C480009F0F0FF00232370544CD4F8A03203F5A8
:102C5800C333A0339B45FFF45FAF514DC4F8A0B216
:102C68002B78002B41F030834E4D2B78002B41F010
:102C78001D824D4994F8A4228D5CE90701F1E7848F
:102C8800AA0701F1A1846B0701F19983474A94F8D7
:102C9800A4321178013393FBF1F201FB123384F86B
:102CA800A43239E7D4F8102141F288339A4201F26C
:102CB80016823B685E2098473B68142098473C4B37
:102CC8003C4AB3F9043082FB03124FEAE378C8EBBD
:102CD800A2080FFA88F85FFA88F016F07FFDC8F3AB
:102CE800072016F07BFD3B685E2098473B681C2058
:102CF8009847002016F072FD002016F06FFD3B6823
:102D08005E20984794F8143148E6DFF8A4A0DFF86D
:102D1800A480412016F088FCBAF9023088FB032011
:102D2800DB17C3EBA00080B216F064FCBAF90030E0
:102D380088FB0320DB17C3EBA00080B216F05AFC17
:102D4800BAF9043088FB0320DB17C3EBA00080B27C
:102D580016F050FC184B3868197809F097FF94F86A
:102D6800503113F0010801F0F481144AC4F84C9171
:102D78000133DBB2A2FB0312D20802EB8202A3EBFF
:102D8800420384F85031A4E60C390020D84E0020C4
:102D9800EC3C00207C390020CC380020981600201C
:102DA80080390020813900208439002088390020AA
:102DB8002C66002067666666C05D0020CDCCCCCC52
:102DC80094F85E31002B41F06C81DB4B1A6802F0FD
:102DD8000803002B48F603414AF60B404BF60F4315
:102DE80049F6074704BF03460F4612F0040F4FF099
:102DF800190118BF1F46920684F85E1103D547F4DF
:102E0800804747F02007CD4B5A79C7F30909002AB4
:102E180041F0BF859B79002B41F0AA869846642033
:102E28004FF0FF3A4FF0000C0A970B97ADF834C0FB
:102E3800CDF83AC0CDF83EC0CDF842C0CDF83090BC
:102E4800ADF83680ADF838A08DF846000AAF0FCF40
:102E5800DFF800E384F805C0AEE80F0097E80F003C
:102E6800AEE807002EF8023B71464FF0010C1B0C30
:102E7800FE271F20C82201F81E39A770A27184F806
:102E880007C0E07094F86E01207180F0F10383EAC6
:102E98000313DAB2130983F0E70343EA022383EA50
:102EA800C2031BB283EA0312D2B2C3F3072383EA35
:102EB800121343EA022383EAC2031BB283F0C80257
:102EC80082EA0212D2B2C3F3072383EA121343EA57
:102ED800022383EAC2031BB283EA0C0787EA0717B7
:102EE800FFB2C3F3072282EA171242EA072200EB75
:102EF8000C0382EAC7070EEB0C0084F86E312780BA
:102F080011F8013B7B4083EA0313DBB21A0982EA1A
:102F1800172242EA032282EAC3031BB29FB281420C
:102F28002780EDD183F07C0383EA0313DBB24FEAF9
:102F3800131E8EEA172E8EEA032E8EEAC30E0FFAA0
:102F48008EFE1FFA8EFADFF810C2A4F800A05FFA0E
:102F58008EFE4FEA1A2A84F828A084F827E00CF598
:102F6800CB7804F12209DCF80000DCF80410DCF866
:102F78000820DCF80C3047460FC70CF1100CCC4584
:102F8800B846F0D1DCF8000038606D4F9CF804308A
:102F980088F8043007F1270884F8BDE184F8BEA159
:102FA80017F8011F286809F071FEB845F8D194F8A0
:102FB8005F31002B41F070806249326809780A203D
:102FC80084F85F01002901F0F0815F4F01293888FA
:102FD800069041F2C1850229B7F802E001F0F484B5
:102FE800B8880590032901F0CE85F8880490042953
:102FF80001F0DC850529388901F0D3850629B7F861
:103008000A9001F0CA850729B7F80C8001F0C2853B
:10301800FB89039394F86E110A920B4683F03002F1
:1030280082EA0212D2B217094849079387F07A0751
:1030380047EA02270988237187EAC202444FC1EB95
:10304800012187FB013A069B4FF0000C63F30F0C3C
:10305800059B6EF31F4C4FF0000E63F30F0E049B9D
:10306800CDF82CC012B28A440027C91763F31F4E4B
:10307800C1EB6A2A039BCDF830E082EA021160F3C3
:103088000F070020C9B268F30F00C2F3072269F3E3
:103098001F4782EA111263F31F404FF000090D9792
:1030A8008DF83DA00E908DF83C9042EA01220DF17A
:1030B800280C82EAC107BCE80F003FB287F0C808B5
:1030C80088EA0818DFF88CE084F805905FFA88F839
:1030D800C7F30727AEE80F0087EA181747EA08235F
:1030E8009CE8030083EAC8031BB283F023024EF86E
:1030F800040B82EA0212D2B2C3F30723079F83EAC2
:103108001213704643EA022383EAC20207F1010C54
:1031180020F814194FF023081621FE27C82384F835
:103128006EC1228084F807800EF1020EA770E1704C
:10313800A371114612E000BFE06500204C66002034
:103148002F180020346600201C5D002084380020E1
:1031580003082080A01600209A16002010F8013BD2
:103168004B4083EA0313DBB21A0982EA112242EACE
:10317800032282EAC3031BB299B270452180EDD1C4
:1031880083F0F40383EA0313DBB24FEA131E8EEADB
:10319800112E8EEA032E8EEAC30E0FFA8EFE1FFA48
:1031A8008EF8E64FA4F800804FEA182C5FFA8EFEDE
:1031B80084F81EE084F81FC07968BA683868FB682C
:1031C80007F5CB78A8E80F0038697969BA6904F27D
:1031D8009717A8E8070004F2B51884F8B5C184F871
:1031E800B4E117F8011F286809F050FDB845F8D177
:1031F80094F866C1BCF1000F40F04887D04B94F8B2
:103208006E71B3F90010B3F90220B3F904309FEDE1
:10321800CD6ADFF840E384F805C007EE103A33685A
:103228000A9387F06A0383EA031306EE901AD9B269
:103238000B0983F0D50343EA012383EAC1031BB2D8
:1032480083EA03115242C9B207EE902AC3F3072357
:1032580083EA111343EA0123F8EEE77AF8EEE66A07
:10326800B8EEC77A83EAC1031BB267EE867A66EEC8
:10327800866A27EE067A002083F0C808CDED0C7A1E
:10328800CDED0B6A8DED0D7A0E900F90109088EAB7
:1032980008160DF12809F6B2C3F30728B9E80F009C
:1032A80088EA161848EA062888EAC6080FFA88F84D
:1032B800AEE80F0088F01E0699E8070086EA0616B1
:1032C800F6B2C8F3072383EA161343EA06238EE807
:1032D800070083EAC6061C20C8214FF005084FF0F6
:1032E8001E0CFE237A1CE070A17184F8668184F8B4
:1032F80007C0A370AEF1100127710EF10C002680F3
:1033080084F86E2111F8013B734083EA0313DBB2A2
:103318001A0982EA162242EA032282EAC3031BB28E
:103328009EB281422680EDD183F0270383EA0313FE
:10333800DBB24FEA131E8EEA162E8EEA032E8EEAB1
:10334800C30E0FFA8EFE1FFA8EFC7C4FA4F800C045
:103358005FFA8EFE4FEA1C2C84F825C084F824E01E
:1033680007F5CB7804F1220938687968BA68FB68F0
:1033780046460FC610374F45B046F5D1724E3B88CA
:10338800A8F8003006F1240784F8BAE184F8BBC134
:1033980016F8011F286809F079FCB742F8D194F8AB
:1033A80067A1BAF1000F40F06B8694F86E81644B08
:1033B800664AB3F90410B2F90620654EDFF898E1C1
:1033C800644F84F805A088F0220080EA0010C0B29B
:1033D800030983F0590343EA002383EAC0031BB2BD
:1033E800B2F5FA6F83EA0310C0B2A8BF4FF4FA62CD
:1033F800C3F30723B2F57A7F83EA101343EA002365
:10340800B8BF4FF47A7283EAC000A2F57A726423D7
:1034180003FB02F28EFB023ED31786FB0162C9173B
:103428004FF0000CC3EBAE13C1EBA201CDF828C0DE
:1034380006B2CDF82CC0CDF830C0CDF834C0ADF808
:103448003A30ADF838100DF1280CBCE80F0086F0C2
:10345800C80E8EEA0E1E5FFA8EFEC6F3072686EAAF
:103468001E1646EA0E260FC786EACE0636B286F044
:103478004A0383EA0313DBB2C6F3072181EA131177
:103488003A46DCF800E042F810E941EA032108F185
:10349800010681EAC30305204A214FF0FE0C84F897
:1034A8006E614FF0C80E142684F8670184F8048012
:1034B80023800437E17184F802C0E67084F806E0DE
:1034C800184612F8011B414081EA0111C9B20B09E3
:1034D80083EA102343EA012383EAC10109B288B2CF
:1034E800BA422080EDD181F0140181EA0111C9B2FC
:1034F8004FEA111E8EEA102E8EEA012E8EEAC10EB8
:103508000FFA8EFE1FFA8EF60C4F26804FEA162908
:103518005FFA8EFE84F81D9084F81CE0796838689C
:10352800BA68FB68B7F8188007F5CB7CACE80F00E1
:1035380038697969ACE8030010E000BF9A160020EA
:103548002C66002088C3E43A2F1800201C5D002058
:1035580067666666A0160020D34D621004F29716BF
:10356800ACF8008084F8B391B04684F8B2E104F274
:10357800B31918F8011F286809F088FBC145F8D16C
:10358800C44BC54A1B781278013B12F00100DBB22C
:1035980014BFC0214021172B03D8C04A134493F805
:1035A80030A0BF4B1A8893071ABF002341F01001BF
:1035B800012312F4027F18BF022312F0100F18BF64
:1035C800062312F0200F18BF1023002841F08C8129
:1035D8004FF0030C94F86E910A9389F0460383EA3E
:1035E8000313DAB2130983F0920343EA022383EA4E
:1035F800C2031BB283EA0310C0B2C3F3072282EAF4
:10360800101242EA002282EAC00212B282F0C80E08
:103618008EEA0E1E5FFA8EFEC2F30722002382EAAC
:103628001E1203208DF82CA08DF82FC08DF82D3098
:1036380042EA0E2C8DF82E108DF830000AAA07CA1F
:103648008CEACE0E0FFA8EFEDFF868A2E3718EEADE
:103658000E1CAAE803005FFA8CFCCEF3072E8EEA54
:103668001C1E4EEA0C2181EACC0C94F808E08AF87A
:1036780000200FFA8CFC8EEA0C0E8EEA0E1E5FFA02
:103688008EFECCF3072282EA1E1242EA0E22607AEC
:10369800A17A94F80BC0637182EACE0212B250404C
:1036A80080EA001E5FFA8EFEC2F3072080EA1E1031
:1036B80040EA0E2080EACE0000B2414081EA0111C2
:1036C800C9B2C0F3072282EA111242EA012282EA51
:1036D800C10212B28CEA020C8CEA0C1C5FFA8CFC58
:1036E800C2F3072282EA1C1242EA0C2294F80CE088
:1036F800607BA17B94F8108084F8049082EACC0265
:1037080012B28EEA020E8EEA0E1E5FFA8EFEC2F327
:10371800072282EA1E1242EA0E2282EACE0212B280
:10372800504080EA0010C0B2C2F3072282EA1012A9
:1037380042EA002282EAC00212B2514081EA011133
:10374800C9B2C2F3072282EA111242EA012282EACE
:10375800C102E17B13B281EA030282EA0212D2B209
:10376800C3F3072383EA121343EA022383EAC2035B
:103778001BB288EA030282EA0212D2B2C3F3072319
:1037880083EA121343EA022383EAC2031BB283F0DB
:10379800320282EA0212D2B2C3F3072383EA121377
:1037A80043EA022383EAC2031BB29AB24FF0FE0C2B
:1037B8004FF0090EC82009F10101DBB284F802C0FC
:1037C80084F803E04FEA122CA07184F86E1122806D
:1037D80084F812C0637438687968BA68B7F80C90CE
:1037E8000AF5C47EAEE807000AF5CC7A8EF80280A6
:1037F800AEF8009084F8A8C184F8A73116F8011F24
:10380800286809F043FAB245F8D1029BC4F8583148
:10381800FFF77EB994F8AC32204AC4F8A8B202EB9C
:103828008302926C42B312AD04F2B3231D4E45F8E5
:10383800203D002104F2C52331800B9380211523FC
:10384800A52784F8B232284684F8B11284F8B072F9
:10385800904728463188FEF750F90A9D124804F52A
:103868002C716D1A152DA8BF15252A4628F05AFC6B
:103878000E4A94F8AC3215700D4A013382FB0312DC
:10388800A2EBE37202EB42029B1A84F8AC32FFF718
:103898004FB900BF50360020A4310020ACE8020820
:1038A8008638002040370020803B0020953B0020D0
:1038B80056555555A0160020D34AD44B92F80BE024
:1038C8003168D4F81C211B88D148891A4FF47A72C0
:1038D800DFB202FB0EF21B0A8777077591424FF0A1
:1038E8000007C37743758770077180F01284C94B4E
:1038F800C9491A689B68C4F818B181FB02E7D21756
:1039080081FB03E1C2EBA702DB17C3EBA103111292
:103918004FEA232C4FF0F40E02770127417780F805
:10392800203030217522782380F821C080F81AE0F1
:10393800C77680F8221080F8232080F82430FFF71B
:1039480040B8DFF8F492D9F8000009F08FF90028A0
:103958003FF4CCA8D9F80000012109F083F902222C
:10396800002387F8742088F80030FFF7BFB894F870
:10397800341194F83531D8F800004A1C013384F822
:10398800342184F8353109F081F9FFF782B8A34C66
:10399800DFF8A8924FF0000A0AE01B2B00F014830E
:1039A8000D2B00F012824FF0010389F801303868BE
:1039B80009F068F9002838D0386809F05BF983B253
:1039C8007E2B32682AD099F801100029EFD194F89B
:1039D8003621002AE1D07D2B00F00C8294F844E1D6
:1039E800BEF1000F04D080F02003DBB284F844114C
:1039F800511CC9B22244092984F8361182F8383199
:103A080000F0EC810829D2D8B4F84221134403EB22
:103A1800132303F0FF03A4F84231C8E784F836A162
:103A280084F837A189F801A0C1E794F8453133B18A
:103A380094F8393184F84501302B00F0498794F81F
:103A48003721774BDFF8F8C1DFF8F8E1DFF8F8A1A4
:103A58000127104600283FF42CA83268A2EB080280
:103A6800012A00F2AD8194F84691B9F1000F40F0B7
:103A7800C28294F8471133F8112012B984F84771BB
:103A8800E8E70131B2F5826F84F8471100F002814E
:103A98001FD9B2F5E26F00F09A8034D9B2F5046FFD
:103AA80000F0A480B2F5116F00F04781B2F5E46F21
:103AB800D0D110465B4A176C918A642303FB07F345
:103AC80093FBF1F115F0E6FD002384F83731FEF79A
:103AD800F0BFB2F5007F00F0B9802CD8B2F5807F36
:103AE80000F04581B2F5887FB4D1DCF80020520798
:103AF800B0D500214FF4887015F0CCFD002384F870
:103B08003731FEF7D6BFB2F5C06F00F0B380B2F51B
:103B1800E06F9FD1434A906B918A642303FB00F3C3
:103B28004FF4E06093FBF1F115F0B4FD002384F845
:103B38003731FEF7BEBFB2F5047F00F02781B2F53A
:103B4800806F87D194F848310133DBB2032B00F240
:103B5800588142F2107184F8483101FB03F1324B6D
:103B68001B88002B40F04B810131304B1B78DF075D
:103B78002F4B1B8848BF0431D80748BF0A319A0722
:103B880048BF14311F0648BF2831D80548BF28311F
:103B98005A0748BF64311F0748BFC831980548BF56
:103BA80001F5C8719A0648BF01F57A71DF0648BF6A
:103BB80001F5FA61580648BF01F57A614FF4806053
:103BC80015F068FD002384F83731FEF772BF104600
:103BD800144AD76B918A642303FB07F393FBF1F133
:103BE80015F058FD84F83791FEF763BF114BB3F910
:103BF800041001EB81011046490015F04BFD84F8D3
:103C08003791FEF756BF00BF1C3200201432002047
:103C18004C390020443700206766666698160020F5
:103C2800ACE80208E465002080660020A43100208A
:103C3800863800202C660020FC440020000000206C
:103C4800E06500204C6600202A3200209EF806100D
:103C580000293FF4FFAEC44BC4491B68104681FBE2
:103C68000321DB17C3EBA10115F014FD84F837918C
:103C7800FEF71FBF9EF80620002A3FF4EBAEBA4BB2
:103C88004FF4C060996815F005FD002384F83731BA
:103C9800FEF70FBFDCF8002012F020097FF4DAAE3F
:103CA800B34A1168090600F1F585B24A127B002A69
:103CB8003FF4D0AE94F84911032900F29486DFE866
:103CC80001F032281902AC4B1B6859799A79DB79D3
:103CD80001F1407101EB022101EB0341002384F85B
:103CE80049314FF4826015F0D5FC002384F8373150
:103CF800FEF7DFBEA14B1A68137A507992781B043D
:103D080003EB002313444A1C84F8492103EB0161A7
:103D1800E7E79A4B1A68D379107952781B0403EBBA
:103D280000231344EFE7954B1A689379D0781278FB
:103D38001B0403EB00231344E5E79EF80520002A43
:103D48003FF488AE9AF8001000293FF483AE8C4BFC
:103D58001B8803EB83035B004FF4116093FBF1F1C5
:103D680015F098FC002384F83731FEF7A2BEDCF882
:103D7800002051077FF56EAE00214FF4807015F0DA
:103D880089FC002384F83731FEF793BE9EF805209E
:103D9800002A3FF45FAE9AF8001000293FF45AAEAB
:103DA800744B5B7B002B00F09B85754B1B8893FB4A
:103DB800F1F101EB810149004FF4047015F06AFC40
:103DC800002384F83731FEF774BE4FF0010184F800
:103DD800361184F83831A4F84221E8E5B4F84221D4
:103DE800C2F1FF0293427FF4DEAD4FF0010384F885
:103DF8004531D8E54FF0010384F84431D7E5023165
:103E0800B3E6012384F8483142F21071A7E63B6813
:103E18005E2098473B68022098475A4B534AB3F9AB
:103E2800503082FB03124FEAE378C8EBA2080FFA7E
:103E380088F85FFA88F015F0D1FCC8F3072015F070
:103E4800CDFC3B685E2098473B68032098474E4B63
:103E58001B78D90740F1318125F08CFD4B4B9FED44
:103E68004C7AD3ED037A67EE877AFCEEE77ACDEDEC
:103E7800027ABDF80830002800F02285D8B24FEA4F
:103E8800132815F0ABFC404615F0A8FCDFF80881B4
:103E980098F80530002B40F0C4820AA93D4815F077
:103EA80061FC3B685E2098473B6813209847BDF942
:103EB80028805FFA88F015F091FCC8F3072015F008
:103EC8008DFC3B685E2098473B681B209847BDF9EE
:103ED8002A805FFA88F015F081FCC8F3072015F0F6
:103EE8007DFC3B685E2098473B68232098474E201E
:103EF80015F074FC002015F071FC0AA9254815F08E
:103F080031FC3B685E2098473B6812209847BDF912
:103F180028805FFA88F015F061FCC8F3072015F0D7
:103F28005DFC3B685E2098473B681A209847BDF9BE
:103F38002A805FFA88F015F051FCC8F3072015F0C5
:103F48004DFC3B685E2098473B68222098474520F7
:103F580015F044FC002015F041FC3B685E209847B2
:103F680094F81431FEF71DBD443700206766666675
:103F7800444D00201C320020E8660020B86500206F
:103F880014320020B04A0020A43100202C32002036
:103F9800CDCC4C3E809698004C66002008F0C2FBC1
:103FA800B54B1B68C01A40F6B833984200F2C68079
:103FB800DFF804A39AF804303A2B00F09283002328
:103FC80088F80030FEF792BD386808F05BFE0028DC
:103FD8007FF4E9AC4FF0010384F83731E7E4C4F823
:103FE800283184F82031DFF8D48215F0A1FB94F849
:103FF8002C31FEF733BDA149062015F06DF90023D9
:1040080084F8460184F83731FEF753BD4FF00009B4
:104018003B6884F814915E203468DFF8A4829847DE
:104028003B6817209847484615F0D8FB944BA3FBEC
:1040380004239B0BA8FB03125209C2EB0212A3EB49
:104048008203D8B215F0CAFB3B685E2098473B68EC
:10405800182098478B4BA3FB04239B09A8FB03124A
:104068005209C2EB0212A3EB8203D8B215F0B6FBD9
:10407800484615F0B3FB3B685E209847FEF794BCB2
:104088000AF1FF3A84F867A1FFF7BFBB0CF1FF3CC8
:1040980084F866C1FFF783B9013B84F85F31FFF705
:1040A800A7B8013B84F85E31FEF781BF76493A2014
:1040B80015F012F92870FEF72FBDDFF80882734B50
:1040C800B8F80890A3FB09394FEA99095FFA89F013
:1040D80015F084FB4FEA192015F080FBD8E63B6801
:1040E8005E2098473B6810209847404615F076FBBD
:1040F800404615F073FB3B685E2098473B682120DB
:104108009847404615F06AFB404615F067FBFEF7F6
:10411800D0BD5F4B32681B78C4F81C21013B012BD2
:104128003FF6E5AB1022022382700371FFF7DFBB75
:1041380015F0EEFA01233B70FEF761BC554AB2F860
:10414800523100210133A2F8523188F80010FEF7ED
:10415800CDBC514B1B88DA0515D4D80600F1308444
:10416800990600F13C845A0600F14884180700F1CA
:104178005284D90700F1EC8413F0020F0CBF4FF002
:1041880004084FF00C08454B454A1B78D27803F0D9
:1041980001030AB143F002035320029315F044FAD5
:1041A800404A128802EB820202EB8202900080B23F
:1041B80015F020FA002015F01DFA3B4A3B491288F9
:1041C8003868C2EBC212520081FB023111444FEA37
:1041D800E27ACAEB612A5FFA8AFA514608F056FD7C
:1041E800334B38681A78029B48EA0308304B8AEA4E
:1041F800020A002183F800A008F048FD414638680B
:1042080008F044FD2A4B2A4A1B78386888EA0303D9
:10421800DBB21946137008F039FD94F85031002BC1
:104228007EF4A3AD4F2015F0FFF922F063F822F0D9
:1042380061F822F05FF80121386808F027FD1D4A6F
:104248001B4B92F800801B78194A386808F001085F
:1042580083F001034146137008F018FD144B144A0B
:104268001B78386888EA03031946137008F00EFDB6
:1042780094F85031FEF779BD7C44002097960108E8
:1042880073B2E745D34D62103DB70108CDCCCCCC15
:104298008A3800209816002086380020A431002093
:1042A8005C66002014320020843800200308208037
:1042B800C05D00202834002064440020E83300203A
:1042C800898888884C660020AE4EAF4B0093002446
:1042D800A6F13F01AD4BAE4A089106F8404CAD49F6
:1042E80009960AA8FDF7E0FC089E731C0893347031
:1042F800089B2922591C08911A70089BEA22591C0C
:1043080008911A70089BC822591C08910AA81A70AB
:1043180026F0D6FF471C0AA93A46089827F002FF5C
:10432800089AD31901330893D455089B5A1C08924C
:104338001C70089B5A1C08921C70089B5A1C0892F7
:104348001C70089B5A1C08921C70089B5A1C0892E7
:104358001C70089B5A1C08921C70089B5A1C0892D7
:104368001C70089B5A1C08921C70089B5A1C0892C7
:104378001C70089B5A1C08921C70089B5A1C0892B7
:104388001C70089BFF22591C08911A70089B012277
:10439800991812A808911A7050F8283D9B1B337081
:1043A80017F098F92C70FEF7B7BB8846894608467F
:1043B800049105918E4606910391FEF72BBE764A2D
:1043C800704B12680B93A3F1400500202121D70000
:1043D80003F8400CA97040F1D08270490326704B55
:1043E8001B88580500F1C682DA0700F1F58203F050
:1043F80002036C4A002B1CBF032611466A4F324643
:10440800384627F08FFEF31912A80133B91E40F879
:10441800203D00225B1AF2556B7017F05BF9FEF72E
:1044280035BC624B93F800A0BAF1000F3FF435ADEC
:104438005F4AB4F816E111883B6802924FEA0E1EF3
:1044480064201FFA8EFE00FB01A14FEA4A00B1FB6F
:10445800F0F14EEA012E1FFA8EFEC1F303215E2011
:104468004EEA010998473B68062098475FFA89F0A9
:1044780015F0B4F94FEA192015F0B0F9B4F816316F
:10448800029A4C49B2F800904A7A01339BB2012A49
:1044980093FBFAF00AFB1033A4F8163100F04983B5
:1044A8006E2345484A7B03FB09F380FB03014FEA6F
:1044B800E379C9EBA1092AB13C4B1FFA89F91B78AA
:1044C80099FBF3F93B68DFF8FCA05E2098471FFAD8
:1044D80089F93B683A209847AAFB093A4FEA5A1AE1
:1044E8001FFA8AF3D8B2029315F078F9029B180ADA
:1044F80015F074F93B685E2098473B683B20984765
:10450800642303FB1A939BB22C48053380FB0320DA
:10451800DB17C3EBA000C0B215F060F9002015F05E
:104528005DF93B68DFF898A0DFF890905E20984727
:104538003B6828209847DAF8003089FB0329DB1705
:10454800C3EBA9095FFA89F015F048F9C9F3072008
:1045580015F044F93B685E2098473B68042098476B
:10456800B8F80830002B40F04D82DAF8083083F3B1
:1045780010085FFA88F015F031F9C8F3072015F034
:104588002DF98AE4CC380020B1650020981303087F
:10459800A0130308AC130308203400207C1303087D
:1045A80086380020941303088F3800202A32002010
:1045B800143200201C320020310CC3306766666656
:1045C800443700201F85EB51CC4ACD4B0B9212AEDD
:1045D800A2F13D0046F8200D1988CA4FA2F1400308
:1045E80000204FF00A0E02F8400C082283F801E080
:1045F80030469A70FDF75DFA3B68C349DA1781FBCC
:104608000313C2EBA30399B23046FDF752FA0CF03C
:104618000BFBBF680A9B3A0C591C0A911A700A9B3B
:104628003A0A591C0A911A700A9B5A1C0A921F705E
:104638000A9B5A1C0A921870304617F04BF8FEF77E
:1046480022BBC4F824B187F80090FEF7D8B9AF4F61
:104658009FEDAF8AB7F90220A8480B9007EE902A81
:10466800F8EEE77A12AE67EE887AA0F13D01FDEE2A
:10467800E77A46F8201D00F8403C0823CDED027A81
:1046880000F83F3C1E23BDF8081000F83E3C3046B9
:10469800FDF70FFAB7F9003007EE903AF8EEE77A2F
:1046A800304667EE887AFDEEE77ACDED027ABDF8FE
:1046B8000810FDF7FEF9B7F9043007EE903AF8EE66
:1046C800E77A304667EE887AFDEEE77ACDED027A32
:1046D800BDF80810FDF7EDF9304616F0FBFFFEF7C0
:1046E800CFBA9AF80240C4B1013CE4B20134544450
:1046F8005146002211F8013B534083EA0313DBB211
:10470800120ADF0042EA03228C4287EA131382EA84
:104718000302EFD1002A7FF452AC794A7D4F794BDE
:1047280012887D4CFA61DFF808921A68FA629B6871
:10473800B4F85221F8660021FB64D9F80000F96347
:10474800FA6506F023FE029000287EF4CAA9022129
:10475800D9F8000008F086FA94F854319AF8032042
:104768000392642B4FF0040287F8742040F05781BD
:1047780094F85531072B04BF9DF8083084F855315B
:1047880094F85531069307EB031ADAF804100291EE
:10479800084626F095FDDAF8081005915FFA80FAC8
:1047A800084626F08DFDC0B204900AEB0002069B75
:1047B8005A48029902900832C27123F00F028646C5
:1047C8008272049803F00F0300EBCA008EF80D30D4
:1047D80052468EF80E000EF10F0027F0A3FC504B46
:1047E800049A05990AF10900184427F09BFC0298DD
:1047F800C37903F1010ACBB1013B5FFA83FC0CF1E9
:10480800080CDFF830E184440023073010F8011B5E
:1048180059408B00CA0883EA410302F018024B4052
:104828004EFA02F253408445DBB2EFD13C4A03987A
:104838000AF8023021F02CFD94F85531002201339A
:1048480084F8553184F85421029BDDF808A09B7840
:104858005BB11AF80510D9F8000008F017FA01350D
:104868009AF80230EDB2AB42F3D894F854310322EF
:10487800013384F8543187F8742088F80020FFF752
:1048880062B80221D8F8000008F0ECF994F82C314D
:10489800FEF7E4B81023042218460AA98DF82A90D6
:1048A8008DF82B908DF82C908DF82D908DF8283060
:1048B8008DF8292014F0D0FE84F83791FEF7F9B866
:1048C800184A1268D2067FF5D9AA8046FFF7D9BAE6
:1048D8001549881F14F0A4FD84F84601FFF7AFB806
:1048E800074B1988FFF765BA104AD278002A0CBF1F
:1048F8004FF0040C4FF0050CFEF76CBECC380020CE
:104908001432002044370020676666662C66002053
:1049180058A08B41000000209816002078590020EC
:104928007E590020444D0020D81700205C660020E6
:10493800FC4400200007090E0123D8F800003B7052
:1049480008F098F90746D8F8000008F093F97F06B0
:104958007EF455A88E287EF452A894F82031002BB6
:104968007EF46AA8944BC4F828312D2384F82C319E
:10497800FEF74CB80326914940E5914B914A1B68D4
:10498800914903F4800383420ABF11460326042693
:1049980025E58E499A790B8803EB830303EB8303A0
:1049A8004FEA83081FFA88F8002A00F0DE80884B57
:1049B8001B680FFA83FA0CF037F940B2FEF732BAE7
:1049C8004FF03408FFF7DFBB984699461846049322
:1049D80005930393FEF71EBB7E4904260EE54FF0B0
:1049E8002408FFF7D0BB4B1CDBB2042B84F84931F9
:1049F8004FEA01617FF475A9FFF770B94FF010080D
:104A0800FFF7C1BB0CF010F914F0E8FE002014F019
:104A1800E5FEFFF742BA4FF02008FFF7B4BB97F85E
:104A280075A06D4904951AF00F0F04BF0AF1010A29
:104A38005FFA8AFABAF1070F28BF4FF0010A4FEA66
:104A48000A1C07EB0C03187C644B02930A1800231A
:104A580092F82410614A93725FFA8CF31A46604BFD
:104A6800964607EB0C024EEA000001291870D2683E
:104A780003F101000CD90239C9B28D1C1D4403464B
:104A880003F8012BAB424FEA1222F9D10131084455
:104A9800BC4422F060030AF1010A9CF811205FFA75
:104AA8008AFA1343BAF1080F037000F1010366D0C4
:104AB8004FEA0A1C07EB0C01494A087C46490144A5
:104AC8009A1A91F8241055180EF1100E132D5FFA4A
:104AD8008EFEC6DD049D0298DFF80CE1D1B28B1D75
:104AE800DBB243F04002C27103F1010CCBB14B1DA4
:104AF800DBB20833C31804930EF10100002310F849
:104B0800011B59408B0083EA4103CA084B403549D1
:104B180002F0180241FA02F25340049A8242DBB2D0
:104B2800EDD103980CF80E3087F875A021F0B0FB92
:104B38008AE63B685E2098473B68392098475FFAC9
:104B480089F014F04BFE4FEA192014F047FEE8E410
:104B58004FF00808FFF717BB984699461846049384
:104B680005939E460393FEF755BA4FF0FF3320E7AF
:104B7800174B9046B3F900A06420FEF753B9184AC2
:104B8800049D9A1AA7E798469946184604930393F2
:104B9800FEF740BA0393FEF73DBA98460393FEF733
:104BA80039BA984699460393FEF734BA9846994617
:104BB80018460393FEF72EBA4C39002088130308D1
:104BC800444D0020801303087C130308143200208E
:104BD800443700208C130308ACE8020878590020F9
:104BE800855900200007090E7E5900202DE9F04F55
:104BF80095B0B0F908500D81EDB2442D00AF0C46C8
:104C0800904600F01784064632D9812D00F05D8366
:104C180000F28680542D00F0B38040F2BD806E2DE6
:104C280000F0D683802D40F0B9806A4B1D780B3D8B
:104C380015F0FF0514D0DFF8C4E100220A26216828
:104C4800BEF80030481C20600E702168FF2B02F16E
:104C58000102A8BFFF23481CAA4220600B70EEDBAC
:104C680001252B46284654376381BD46BDE8F08FA1
:104C7800052D00F0CD831FD8022D79D040F2048392
:104C8800032D00F09B83042D40F088805249204674
:104C98002A46FCF704FF00212046FCF72EFF226875
:104CA8000021531C0125236028462B4654371170D8
:104CB8006381BD46BDE8F08F242D57D040F29A821B
:104CC800282D00F03D83382D68D10A68434B012513
:104CD800511C21601570226805215019206011703F
:104CE80022680A2150192060117022680021501989
:104CF800206011702268197850192060117022689C
:104D080059785019206011702268997853192360D6
:104D18002B461170284654376381BD46BDE8F08F95
:104D2800A02D11D040F28582B82D00F04583FE2DCC
:104D380034D12B4D05F1080635F8021B2046FCF747
:104D4800DCFEB542F8D18BE7264B08461968FCF71C
:104D5800BDFE254B20461968FCF7B8FE234B1968A1
:104D680020460125FCF7B2FE2B467BE7204BF6E7F1
:104D78000422204920460125FCF791FE2B46C9E76D
:104D88000B6800215A1C22601970226801255319EA
:104D980023602B461170BDE7522D80D0214628464E
:104DA8000AF0A2FA034600287FF45AAF742D00F0E7
:104DB8007E82772D24D13268716891421EBF531CC0
:104DC800336011780C4A08BF1946204620F02CF8A9
:104DD80046E700BFB2310020B1650020EF40002057
:104DE80008320020ACF7FF1FB0F7FF1FB4F7FF1F12
:104DF800284200201814030809410208C41C002096
:104E0800F52D01F06882472D00F04083292D336885
:104E180001F00982392D01F0F381212D01F0D081B3
:104E280071680B3DCA1AEF2D00F25B8401A050F89F
:104E380025F000BF1D5C0008EB560008EB56000883
:104E4800EB560008EB560008EB560008EB56000836
:104E5800EB560008EB560008EB560008EB56000826
:104E6800EB560008EB560008EB560008EB56000816
:104E7800EB560008EB560008EB560008EB56000806
:104E8800EB560008EB560008EB560008EB560008F6
:104E9800EB560008C95B0008EB560008675B000882
:104EA800EB5600083D5B0008EB560008EB5600087F
:104EB800EB560008235D0008EB560008AD5C0008BF
:104EC800EB5600087B5C0008EB560008555C0008B0
:104ED800EB5600082B5B0008EB560008D35A000875
:104EE800EB560008815A0008EB560008EB560008FC
:104EF800EB560008EB560008694C0008EB56000812
:104F0800655A0008EB560008EB5600089561000842
:104F1800EB5600083B610008EB560008EB5600080A
:104F2800EB560008EB5600082F610008EB56000806
:104F3800EB560008EB560008EF600008EB56000837
:104F4800115F0008EB560008EB560008A15E000848
:104F5800EB560008EB560008EB560008EB56000825
:104F6800EB560008EB560008EB560008CD5D00082C
:104F7800EB5600084B5D0008EB5600080D60000872
:104F8800EB5600085F5F0008EB560008C760000892
:104F9800475A0008EB560008EB560008EB56000885
:104FA800EB560008EB560008EB560008EB560008D5
:104FB800EB560008EB560008EB560008EB560008C5
:104FC800EB560008EB560008EB560008EB560008B5
:104FD800EB560008EB560008EB560008EB560008A5
:104FE800EB560008EB560008EB560008EB56000895
:104FF800EB560008EB560008EB560008EB56000885
:10500800EB560008EB560008EB560008EB56000874
:10501800EB560008EB560008EB560008EB56000864
:10502800EB560008EB560008EB560008EB56000854
:10503800EB560008EB560008EB560008EB56000844
:10504800EB560008EB560008EB560008EB56000834
:10505800EB560008EB560008EB560008EB56000824
:10506800EB560008EB560008EB560008EB56000814
:10507800EB560008EB560008EB560008EB56000804
:10508800EB560008EB560008EB560008EB560008F4
:10509800EB560008EB560008EB560008EB560008E4
:1050A800EB560008EB560008EB560008EB560008D4
:1050B800EB560008EB560008EB560008EB560008C4
:1050C800EB560008EB560008EB560008EB560008B4
:1050D800EB560008EB560008EB560008EB560008A4
:1050E800EB5600081D5A0008EB560008015A000844
:1050F800EB560008EB560008EB560008EB56000884
:10510800EB560008EB560008EB560008EB56000873
:10511800EB560008EB560008EB560008EB56000863
:10512800EB560008EB560008A3590008EB56000898
:105138006B590008EB560008AD5800089358000852
:105148004F590008EB56000879580008EB5600083C
:1051580051580008EB560008F1570008EB560008B4
:1051680089570008EB560008EB5600085F570008FF
:1051780009570008F556000837570008CD560008AB
:10518800A3560008EB560008EB560008EB5600083B
:10519800EB560008EB560008EB560008EB560008E3
:1051A800EB560008EB560008EB560008EB560008D3
:1051B800EB560008EB560008EB560008EB560008C3
:1051C800EB56000883560008EB560008EB5600081B
:1051D8002B560008EB560008EB560008EB56000863
:1051E800EB560008EB560008EB560008EB56000893
:1051F80013560008202D7FF4D1AD0B68914D591C32
:105208006A7821601A7023682A78591C21601A70FC
:105218002368AA78591C21601A7029892046FCF74E
:105228006CFC23686A79591C21601A702268A97974
:1052380037E5822D7FF4B2AD0B68834A834D117830
:10524800804A581C2060197011892046FCF755FCCB
:105258007F4B22681B88FF2B02F10101A8BFFF23A7
:1052680021601370A96881F3100189B22046FCF708
:1052780044FC296801F30F0189B22046FCF73DFC84
:10528800744B226819780CE5012D7FF487AD0B6803
:105298000022591C21601A7023685A1C22601D7054
:1052A80022682421531C23602B46117032E5326892
:1052B800716891421EBF531C33601178664A08BF5B
:1052C800194620461FF0B0FDCAE4644B1E780A3E1A
:1052D80016F0FF063FF4C4AC614BDFF8A8811E440A
:1052E80003F101090A2314E0502B00F05C87002524
:1052F80029462268501C206020461370FCF7FDFBED
:1053080029462046FCF7F9FBB1453FF4A9AC19F84A
:10531800013B0A2BE8D1534A9568116805EB8505CE
:105328004FF6FF726D009542A8BF15469142A8BF7F
:10533800114625EAE57521EAE171ADB289B2D8E7EF
:105348000B68DFF84491484E591C022221601A70FC
:1053580023684FF006085A1C226083F800802368EF
:105368000A22591C21601A70236801255A192260E3
:105378001D70B9F800102046FCF7BFFBB9F8021001
:105388002046FCF7BAFB23685A19226083F800808C
:1053980023685022591921601A702368002259196C
:1053A80021601A7031882046FCF7A7FB71882046D7
:1053B800FCF7A3FB2B46ADE42C4BD0E40B685A1C3E
:1053C8000A601D700B680222591C21601A7066E47D
:1053D8001F4B0A681B881D4DFF2BA8BFFF23511CBC
:1053E80021601370A96881F3100189B22046FCF787
:1053F80084FB1F4B20461988FCF77FFB296801F3C3
:105408000F0189B220460125FCF777FB2B4681E482
:105418000B2218492046FCF742FB08221649204671
:10542800FCF73DFB0125072214492046FCF737FB12
:105438002B466FE4002A3FF413AC114B136001258F
:105448002B4667E44C6600202A32002044370020AF
:10545800143200208A380020E94C0208B2310020BA
:1054680004E90208801C0020B41C0020D429002074
:1054780084380020201403082C1403083814030867
:10548800C5F20008B81C0020003600207268356894
:105498007B623046551BFCF7DBFA052D38627B6AC8
:1054A80000F298878026B346012594E80600521A30
:1054B800103A9642C8BF1FFA82FBBD4A396A926801
:1054C8003A61521A9345396A7B622046FA6088BF6E
:1054D8001FFA82FBFCF7FAFA7B6A002B00F0588768
:1054E800002D40F0D7862368C7F800D05D71C0B0A2
:1054F8000533C7F808D0FB61BBF1000F01F0268027
:105508003B6A3A69934280F0F287AA463E6A7D6216
:105518007C6080255446FB681C1BA54BB4F5807F36
:1055280028BF4FF480749B6832199A4288BF9C1B2D
:10553800FCF70AFE2246BC6830462146FCF784FE8A
:10554800F969B86104EB000C0B787B61644530D2D3
:10555800DFF884920CF1FF3C04F1FF3E1EF8013F96
:1055680009EB830219F823405688FCB100234FF455
:10557800004204F1FF3816424FEA520202D008787E
:10558800284308706D0806D10AF1010A4D701FFA08
:105598008AFA01318025D34505D8E645C0F0098649
:1055A800984500F3068601339C42E4D1F445D5D1F1
:1055B800F9617B6ABA6913449BB2D3457B6206D909
:1055C8007B6A3A6A1C46D6183B699E42A3D37C681C
:1055D800802D1CBF0AF101031FFA83FA0AF10201A8
:1055E80089B22046FCF789FA2368796A01255A1995
:1055F800226020461D70FCF780FA2368534423601C
:105608002B46D7F800D0FFF785BB6A4B1B78DB0722
:1056180067D401250AF066FE0AF00EFF2B46FFF755
:1056280079BB5A1C32601A780F2A5AD8991C3160F3
:10563800C2EBC202604958788854D81C30600A44CA
:1056480099785170191D3160D9789170591D316060
:105658001979D170991D316059791171D91D31604D
:105668009979517103F108013160DB799371012552
:105678000DF0D4FB2B46FFF74DBB3046FCF7FFF986
:10568800DFF84C81A8F80E003046FCF7F8F9012540
:10569800A8F80C002B46FFF73DBB3046FCF7EFF9A6
:1056A800DFF83881A8F810003046FCF7E8F9A8F8C8
:1056B80012003046FCF7E3F90125A8F814002B4640
:1056C800FFF728BB1A46591C316012F8020B3260EA
:1056D800DA1C597832609A7816F0BEFB00287FF4FD
:1056E800BFAA4FF0FF352B46FFF714BB334B3449A5
:1056F80018684E22012526F015FD2B46FFF70ABB38
:1057080019465A1C32602F4A11F8020B107031608A
:1057180059785170D91C31609B7893703046FCF7EA
:10572800AEF9294B0125D8802B46FFF7F3BA1A4664
:10573800591C3160254912F8020B0870326024495F
:105748005A788A70DA1C3260224A9B789370012555
:105758002B46FFF7DFBA3046FCF791F9DFF868808F
:10576800A8F800003046FCF78AF9A8F8020030468D
:10577800FCF785F90125A8F804002B46FFF7CABAFB
:10578800DFF85C9099F80030002B3FF469AADFF845
:10579800548000253046FCF772F910F003F999F8A7
:1057A8000030A8EC010A01359D42F3DBFFF758BA37
:1057B80078140020A431002048270020B865002074
:1057C800F8F2020808360020282C00209C4A002005
:1057D800103600202036002008E90208C8610020A1
:1057E800B2310020802B00200D2A7FF47AAF5A1C9A
:1057F80032601D78072D3FF674AFDFF8B09330465E
:105808004FF00C08FCF73BF908FB05F809EB080515
:10581800A8803046FCF733F9E8803046FCF72FF9CA
:10582800336828811A46591C316012F8021BA97284
:1058380032605B78EB723046FCF70AF9012549F8CB
:1058480008002B46FFF766BA5A1C3260187806061D
:1058580000F15186CA4B1B78DD073FF501AA0328E2
:1058680028BF002001250AF015FD2B46FFF752BA84
:10587800C34B1B78D8073FF5F3A901250AF026FD8D
:105888000AF0DAFD2B46FFF745BABD4B1B78D9075E
:105898003FF5E6A9BB4B4FF4C87201251A802B4689
:1058A800FFF738BA092A7FF71CAFDFF804831A46D6
:1058B800591CD8F80050316012F8021B2970326068
:1058C8005A78AA70DA1C32609A78642A03F10401C3
:1058D800A8BF64226A713160DA78642A03F105018D
:1058E800A8BF6422AA7131601A79EA719A1D3260E0
:1058F8005A79642A03F10701A8BF64222A72316029
:105908009A79EA7003F108023260DB792B7130462C
:10591800FCF7B5F8726833686881D11A00290CDD84
:10592800591CD8F800003160521A002A19784172BF
:1059380003DD9A1C32605B784370012524F066F819
:105948002B46FFF7E7B98E4B1B78DA073FF588A996
:105958008D4A1378012543F0040313702B46FFF793
:10596800D9B98A4A1068DA1C01462133951E356078
:1059780012F8035C0D70551E356012F8025C4D700C
:10598800326012F8015C8D7003329A4201F1030112
:10599800ECD10FF0D3FEFFF763B9C2F34705122D20
:1059A8003FF69FAEC5B107F1500307F12A0903EB93
:1059B800450AC846AAF1260A3046FCF760F828F8D6
:1059C800020FC245F8D1724B39F8022F23F8022F83
:1059D800C845F9D1112D09D86E4A6B00023B134412
:1059E8000021223223F8021F9A42FBD16A4A01237E
:1059F8001D461370FFF78EB9DFF8B88100233046D3
:105A0800C8F80030FCF724F80125C8F800002B4638
:105A1800FFF780B91A46591C316012F8025B3260F0
:105A2800DA1C587832609978002D00F0EE85012D47
:105A38007FF416A922F0E4FD2B46FFF76BB9504A14
:105A4800127812F001017FF44CAE5A1C32601878BB
:105A5800012522F025FD2B46FFF75CB9591C1A4693
:105A680031604E4912F8020B887032605B784B70D7
:105A780001252B46FFF74EB90721B2FBF1F1C1EB27
:105A8800C105521B7FF42DAEC9B201F1FF395FFA8F
:105A980089F900293FF4E4A8DFF804A109F1010914
:105AA80015465A1C326093F900103D4B4FF0000820
:105AB80093F902208A4203F1080300F0AD8408F14B
:105AC8000108B8F1060FF3D10BE65A1C32601A78B8
:105AD8000E2A3FF606AE991C31605D78032D3FF61D
:105AE80000AE3048062101FB02F1421803F1030E13
:105AF8005571C6F800E09D784554191D3160D97874
:105B08005170591D316019799170991D3160597919
:105B1800D170D91D31609B79137101252B46FFF790
:105B2800F9B85A1C3260204A1B78537501252B4658
:105B3800FFF7F0B83046FBF7A2FFDFF87C80C8F823
:105B480000003046FBF79BFFC8F804003046FBF71F
:105B580096FF0125C8F808002B46FFF7DBB8DFF8E9
:105B68005C800023C8F800303046FBF771FFD8F896
:105B7800003001250343C8F800302B46FFF7CAB8A8
:105B8800A43100200667002028340020B8650020D2
:105B98008243002084430020A84300202C360020A4
:105BA800CC5E0020E0290020D84E0020542600209A
:105BB800E8660020D4290020B424002028420020D0
:105BC8005A1C32601D78132D3FF68BAD9A1C32603B
:105BD80058787B621FF062F900283FF482AD7B6A37
:105BE800BD4A017802F82510D91C316002EB850204
:105BF80099785170191D3160D8789070581D3060AF
:105C0800B6491B79D3700868012523F08DFE2B4611
:105C1800FFF780B8B249102A13464FF0000228BF98
:105C280010230A604A608A60CA600A74002B3FF435
:105C380017A83268013913440132326012F8010C96
:105C480001F8010F9A42F7D1FFF70AB8591C3160E1
:105C58001D781F2D3FF645AD052A7FF442AD30462D
:105C6800FBF7F6FE9F4B43F8250023F069F9FEF792
:105C7800F7BF9C4D05F140083046FBF700FF33683D
:105C8800A5F88000591C1A46316012F8021B85F8E5
:105C9800821032605B7885F883300435A845EBD1F3
:105CA800FEF7DEBF5A1C32608F4D1B782B723046D0
:105CB800FBF7E5FEA8833046FBF7E1FE2883304674
:105CC800FBF7DDFE32686883531C33601278EA7490
:105CD8007268D31A032B00F319843368D11A052983
:105CE8000EDD5A1C32601B78EB723046FBF7B0FEB3
:105CF8003368E8605A1C32601B782B74336872680A
:105D0800D21A002A7EF7ACAF5A1C32601B7885F88D
:105D1800213001252B46FEF7FDBF581C3060734A21
:105D28001D781570091A00297EF79AAF991C316001
:105D38005B78003318BF0123012553702B46FEF70B
:105D4800E9BF1A46591C3160DFF8B48112F8021B0A
:105D580088F80210326066495A780A70DA1C326094
:105D6800644D9A782A711A1D3260DB78092BA8BF16
:105D780009233046AB70FBF782FE336872682880CF
:105D8800D11A012905DD3046FBF779FE33687268C0
:105D9800E8819A4207D05A1C32601B78003318BF3A
:105DA800012388F807300AF0A7FA336872689A4224
:105DB8003EF456AF5A1C32601B78EB7001252B4617
:105DC800FEF7A8BF3046FBF75AFE054612F0C4F8A6
:105DD800FF283EF445AF3F2D00F2C88307F1500875
:105DE800002308F8243D4FEAD509414607F12B0066
:105DF80087F82B3009F1010912F08EF897F82B304B
:105E08005FFA89F905F007054B4505F1010503D14E
:105E180097F82C30AB4203D02946484612F088F850
:105E280033687268D21A012A7EF71AAF5A1C07F132
:105E38005000326000221D7800F8252D12F060F81D
:105E480097F82B30AB420AD02B4B1B683BB19A79A1
:105E5800AA4204D31B681B690BB1284698473368CC
:105E68005A1C3260404600221D7887F82C2012F018
:105E78003BF897F82C30AB423EF4F2AE1E4B1B6851
:105E8800002B3EF4EDAE1B685B69002B3EF4E8AED8
:105E980028469847FEF7E4BE184A1278012A3EF6CB
:105EA800DFAE18465A1C3260DFF8588010F8022B13
:105EB80088F80220DA1C891A306001295878326083
:105EC80040F388833046FBF7DAFD0125A8F8000087
:105ED8002B46FEF71FBF00BF54360020B8650020D0
:105EE800EC35002058370020D84E002050360020CE
:105EF80004360020C8610020142E00201D42002016
:105F08009C4A0020204200205A1C326093F80080EE
:105F1800B8F1110F3FF6E5AB9A1C3260CE4D5B78B5
:105F280005F818303046FBF7AAFD40F6CA03984238
:105F3800A8BF184640F2EE23984205EB4801B8BFC7
:105F480018460125A0F2EE222B46192092FBF0F20A
:105F58004A70FEF7DFBE3046FBF791FD3046FBF78F
:105F68008EFD3046FBF78BFD3046FBF793FD33681B
:105F7800BA4D1946581C2A68306011F8020B82F88D
:105F88002C003160597882F83610D91C31609B7822
:105F980082F837303046FBF77DFD3046FBF77AFD57
:105FA8003046FBF777FD3046D5F80080FBF767FDF4
:105FB800A8F83A003046D5F80080FBF760FD336852
:105FC8007268A8F83800D11A01290ADD591C2A6814
:105FD80031601B7882F82E303046FBF75BFD336862
:105FE8007268D31A032B0BDD3046D5F80080FBF717
:105FF80046FDA8F8320030462E68FBF740FDB08613
:106008002868C6E45A1C3260944DDFF87C821B78FD
:1060180088F805303046D5F80090FBF730FDA9F830
:1060280020003046D5F80090FBF729FD72683368E8
:10603800A9F81E00D11A072919DD3046FBF71FFD04
:10604800A8F80A003046FBF71AFDA8F80C003046FD
:10605800D5F80090FBF713FDA9F822003046D5F8D3
:106068000090FBF70CFD33687268A9F82400D11A78
:1060780003290BDD3046FBF702FDA8F80E00304679
:10608800FBF7FDFC33687268A8F81000D21A002AE2
:1060980005DD591C2A6831601B7882F826300AF021
:1060A8002BF91CF0A7FD6E4B1B68002B00F05382E8
:1060B800286801250CF046FF2B46FEF72BBE1A4632
:1060C800591C3160674912F8020BC8703260664982
:1060D8005A784A71DA1C3260644A9B78D370012579
:1060E8002B46FEF717BE1A46591C614D316012F84F
:1060F800021B297132605B786B713046FBF7BFFC7D
:10610800336828805A1C32601B78AB713046FBF725
:10611800B6FC336868805A1C32601B78EB71012525
:106128002B46FEF7F7BD0125FCF770F82B46FEF766
:10613800F1BD5A1C32604F4A1B78DFF8508113704A
:106148000023C8F800303046FBF782FC3368D8F8E3
:1061580000204949494D10435A1CC8F800003260D4
:106168001B780B723046FBF78AFC28603046FBF739
:1061780086FC68603046FBF782FCA8603046FBF777
:106188007EFC3046FBF77BFCFEF76ABD3C4A03F118
:1061980008010133336013F8010C02F8010F99422A
:1061A800F7D1FEF75DBDD8F80850D8F80010FFF712
:1061B800B5B8FB697C681A463B7D1370FFF708BACF
:1061C8001A46591C31602F4D12F8021B6970326053
:1061D8005A782A70DA1C32609B78AB703046FBF72D
:1061E8004EFC33682881591C1A46316012F8021B8C
:1061F800697132605B78AB7101252B46FEF78ABD69
:106208005A1C32601A780A2A00F0F7803046FBF7E9
:1062180041FC3046FBF73EFC01253046FBF73AFCD3
:106228002B46FEF777BD5A1C32601B780A2B00F00C
:10623800DE80502BA2D13046FBF721FCDFF85080DE
:10624800A8F800003046FBF71AFC0125A8F8020060
:106258002B46FEF75FBD00BF4C450020B865002007
:106268003436002010360020943A002020360020D2
:10627800402C002050360020D84E0020B4240020A6
:10628800D74E00204C6600209C4A0020284200205F
:10629800B41C0020C04B3A6A9B68D4F800905A445A
:1062A8009A4200F21181FBF74FFF5A464946386A75
:1062B800FBF7CAFF236803442360B042BEF6D0ACA4
:1062C800002100E0236801305A1C864222601970C0
:1062D800F8D1FEF7C5BC336872689A4240F0CB80AB
:1062E800AE4BFF221A704FF0000AAD4D21F00AFFA5
:1062F80051462022AB4885F800A028F092F987F88B
:106308002CA097F82C30072B00F2EF80DFF8BC9216
:10631800A44E524697F82C3003EB430309EBC30312
:106328005B7CE3B197F82C3003EB430309EBC30321
:1063380020215B699BB197F82C3003EB430309EBF1
:10634800C303586946F82200FAF777FC2B7856F809
:106358002300FAF79CFE2A780132D2B22A7097F805
:106368002C300133DBB287F82C3097F82C30072B10
:10637800D0D92368591C21601A70B8F1000F3EF477
:106388006FAC894BC8F8003001252B46FEF7C2BC1C
:10639800002D7FF47FAF59462046FBF7AEFB2368FC
:1063A8005A1C22601D707C4B26689D683B6A0BEB6B
:1063B8000302954280F01B813B6AED1AFBF7C4FE8D
:1063C8002A463146386AFBF73FFF236803442360B7
:1063D800FEF746BC3046FBF752FB326871687B6AB1
:1063E800914283463DD106461D46FFF75EB83046CA
:1063F800FBF745FBDFF8D88122E79A1C32606B4A2D
:1064080059781170D91C316099785170191D316013
:10641800DB789370FEF724BC0AEBC80B30468BF888
:106428000210FBF72CFB32682AF838001346511C7F
:10643800316013F8021B8BF80310336053788BF824
:106448000430D31C336093788BF80630131D336007
:106458000135D2788BF80520A9457FF422ABFEF7E9
:10646800FFBB511C316012781D46131C064618BF2D
:106478000123FFF71AB85A1C19463260474811F829
:10648800022B027031605B784370042A03D9FF2A1B
:106498007EF405AC27E746490978994205D8022ACF
:1064A8007EF4FDABFF2B7EF4FAAB236801255A1965
:1064B80022601D70B8F1000F3EF4D2AB3D4BC8F816
:1064C80000302B46FEF726BC3A6AA3EB0208FBF71E
:1064D8003BFE42464946386AFBF7B6FE236803444A
:1064E8002360002D3EF4BCABE7E6524641E77D62EF
:1064F800AA46FFF773B800F07F00032828BF0020E2
:10650800012522F099F82B46FEF704BC3046FBF72C
:10651800B6FAA8843046FBF7B2FA33687268E884A2
:10652800D11A03297FF7DAAB1A46591C316012F8E1
:10653800021BA97732605B7885F820303046FBF77C
:106548009EFA336872686884FFF7C8BBDA46C7F8F2
:1065580024B0FFF743B818481849194A194B036083
:1065680001250B6013602B46FEF7D4BB07F12C08FE
:10657800404611F0ADFCBB8DAB423FF451AC124B21
:106588001B68002B3FF44CAC1B689B69002B3FF445
:1065980047AC2846984743E4781400206419002043
:1065A8002F2500208044002059200108EF400020BA
:1065B800B2310020DDF20008C02700201428002096
:1065C8007C280020F7040008142E00200861002011
:1065D80000360020104A99781288012512FB00F233
:1065E8002B4692FBF1F2A8F80020FEF793BBFBF7CD
:1065F800ABFD5A463146386AFBF726FE236801256B
:10660800034423602B46FEF785BB01250EF002FFED
:106618002B46FEF77FBB00BF806800202DE9F04FB6
:106628002DED0C8B3C4B1B7895B0012B099001F09C
:106638006D863A4C94F80021002A41F0C180072B5E
:10664800374D01F05E86002305936B683448984700
:10665800002800F06981B5F8B470002285F855204B
:10666800002F40F04387B5F93E00AA6AB5F93C60AF
:10667800696AB5F94030DFF8B4B0821AE86A6A632B
:10668800711A1B1A2963274895F85610AB6317F03F
:106698003FFFDBF80030990040F1F080D5ED0D5A4E
:1066A800D5ED0C7A204A94ED656AD4ED666A94EDCE
:1066B800677AD4F8A0311268B8EEE58AD5ED0E5A9B
:1066C800F8EEE77AF8EEE58A013377EE867A38EE67
:1066D800268A78EE878A9342C4ED657A84ED668AC5
:1066E800C4ED678AC4F8A03101F0D0830A4B1F7843
:1066F800142F02F011870023D4F8A8610693062E00
:1067080000F2AF80DFE816F0D81535156A149D162B
:1067180014004915CE1400BF043200206819002067
:10672800B04A0020E04A0020383D0020444D0020B7
:10673800D84B1A78D4F8ACE1DFF8D0C39FEDD67AFD
:106748004FEACE000CEB000383ED007A002A7DD0DF
:10675800D249B0EE476AF0EE476A0023F1EC017ABD
:10676800013367EEA77A05EE903AB4EEE77AF1EED8
:1067780010FAF8EEE55AB8BFB0EE677A934276EEB3
:10678800A76AA7EEA56AE9D1F5EEC06A0CEB00038B
:10679800F1EE10FA83ED007A58DDC6EE265AC04BAA
:1067A800C04A1288F7EE007A75EEE75AD3ED007A00
:1067B80065EEA77AFDEEE77A17EE903A812B43F360
:1067C8001C859342A8BF134607EE903AF8EEE77A85
:1067D800B54B00EB0E0103EB810393ED057AD3ED86
:1067E800003A93ED066A93ED014AD3ED046AD3EDBE
:1067F800034A93ED025AA3EEA77AA4EE276A66EE3F
:10680800C76AA7EE646ABDEEC77AE5EE276A17EE97
:10681800101A812983ED056AC3ED066A43F3EA84F9
:106828008A42A8BF0A4607EE902AF8EEE77AFCEEFD
:10683800E77ACDED077ABDF81C300CEB00029380A7
:10684800BEF1000F02D1132F04F05181152F42F031
:106858001A846044DFF8B882838828F81E30D4F898
:10686800A861924B013683FB06239A19F317C3EBF1
:10687800A203C3EBC303F61AC4F8A8618C4B1B78B8
:10688800002B01F0A3808B4EDFF88892DFF880A2FE
:1068980006F5BC780027884BD5ED087A1B78172BAE
:1068A80001F0888396ED007AB8EEC78A082B28EEA7
:1068B800278A07D1B0EE480A069325F0A7FD069B64
:1068C8002AF81700DBF8002092000BD5002F04F0FF
:1068D8003084B0EE480AD5F8143208F170009847B1
:1068E800B0EE408AB0EE480AD5F83431A8F170000D
:1068F8009847D5F8A431404698476F4B1B78032B2F
:10690800B0EE408A01F06383D6F8F800D5F8B830C5
:10691800B0EE480A98470137032F08F12408A9EC7C
:10692800010A06F10406B6D1634B93F80090B9F159
:10693800070F00F0988694F8B831002B40F0A08635
:106948005E4B5B79002B40F0CB8501235A4A84F8D3
:10695800B8311278072A02F0238000230B93584B92
:1069680094ED709A93ED007A564BD4ED6FCAD3F834
:1069780000A0554B0693F7EE007A37EEC9CA534B81
:1069880008932CEE07CA524B0A93B4EEE7CA514B50
:1069980007930025F1EE10FA4F4BDFF87C91DFF8F2
:1069A8007CB1DFED4E8A9FED4EAADFED3BBADFEDFD
:1069B8004D9A9FED4DBADFED4DAADFF864814C4F3B
:1069C800059388BFB0EE67CA2E464A4B99ED008AF8
:1069D8002B44D3ED007AF5EE407AF1EE10FA17D099
:1069E800454B2B44D3ED006A38EE667AB0EEC76AA1
:1069F800F4EEC67AF1EE10FA08D5B5EEC07AF1EEEB
:106A080010FACCBF37EEA68A36EEE78A83ED008A05
:106A1800069B1A88930700F08580022E00F082807A
:106A28009AF82E10354B07EE901A2B4493ED007A06
:106A38004B42F8EEE76A07EE903A26EE877AF8EED0
:106A4800E77AB4EEE77AF1EE10FA0AD407EE901A74
:106A5800F8EE677AF4EEC77AF1EE10FA88BFF0EE36
:106A6800477A274B274903EB460331F91600B3F958
:106A78000C30C01A07EE100AB8EEC77AD007E7EE56
:106A8800687A40F10586204B93ED008A27EE888AC4
:106A980048E000BF3E3D00200000000068190020CB
:106AA800403D00203C3D0020743F00209324499243
:106AB800353D0020E04A0020043200209C4A002096
:106AC8004C2B0020B8650020863800207800002074
:106AD800A4310020344D00202C340020CDCCCC3DF6
:106AE800AE47813F0000C84200003443610BB63B0B
:106AF80038340020402B00202C1B0020D41A002002
:106B0800103600202C660020282B00205C3F002037
:106B180008320020384D00206C1A0020BC270020C5
:106B280044340020079B94F8D0212B44D3ED01DA9C
:106B380038EE6DDA002A3DD0D24BD4F8D421099929
:106B48001B688A1A9A4235DD9AF84830022B01F000
:106B58009B87022E04F09082CB4B1B68990740F16B
:106B68001C87CA4BCA49DFF890E331F916C09EED7D
:106B7800008ADFF888E3C7ED00BA03EB460028EE89
:106B8800288AB0F90C00A0EB0C0007EE900AF8EE8A
:106B9800E77ADEF8000027EE888A904238EE6DDA50
:106BA800C1F22681F7EE007AB4EEE79AF1EE10FA18
:106BB80001F1F580B74B2B4493ED000A059B2CEEB1
:106BC800800A022E20EE0D0AA3EC010A059304F0B8
:106BD8001182089BDBED007A93ED007AAE4BD7ED7E
:106BE800006A93ED006AAD4B67EE277A2B4427EED7
:106BF8008C7AD3ED007A67EE277AF0EE665AEDEEDE
:106C0800275AB1EE467AB4EEE57AF1EE10FA08DCCE
:106C1800B4EEE56AF1EE10FA8CBFB0EE657AB0EE2C
:106C2800467A94ED706AF7EE007AB4EEE76AF1EE10
:106C380010FAACBF0123002343B1F0EEE66AF0EE90
:106C4800C77AF4EEE67AF1EE10FA01D587ED007A0C
:106C5800022E04F09081924A924B52F826001B684B
:106C6800B0EE6D0A9847904A904B52F826001B6880
:106C780098479AF8373023B1069B1B88002B00F001
:106C88006B85B0EE6B8A8A4B9BED007A38EE400A32
:106C98002B4493ED008A83ED000A9AF8483030EED1
:106CA800480AC0EE077A2BB30A9B1B78DB0721D56D
:106CB800B7EE007AB4EEC79AF1EE10FA04DB94F856
:106CC800D031002B00F05587D4F8D431099AD31A63
:106CD8006C4A12689A420DDD764B93ED007AB0EE5D
:106CE800CDDAB4EEC7DAF1EE10FA41F19D80002357
:106CF80084F8D031704B94F8E0212B4493ED007A5E
:106D08002CEE877A67EE277AC8ED007A32B9059BB0
:106D1800C7ED00BA43ED01BAC8ED00BA0136032E3B
:106D280009F1040908F1040807F1040705F104054D
:106D38007FF44BAE614B1B78072B01F03383012B9B
:106D480001F01B86002794F8E831002B40F0EF850E
:106D58005B4A5C4B10681B6810F4805A93F82C301F
:106D680040F05E86584A594992ED006A498B584A64
:106D780084ED7E6A92ED007A564A84ED7F7A07EEBA
:106D8800901AF8EEE76AD2ED037A534A84ED7C6AEA
:106D980037EE467A77EEE67AD2ED006A84ED7B7AB2
:106DA800012284F80022C7EEA65A4C494C4A91EDBC
:106DB800005A4C499FED4C6A91ED004A4B49DFED72
:106DC8004C6AD1ED004A92ED007A35EE045AF7EE9E
:106DD800007AF4EEE75A35EE245AF1EE10FA88BF3D
:106DE800F0EE675A25EE065AF4EEE65AB1EE476A17
:106DF800F1EE10FAB4EEC65AB8BFF0EE665AF1EEEC
:106E080010FAC4ED815A01F1CE80B4EEC75AF1EE02
:106E180010FA88BFB0EE475A304ADFED336AD2ED38
:106E2800017A304A92ED014A304A77EE847AD2EDFF
:106E3800014A77EEA47A67EEA67AB4EEE76AF1EE35
:106E480010FA08DCB4EEE77AF1EE10FA8CBFB0EE77
:106E5800676AB0EE476A214ADFED236AD2ED027A0B
:106E6800204AD2ED024A234A77EEA47A92ED007ABC
:106E780067EEA67AB1EE473AF4EEC37AF1EE10FA6D
:106E880047D43DE0542B0020E06500201036002058
:106E98002C660020FC2A0020702B0020082B0020E4
:106EA800C4270020C027002018280020142800200C
:106EB800401B0020602B0020142B002004320020EF
:106EC800444D0020B865002088340020D84E0020AA
:106ED800E03500202C320020302C00202C340020FB
:106EE800742B0020383400206F12833A4434002079
:106EF80000000000782B0020282B0020502B0020B9
:106F0800F4EEC77AF1EE10FA8CBFB0EE473AB0EE65
:106F1800673AF04A52780AB9B1EE433A002B41F089
:106F28006283F7EE003AEC4D2A78002A02F0548684
:106F3800EA4BDFEDEB7AD3ED024AD3ED016A93ED2C
:106F4800037A66EE244AE5EE264AE3EE074A63EE44
:106F5800A44AF4EEE74AF1EE10FAB4BFB0EE674A7D
:106F6800B0EE644A98BFF0EE647A012ACDED0C4A7F
:106F780002F0578693ED067AD3ED052AD3ED076A1A
:106F880026EE077AA5EE227AA3EE267A23EE877AF2
:106F9800B4EEE77AF1EE10FAB4EEC47A8CBFF0EEF4
:106FA800676AF0EE476AF1EE10FA88BFF0EE676A9A
:106FB800B4BFF0EE447AF0EE477A022A8DED0D7AEE
:106FC80000F0DE8093ED0A7AD3ED092A93ED0B4A9F
:106FD80026EE077AA5EE227AA3EE047A23EE877AC4
:106FE800B4EEE67AF1EE10FAB4EEE77A8CBFB0EEC2
:106FF800664AB0EE474AF1EE10FA98BFF0EE446ADE
:10700800A8BFF0EE477A032A8DED0E7A00F0B8801B
:1070180093ED0E7AD3ED0D2A93ED0F4A26EE077AFB
:10702800A5EE227AA3EE047A23EE877AB4EEE67A06
:10703800F1EE10FAB4EEE77A8CBFB0EE664AB0EE25
:10704800474AF1EE10FA98BFF0EE446AA8BFF0EE96
:10705800477A042A8DED0F7A00F0928093ED124A58
:10706800D3ED112A93ED137A26EE044AA5EE224AAF
:10707800A3EE074A23EE844AB4EEE64AF1EE10FA8C
:10708800B4EEE74A8CBFB0EE667AB0EE447AF1EE21
:1070980010FA98BFF0EE476AA8BFF0EE447A052AC6
:1070A8008DED104A6CD093ED164AD3ED152A93ED69
:1070B800177A26EE044AA5EE224AA3EE074A23EEE3
:1070C800844AB4EEE64AF1EE10FAB4EEE74A8CBF11
:1070D800B0EE667AB0EE447AF1EE10FA98BFF0EEB0
:1070E800476AA8BFF0EE447A062A8DED114A47D0C8
:1070F80093ED1A4AD3ED192A93ED1B7A26EE044A2A
:10710800A5EE224AA3EE074A23EE844AB4EEE64AE5
:10711800F1EE10FAB4EEE74A8CBFB0EE667AB0EE44
:10712800447AF1EE10FA98BFF0EE476AA8BFF0EE85
:10713800447A072A8DED124A22D093ED1E7AD3EDB8
:107148001D2A93ED1F4A26EE077AA5EE227AA4EEB1
:10715800037A27EE237AB4EEE67AF1EE10FAB4EE6B
:10716800E77A8CBFB0EE666AB0EE476AF1EE10FAC5
:107178008DED137A98BFF0EE466AA8BFF0EE477A15
:1071880077EEE67AF7EE006AF4EEE67AF1EE10FAB8
:10719800C4ED707A43F3908486EEA77A022ADDED77
:1071A8000D7A67EE244A67EE877ACDED0C4ACDED6D
:1071B8000D7A2DD0DDED0E7A67EE877A032ACDEDB4
:1071C8000E7A25D0DDED0F7A67EE877A042ACDEDA9
:1071D8000F7A1DD0DDED107A67EE877A052ACDED9E
:1071E800107A15D0DDED117A67EE877A062ACDED93
:1071F800117A0DD0DDED127A67EE877A072ACDED88
:10720800127A05D0DDED137A27EE877A8DED137AA1
:10721800344B1E6816F0805601F09180F6EE005A45
:10722800C4ED815A002A02F0CC842F4BD4ED7F4A5A
:1072380093F8038094F900320A99D4ED7E6A91F8A4
:1072480000E0DFF8B0C02949DFF8AC90B1F90610CA
:107258009CED007A059106EE103AFDEEE44A244BC7
:1072680099F80090B3F81AB094ED7B5AD4ED7C7A73
:1072780014EE903AFDEEE64A00F0100C00F480009F
:107288000EF0010EB8EEC66A14EE901A0690B8F128
:10729800000F41F0EB81DFF84480BCF1000F41F0B2
:1072A800968098ED007ADDED0C6ADFF850C025EE87
:1072B800877AA6EE267AF0EE676AE5EE076ABDEEF3
:1072C800E67A17EE106A17EE100A9E42A8BF184613
:1072D80016E000BF50360020B2310020A02B00205D
:1072E80000000000203400205C6600201C5D0020A7
:1072F800D84E00207C2B0020EC6100206034002058
:10730800B142C8BF084607EE100AB8EEC77A012A8C
:107318008CED007A00F0DC8098ED047ADDED0D6AE2
:1073280025EE877AA6EE267AF0EE676AE5EE076A1A
:10733800BDEEE67A17EE106A17EE100A9E42A8BF55
:107348001846B142C8BF084607EE100AB8EEC77A19
:10735800022A8CED017A00F0BB8098ED087ADDED09
:107368000E6A25EE877AA6EE267AF0EE676AE5EED3
:10737800076ABDEEE67A17EE106A17EE100A9E420B
:10738800A8BF1846B142C8BF084607EE100AB8EEB3
:10739800C77A032A8CED027A00F09A8098ED0C7A6D
:1073A800DDED0F6A25EE877AA6EE867AF0EE676A3B
:1073B800E7EE056ABDEEE67A17EE106A17EE100AD8
:1073C8009E42A8BF1846B142C8BF084607EE100A39
:1073D800B8EEC77A042A8CED037A79D098ED107A42
:1073E800DDED106A25EE877AA6EE867AF0EE676AFA
:1073F800E7EE056ABDEEE67A17EE106A17EE100A98
:107408009E42A8BF1846B142C8BF084607EE100AF8
:10741800B8EEC77A052A8CED047A59D098ED147A1B
:10742800DDED116A25EE877AA6EE867AF0EE676AB8
:10743800E7EE056ABDEEE67A17EE106A17EE100A57
:107448009E42A8BF1846B142C8BF084607EE100AB8
:10745800B8EEC77A062A8CED057A39D098ED187AF5
:10746800DDED126A25EE877AA6EE867AF0EE676A77
:10747800E7EE056ABDEEE67A17EE106A17EE100A17
:107488009E42A8BF1846B142C8BF084607EE100A78
:10749800B8EEC77A072A8CED067A19D098ED1C7ACF
:1074A800DDED136A65EE875AE6EE265AE5EE257A93
:1074B800FDEEE77A17EE900A8342A8BF03468142A1
:1074C800C8BF0B4607EE903AF8EEE77ACCED077A9C
:1074D800BEF1000F40F03882002A40F0308233E2DB
:1074E800AB4B1B78013BDBB2FFF730BAA94B0793D4
:1074F8004FF47A761B68B6FBF3F3C3EB4316A64941
:10750800DFF8B88291F801A0A449B8F9060091F80B
:10751800009003EB8603DE00B6B2B74202F0E480C7
:10752800D5F88810B5F93CE0EB6E4A1C07EE90EAF6
:107538007344012AC5F88820EB66F8EEE77A02F072
:10754800DE80D5ED1E5AD5ED206A07EE102A37EEFB
:10755800E56AB8EEC75A012F86EE057A37EE257A26
:1075680077EEC77A85ED1F7AE7EE866A85ED1E7A93
:10757800F0EE667AC5ED216AC5ED206A02F09484C2
:10758800D5F89C10B5F93EE02B6F4A1C07EE90EA3F
:107598007344012AC5F89C202B67F8EEE77A02F0BD
:1075A800C780D5ED235AD5ED256A07EE102A37EEA8
:1075B800E56AB8EEC75A012F86EE057A37EE257AC6
:1075C80077EEC77A85ED247AE7EE866A85ED237A29
:1075D800F0EE667AC5ED266AC5ED256A02F0988454
:1075E800D5F8B010B5F940E06B6F4A1C07EE90EA89
:1075F8007344012AC5F8B0206B67F8EEE77A02F009
:10760800B080D5ED285AD5ED2A6A07EE102A37EE54
:10761800E56AB8EEC75A012F86EE057A37EE257A65
:1076280077EEC77A85ED297AE6EE276A85ED287A1E
:10763800F0EE667AC5ED2B6AC5ED2A6A02F05C8425
:10764800A8F80600B5F8B430544A013B92F8009007
:10765800A5F8B43007990023B9F1070F4B608B6088
:10766800CB607FF468A905F05DF8059BDFF84C81D5
:10767800C01A94F8B831A8F80000002B3FF460A9AC
:10768800013B84F8B83115B0BDEC0C8BBDE8F08F28
:1076980094ED5E7AB1F90000D4ED5F6AB1F902E0C9
:1076A8003F4AF4EEC76A80EAE0738EEAEE71A3EB14
:1076B800E073F1EE10FAA1EBEE71B8BFF0EE476A95
:1076C8008B42B8BF0B4607EE103A1378B8EEC77A6C
:1076D80027EE287A002B40F01D82324B93ED006A8A
:1076E800B4EECA6AF1EE10FA41F1DC80F7EE005A06
:1076F80075EEC65A3BEE477A65EEAA5A2A4BA7EEB4
:10770800256A93ED007A26EE076AB5EEC06AF1EEB7
:1077180010FA40F21086C9EE865AB7EE007AB0EE3B
:10772800476AA6EEE56AF0EE466AF4EEC76AF1EE3D
:1077380010FA88BFF0EE476AF5EEC06AF1EE10FA6B
:10774800B8BFF0EE6B6A194B93ED007A67EE877A53
:10775800A7EEA68AFFF7E6B9154B164A2B4493ED18
:10776800007AD2ED007A144B67EE277AF7EE006ABA
:10777800F4EEE67AF1EE10FA93ED007A88BFF0EEB7
:10778800667A67EE877A27EE888AFFF77CBA00BFA9
:1077980004360020344D00209C4A0020043200208A
:1077A800342B00203C2B0020302B00202C2B0020D9
:1077B800E01A0020242B0020202B00200832002073
:1077C800072B02F029820026DFF83CB3B64DDBF820
:1077D8000030590501F16B80B44B1B78002B40F049
:1077E800F381B34F94F8123123B1B24A1288920749
:1077F80042F0A88194F81821002A41F06280BB7FEA
:10780800002B00F0F383022B02F01680032B01F00B
:10781800BE82A94B5B88F97F0231C9B2002A01F008
:10782800FC87002B01F0F987A4480068B3FBF0F34C
:107838000FFA83F9A4F84891002903F0458107EE6F
:10784800909AF8EEE77AF7EE006A86EEA77A9C4BF4
:107858000129D4ED576AD3ED007A77EEE67A67EE20
:10786800877AC4ED537A21D0D3ED017AD4ED586AE2
:1078780077EEE67A022967EE877AC4ED547A15D056
:10788800D3ED027AD4ED596A77EEE67A032967EEEA
:10789800877AC4ED557A09D0D3ED037AD4ED5A6AC4
:1078A80077EEE67A67EE877AC4ED567A85480078EF
:1078B800092803F02D81B9F1000F40F39E8391B39D
:1078C80094ED577AD4ED537A77EE877A0129C4ED8F
:1078D800577AC3ED007A21D094ED587AD4ED547AD2
:1078E80077EE877A0229C4ED587AC3ED017A15D06C
:1078F80094ED597AD4ED557A77EE877A0329C4ED59
:10790800597AC3ED027A09D0D4ED5A7A94ED567AB1
:1079180077EE877AC4ED5A7AC3ED037A01390229E2
:10792800B8BF0221C9B2002A18BF022166E30A9B28
:10793800654D1B78DE0700F163812A7822B1920039
:107948006249634824F0EEFB624B1B68002B40F051
:107958002E83614B1B789BB1287870B1DFF870815A
:10796800DFF8A8910026F0B2D9F80030B8EC010A87
:107978009847287801368642F5DB584B1B689847AC
:10798800504B1B78072B00F0DF84012384F800316B
:1079980015B0BDEC0C8BBDE8F08F514BC7ED00BAAC
:1079A8001B689342BFF6FEA84E4B1A88002384F842
:1079B800D031002A41F08E864B4A4C4B117818681A
:1079C80081F00101F9F7B0FBFFF7F4B8484EDFF892
:1079D800409106F5F47806F51577F6EC017A95ED01
:1079E800080AD5F81432F8EEE77A404627EE800AFE
:1079F8009847A8F1E000D5F834319847A8F170000D
:107A0800D5F8A4319847D6F8F400D5F8B830984797
:107A180008F124084745A9EC010ADED1FEF784BF26
:107A28000A9A1278D50703D4214A128BA4F8F421B4
:107A3800304A2349128891ED037A07EE902AF8EE2E
:107A4800E77AB4EEE77AF1EE10FA41F281802A493A
:107A5800098807EE901AF8EEE77AB4EEE77AF1EEC5
:107A680010FAC0F2E7872549254AD1ED006A92ED60
:107A7800006A2449C4ED7E6ABCEEC75A76EE665A9F
:107A880015EE102AC4ED7C6AC4ED7B5A84ED7F6A3A
:107A9800A4F8F4210122D1ED006A84F8002277EEDF
:107AA800677AFFF780B900BFB04A00208A14002027
:107AB800D84E002086380020346600203436002056
:107AC8002C32002004320020B2310020802B00200C
:107AD80060340020B8270020F4640020E86100200A
:107AE800502B0020C8580020CA580020CC5800202D
:107AF800E04A0020342C0020362C0020202C0020C6
:107B0800E03500203C2C0020444D0020E06100209E
:107B1800384D0020CC4B93ED005AB5EEC05AF1EE2B
:107B280010FA40F30884C94BD3ED004AF5EEC04A79
:107B3800F1EE10FA40F3FF8334EEC77A66EEE95AA5
:107B480087EE246AC5EE856AB7EE007AB4EEC76A96
:107B5800F1EE10FA88BFB0EE476AB5EEC06AF1EEF2
:107B680010FA76EE876AB8BFB0EE6B6A66EE266AE0
:107B7800DBE5B74A92ED007AF0EEE76AF4EEC76A01
:107B8800F1EE10FA7FF7A0A8B24A92ED007AF0EE73
:107B9800CD6AF4EEC76AF1EE10FA7FF795A8AE4AFF
:107BA80099ED007AD2ED006AB0EEC77AB4EEE67AC3
:107BB800F1EE10FA7FF588A801220999C4F8D411CA
:107BC80084F8D021FFF784B8A44BA54FB3F9062059
:107BD8007B8B9A423FF706AEA24B1B78012B01F034
:107BE8000786192B01F004860E2B3FF4FBAD082BFA
:107BF8003FF4F8AD9C4B00229A60C4F80C21F1E5E3
:107C08002B78002B3FF4A0AED4ED5F3A94ED5E6A7A
:107C1800D4ED7C7A954A94ED7B7AD2ED005A94EDB6
:107C28005C4AD4ED5B4ADFF85C82DFF85CC2F4EEB4
:107C3800C63AF3EE046AF1EE10FA37EEA65A00F1EE
:107C4800F78798ED026A26EE446AF0EE674AE6EE98
:107C5800074AF4EEC54A34EEE66AF1EE10FA48BF78
:107C6800B0EE656A012B8CED006A3FF46DAE98EDBD
:107C7800066A26EE446AF0EE674AE6EE074AB4EE74
:107C8800E45A34EEE66AF1EE10FA88BFB0EE656A9F
:107C9800022B8CED016A3FF457AE98ED0A6A26EE86
:107CA800446AF0EE674AE6EE074AF4EEC54A34EE57
:107CB800E66AF1EE10FA48BFB0EE656A032B8CED68
:107CC800026A3FF441AE98ED0E6A26EE446AF0EE81
:107CD800674AE6EE074AB4EEE45A34EEE66AF1EE95
:107CE80010FAC8BFB0EE656A042B8CED036A3FF446
:107CF8002BAE98ED126A26EE446AF0EE674AE6EE7D
:107D0800074AB4EEE45A34EEE66AF1EE10FAC8BF58
:107D1800B0EE656A052B8CED046A3FF415AE98ED5C
:107D2800166A26EE446AF0EE674AE6EE074AF4EE73
:107D3800C54A74EEE66AF1EE10FAB8BFF0EE656A6D
:107D4800062BCCED056A3FF4FFADD8ED1A6A66EE56
:107D5800C46AF0EE674AE6EE874AB3EE046AB4EE08
:107D6800E45A74EEC66AF1EE10FAC8BFF0EE656A1E
:107D7800072BCCED066A3FF4E7ADD8ED1E6A26EE78
:107D8800C44AE4EE077AB4EEE75A77EEC67AF1EE23
:107D980010FAC8BFF0EE657ACCED077AD4E50799FA
:107DA800334BD1ED017A93ED007AF0EEE77AF4EEF9
:107DB800C77AF1EE10FA7EF5FDAED1ED027AF0EE5B
:107DC800E77AB4EEE77AF1EE10FA7EF7F3AED1ED8A
:107DD800037AF0EEE77AB4EEE77AF1EE10FA7EF77E
:107DE800E9AE244B1B689A077FF5DEAD2249234B89
:107DF800B3F90C20B1F900E02148AEEB020E00689F
:107E08008EEAEE72A2EBEE728242BEF6D3AEB3F900
:107E18000E30B1F90220D21A82EAE273A3EBE273C0
:107E280098427EF7C7AEBFE50B4B99ED007AD3EDCC
:107E3800006AB0EEC77AB4EEE67AF1EE10FA7EF791
:107E480059AFFEF754BF00BF302B0020382B00205D
:107E5800642B0020602B0020682B00201C5D002074
:107E6800D84E0020503600202C3200207C2B0020D9
:107E78005C2B0020E06500202C66002010360020D6
:107E8800582B0020A02B00206034002007EE103A69
:107E9800524BDFF854811B78C4F8A071B8EEC77A4A
:107EA800F7EE006A132B86EE879AB8F90400B4F847
:107EB800A47195ED080A01F07583494B494A93ED81
:107EC800001A93ED053A93ED122A93ED176AD3ED54
:107ED800091A93ED0E4AD3ED015AD3ED063A93ED04
:107EE8000A7A93ED0F5AD3ED132AD3ED186AD3ED1E
:107EF800044AD3ED030A67EE897A69EE288A29EEE7
:107F0800088AA1EE273A02EB87060021A2EE286A2A
:107F1800C4F89411C4F89811A1EE884AE5EEA73A7E
:107F2800A7EE085A93ED167AD3ED0D5A93ED021A7F
:107F3800D3ED0C1A86ED003AE2EEA86A64EEC34A65
:107F480027EE467A93ED0B2AD3ED152A86ED204AC3
:107F5800E0EEC33A65EEC45A93ED143AC3ED053A20
:107F6800E1EE274AF0EE477AA1EEC45AE2EE085A4B
:107F7800E2EEC66AE3EE287AC3ED064A83ED0E5AAE
:107F8800C3ED0F5A86ED406AC3ED176AC3ED187A40
:107F9800C4F89C117B1C03F01F03A4F8A431A8F8B3
:107FA8000400FEF7A3BBB0EE465AFEF735BF0AF051
:107FB80085FBCEE496ED007A05EB4702B8EEC78A5A
:107FC800928F2AF8172028EE278AFEF77BBC24F028
:107FD8001DFA2AF81700FEF797BC00BF04320020EC
:107FE800E03F00205C3D002008320020A4F8483122
:107FF8009946002A00F07281D74B0221D74ADFED5B
:10800800D86A1068D74A90F802C092F800E002785F
:1080180007EE902AF8EEE77AB0EE007A67EEA67AD5
:10802800F4EEC77AF1EE10FA40F30E8337EEC77A12
:10803800DFEDCD6AB0EE676AA7EE266AB0EE467A43
:108048009FEDCA6AD3ED006A66EE866AB0EEE66A0C
:10805800C4ED5B6A84ED5E6ABCF1000F13D005EED7
:1080680090CAB8EEE55ADFEDBE5A66EEA64A25EE8E
:10807800255AF7EE005A75EEC55A64EE864AE4EEC4
:10808800855A66EEA56ADFEDBA5A427927EE257A57
:1080980027EE267ACAB1DFEDB26ADFEDB65A26EED0
:1080A800266A06EE902AF8EEE66A26EE266AB4EE0E
:1080B800E56AF1EE10FA00F38085F7EE005A35EE26
:1080C800C66AC5EE866A27EE267ABEF10C0F9FEDCA
:1080D800AA8ADFEDAA6A00F00985B4EEC87AF1EE43
:1080E80010FA98BFB0EE478AB4EEE68AF1EE10FABD
:1080F800B8BFB0EE668A84ED418A002900F0E280BC
:10810800B0EE007AF4EEC77AF1EE10FA05DD37EE3C
:10811800C77ADFED956AE7EE267A93ED017ADFED0F
:10812800936A27EE267AB0EEC76A84ED5C7A84ED0E
:108138005F6ABCF1000F13D006EE90CADFED885AD3
:10814800F8EEE66A27EE075A66EEA56AF7EE005AD9
:1081580075EEE65A25EE065AE5EE265A27EE257AFA
:10816800DFED836A827967EEA67A67EE877AAAB12D
:1081780007EE102AB8EEC77ADFED795ADFED7D6A8F
:1081880027EE067A27EE257AB4EEE67AF1EE10FAB3
:1081980040F30585DFED7A6A67EEA67ABEF10C0F2B
:1081A80000F08384DFED746A9FED747AF4EEE67A6A
:1081B800F1EE10FA88BFF0EE667AF4EEC77AF1EEC7
:1081C80010FAB8BFF0EE477A0129C4ED427A79DD9A
:1081D8004278DFED636A07EE902AF8EEE77AB0EEB0
:1081E800007A67EEA67A427AF4EEC77AF1EE10FAD0
:1081F80005DD37EEC77ADFED5C6AE7EE267A93EDA8
:10820800027ADFED5A6A27EE267AB0EEC76A84ED65
:108218005D7A84ED606A9AB106EE902ADFED505AD5
:10822800F8EEE66A27EE075A66EEA56AF7EE005AF8
:1082380075EEE65A25EE065AE6EE855A27EE257AB9
:10824800DFED4B6AC37967EEA67A67EE877A0BB3E0
:1082580007EE103AB8EEC77ADFED415ADFED456A0E
:1082680027EE067A27EE257AB4EEE67AF1EE10FAD2
:108278000CDCB5EEC07AF1EE10FA01F1C082B7EE6F
:10828800006A36EE477AC6EE076A01E0DFED3C6A1F
:1082980067EEA67ABEF10C0F00F04584DFED366A72
:1082A8009FED367AF4EEE67AF1EE10FA88BFF0EE3A
:1082B800667AF4EEC77AF1EE10FAB8BFF0EE477AB4
:1082C800C4ED437ABEF1090F00F0D38397F821700B
:1082D800002F40F06A83002384F81831294B1B785B
:1082E80023B9294FBB78002B41F0AD821D4B1B7879
:1082F800072B00F022840022072B84F800217EF44B
:10830800A2A904F00FFA0590FEF79FB91F4B204C65
:108318001A68204BDFF8888094F80001D2691B881E
:10832800A8F80020A8F8023000287FF44CAA05908D
:10833800194DFEF78AB9DFED196AFFF704BA410251
:108348003EF56CAFFEF76EBF04F0ECF9144BC01BA2
:10835800D880FFF71ABB00BF2C320020E866002047
:108368000AD7233C04320020D7A368416F12033B8D
:1083780000004843A4707D3F00C0F94400C0F9C420
:108388000000C8429165002020420020A83A002041
:1083980068190020AE2C0020B04A00200000000020
:1083A8000832002004F0BEF9A94B0B9A1B78DFF8BD
:1083B800B482801A012BA8F8020000F0E082072B93
:1083C8007EF4C0AC04F0AEF90746FEF7BCBCBEF1C3
:1083D800000F41F05B8498ED007ADDED0C6ADFF860
:1083E80088C225EE877AA6EE867AF0EE676AE7EE0F
:1083F800056ABDEEE67A17EE106A17EE100A9E427D
:10840800A8BF1846B142C8BF084607EE100AB8EE22
:10841800C77A012A8CED007A3FF491AA98ED047A84
:10842800DDED0D6A25EE877AA6EE867AF0EE676AAC
:10843800E7EE056ABDEEE67A17EE106A17EE100A47
:108448009E42A8BF1846B142C8BF084607EE100AA8
:10845800B8EEC77A022A8CED017A3FF470AA98ED3B
:10846800087ADDED0E6A25EE877AA6EE867AF0EEBA
:10847800676AE7EE056ABDEEE67A17EE106A17EE50
:10848800100A9E42A8BF1846B142C8BF084607EE68
:10849800100AB8EEC77A032A8CED027A3FF44FAA85
:1084A80098ED0C7ADDED0F6A25EE877AA6EE867ACE
:1084B800F0EE676AE7EE056ABDEEE67A17EE106A37
:1084C80017EE100A9E42A8BF1846B142C8BF084618
:1084D80007EE100AB8EEC77A042A8CED037A3FF447
:1084E8002EAA98ED107ADDED106A25EE877AA6EEB1
:1084F800867AF0EE676AE7EE056ABDEEE67A17EE71
:10850800106A17EE100A9E42A8BF1846B142C8BFAB
:10851800084607EE100AB8EEC77A052A8CED047AE9
:108528003FF40DAA98ED147ADDED116A25EE877AED
:10853800A6EE867AF0EE676AE7EE056ABDEEE67AA1
:1085480017EE106A17EE100A9E42A8BF1846B142ED
:10855800C8BF084607EE100AB8EEC77A062A8CED9F
:10856800057A3FF4ECA998ED187ADDED126A25EE4C
:10857800877AA6EE867AF0EE676AE7EE056ABDEEC0
:10858800E67A17EE106A17EE100A9E42A8BF184640
:10859800B142C8BF084607EE100AB8EEC77A072AE4
:1085A8008CED067A3FF4CBA998ED1C7ADDED136AC1
:1085B80065EE875AE6EE265AE5EE257AFDEEE77A6D
:1085C80017EE900A8342A8BF03468142C8BF0B46F4
:1085D80007EE903AF8EEE77ACCED077A002A7FF4B6
:1085E800AEA9FFF7B1B91B4B5A79002A3EF499ACF2
:1085F800194A1278002A3EF494AC1B78DFED174A2A
:1086080007EE903A164BB8EE677A1B8807EE902A69
:1086180006EE903AF8EEE77AF8EE666A67EE277AA1
:10862800B7EE007AC7EEA63AF4EEE43AF1EE10FAA5
:1086380088BFF0EE643AF4EEC73AF1EE10FAB8BF2C
:10864800F0EE473AFEF76FBCB0EE677AF8E400BF89
:10865800043200204C6600202A320020713DAA3FD7
:10866800143200200832002060340020BCF1000FD2
:1086780000F09783BEF1000F41F0A287DFF8A485D0
:10868800B9F1000F41F0E185D8ED006ADDED0C4A43
:10869800DFF894C565EEA66ABDEEC77A17EE101A24
:1086A800B0EE667AA4EE867AF0EE676AE7EE056ABF
:1086B800BDEEE67A17EE106A17EE100A9E42A8BFC2
:1086C8001846B142C8BF084607EE100AB8EEC77A86
:1086D800012A8CED007A3FF432A998ED047ADDED99
:1086E8000D6A25EE877AA6EE867AF0EE676AE7EEDF
:1086F800056ABDEEE67A17EE106A17EE100A9E427A
:10870800A8BF18468E42B8BF084607EE100AB8EE52
:10871800C77A022A8CED017A3FF411A998ED087AFC
:10872800DDED0E6A25EE877AA6EE867AF0EE676AA8
:10873800E7EE056ABDEEE67A17EE106A17EE100A44
:108748009E42A8BF18468E42B8BF084607EE100AD8
:10875800B8EEC77A032A8CED027A3FF4F0A898EDB8
:108768000C7ADDED0F6A25EE877AA6EE867AF0EEB2
:10877800676AE7EE056ABDEEE67A17EE106A17EE4D
:10878800100A9E42A8BF18468E42B8BF084607EE98
:10879800100AB8EEC77A042A8CED037A3FF4CFA802
:1087A80098ED107ADDED106A25EE877AA6EE867AC6
:1087B800F0EE676AE7EE056ABDEEE67A17EE106A34
:1087C80017EE100A9E42A8BF18468E42B8BF084648
:1087D80007EE100AB8EEC77A052A8CED047A3FF442
:1087E800AEA898ED147ADDED116A25EE877AA6EE2B
:1087F800867AF0EE676AE7EE056ABDEEE67A17EE6E
:10880800106A17EE100A9E42A8BF18468E42B8BFDB
:10881800084607EE100AB8EEC77A062A8CED057AE4
:108828003FF48DA898ED187ADDED126A25EE877A67
:10883800A6EE867AF0EE676AE7EE056ABDEEE67A9E
:1088480017EE106A17EE100A9E42A8BF18468E420D
:10885800B8BF084607EE100AB8EEC77A072A8CEDAB
:10886800067A3FF46CA898ED1C7ADDED136A65EE84
:10887800875AE6EE265AE5EE257AFDEEE77A17EEF8
:10888800900A8342A8BF03468142D8BF194607EE23
:10889800901AF8EEE77ACCED077A002A7FF44FA811
:1088A800FFF752B8C74B93ED006AFEF72EBFAB68CF
:1088B800002B3EF491AF05F1500128469847FEF78A
:1088C8008BBFC14BC149D3F8EC30086844F620612E
:1088D8008B42A8BF0B46B3F57A7FB8BF4FF47A73C3
:1088E80099B2C006A4F81A11DBF8003041F1D7821A
:1088F800DB0400F16B83B64BD3F800C0BCF932E05F
:10890800B44BB548D3ED037AD4F81C31A0FB010170
:108918008809642191FBF0F11429BDEEE77A04EB94
:108928004308A8BF142101339942C4F81C3117EE3B
:10893800109ADCBF0023C4F81C3104EB4303A8F8E9
:108948002091B3F9203107EE103AB8EEC77A77EEE6
:10895800C77AFDEEE77ACDED057ABDF9141081EA04
:10896800E173A3EBE173734502F397809B4B1946C0
:108978004FF07E530B60FEF742BFDFF8B08203F082
:10898800D1FE974AD4F8E4311268C4F8E401C31A56
:108998009A1A0746A8F80430A8F80620FEF7D3B9B3
:1089A80003F0C0FE0B90FDF7DABF1E218748F9F7E8
:1089B80088FA00283FF48FAC8A4B1B885A063FF58B
:1089C8008AAC94F88431BB4242F0C880834BD4ED22
:1089D800627A93ED010AD4ED435A9FED836ADFED85
:1089E800836A27EEE57A68EE277AA8EE007AE5EE44
:1089F800807AB4EEC67AF1EE10FA88BFB0EE467A05
:108A0800B4EEE67AF1EE10FAF4EEC67AB8BFB0EE3C
:108A1800667AF1EE10FA88BFF0EE467AF4EEE67A5E
:108A2800F1EE10FAB8BFF0EE667A84ED417AC4ED43
:108A3800437A50E4B4F8F411914240F282856C49CB
:108A48006C4AD1ED007A92ED007A6B49C4ED7E7ADA
:108A580077EE676AC4ED7C7A0122C4ED7B6A84ED07
:108A68007F7AD1ED006ADFED657A84F80022FEF79F
:108A78009AB9FDEEC87ADFF8B48117EE903AA8F8F3
:108A88000490A8F8063021E45D4B1B88002B40F0C9
:108A980077855C4A5C4B11781868F8F745FBD4F881
:108AA800D421099B9A1AFEF754B89FED4F7ADFED4F
:108AB8004F6ADFF87881F4EEC77AF1EE10FA98BFC2
:108AC800B0EE677AFDEEE77AB4EEE67AF1EE10FAE8
:108AD80017EE902AB8BFB0EE667A012984ED427A83
:108AE800A8F802203FF774ABFFF7F0BBB4EEC87AE2
:108AF800F1EE10FA98BFB0EE478ABDEEC77AB4EE31
:108B0800E68ADFF82881F1EE10FA17EE102AB8BFCE
:108B1800B0EE668A84ED418AA8F8002000297FF427
:108B2800EFAAFFF7D3BBBDEEE77ADFF8008117EEB7
:108B3800103AA8F80430FFF7B1BB03F0F3FDDFF8F3
:108B4800EC80324B801B1B78A8F80400FFF7D3BBDE
:108B58002F4A3049D2ED006A2F4A91ED006A127807
:108B6800C4ED7E6A84ED7F6A002A40F0E68476EEE2
:108B7800C65AF0EE466ABCEEC76A2849C4ED7B5A6D
:108B880016EE102AC4ED7C6AA4F8F421FF22D1ED78
:108B9800006A84F8002277EEC77AFEF704B9B5EECA
:108BA800C07AF1EE10FA00F12E86B7EE006A36EEC2
:108BB800477AC6EE076AFFF7EFBADFED196AFFF7E3
:108BC80082BA00BF302B00201C0100202034002076
:108BD800B86500202C320020D34D621078000020A8
:108BE800343600208638002000C0F94400C0F9C49B
:108BF800202C0020E03500203C2C00200000000044
:108C0800C8580020CA580020CC5800200432002040
:108C180088340020242C0020EC610020382C00200F
:108C28000000C842A02B0020603400200832002039
:108C380098ED016A26EE646AB0EE674AA6EE074A26
:108C4800B4EEC45A34EE666AF1EE10FAC8BFB0EE5C
:108C5800656A012B8CED006A3EF476AE98ED056AE4
:108C680026EE646AB0EE674AA6EE074AB4EEC45A26
:108C780034EE666AF1EE10FAC8BFB0EE656A022BF0
:108C88008CED016A3EF460AE98ED096A26EE646ADE
:108C9800B0EE674AA6EE074AB4EEC45A34EE666AE6
:108CA800F1EE10FAC8BFB0EE656A032B8CED026ACC
:108CB8003EF44AAE98ED0D6A26EE646AB0EE674A55
:108CC800A6EE074AB4EEC45A34EE666AF1EE10FA1C
:108CD800C8BFB0EE656A042B8CED036A3EF434AE6F
:108CE80098ED116A26EE646AB0EE674AA6EE074A66
:108CF800B4EEC45A34EE666AF1EE10FAC8BFB0EEAC
:108D0800656A052B8CED046A3EF41EAE98ED156A73
:108D180026EE646AB0EE674AA6EE074AB4EEC45A75
:108D280074EE666AF1EE10FAC8BFF0EE656A062BBB
:108D3800CCED056A3EF408AED8ED196A66EEE46A31
:108D4800B0EE674AA6EE874AB3EE046AB4EEC45A98
:108D580074EE466AF1EE10FAC8BFF0EE656A072BAA
:108D6800CCED066A3EF4F0ADD8ED1D6A66EEE44A35
:108D7800E4EE877AF4EEC57A77EEC67AF1EE10FA69
:108D8800B8BFF0EE657ACCED077AFEF7DDBD97F84F
:108D98002030C3EB431103EB8103DB009BB2FEF7EA
:108DA8003ABDDFF80485B9F1000F41F0E480D8ED51
:108DB800006ADDED0C4ADFF8F4C465EEA66ABDEE84
:108DC800C77A17EE101AB0EE667AA4EE867AF0EE3D
:108DD800676AE7EE056ABDEEE67A17EE106A17EEE7
:108DE800100A9E42A8BF1846B142C8BF084607EEFF
:108DF800100AB8EEC77A012A8CED007A3EF468AB07
:108E080098ED047ADDED0D6A25EE877AA6EE867A6E
:108E1800F0EE676AE7EE056ABDEEE67A17EE106ACD
:108E280017EE100A9E42A8BF18468E42B8BF0846E1
:108E380007EE100AB8EEC77A022A8CED017A3EF4E2
:108E480047AB98ED087ADDED0E6A25EE877AA6EE37
:108E5800867AF0EE676AE7EE056ABDEEE67A17EE07
:108E6800106A17EE100A9E42A8BF18468E42B8BF75
:108E7800084607EE100AB8EEC77A032A8CED027A84
:108E88003EF426AB98ED0C7ADDED0F6A25EE877A75
:108E9800A6EE867AF0EE676AE7EE056ABDEEE67A38
:108EA80017EE106A17EE100A9E42A8BF18468E42A7
:108EB800B8BF084607EE100AB8EEC77A042A8CED48
:108EC800037A3EF405AB98ED107ADDED106A25EED5
:108ED800877AA6EE867AF0EE676AE7EE056ABDEE57
:108EE800E67A17EE106A17EE100A9E42A8BF1846D7
:108EF8008E42B8BF084607EE100AB8EEC77A052AB0
:108F08008CED047A3EF4E4AA98ED147ADDED116A4A
:108F180025EE877AA6EE867AF0EE676AE7EE056AAE
:108F2800BDEEE67A17EE106A17EE100A9E42A8BF49
:108F380018468E42B8BF084607EE100AB8EEC77A40
:108F4800062A8CED057A3EF4C3AA98ED187ADDED71
:108F5800126A25EE877AA6EE867AF0EE676AE7EE61
:108F6800056ABDEEE67A17EE106A17EE100A9E4201
:108F7800A8BF18468E42B8BF084607EE100AB8EEDA
:108F8800C77A072A8CED067A3EF4A2AA98ED1C7AD5
:108F9800DDED136A65EE875AE6EE265AE5EE257A88
:108FA800FDEEE77A17EE900A8342A8BF0346814296
:108FB800D8BF194607EE901AF8EEE77ACCED077A93
:108FC800BEF1000F7EF4C0ACFEF786BAAA4BD3F808
:108FD80000C0BCF832E04FEA5E0E91E4DFF8D092B0
:108FE800D4ED017A94ED006AB9F80000D9F814308C
:108FF80077EEA77AF0EE006AB0EE677AA6EE267AE8
:10900800013804EBC002D6EE267A083A1033F6EEA1
:10901800003A27EE237A67EEA37A84ED207AC4ED2E
:10902800217A964CA64604F1800192ED027A92EDDF
:10903800036ADEED036ADEED027A53ED014A13EDB1
:10904800025A37EE674A76EEC65A77EE277AE4EE8A
:10905800845A0138A2F10802E5EE047A0EF1080EEE
:1090680003F1080336EE267A01F10801E4EE877A67
:10907800E5EE475A67EEA37A25EEA37AC1ED007AAA
:1090880081ED017AD1D1142F7DF4EBAB03F04AFBCB
:10909800069BDFF82082C01AA8F80200D4F8A8615D
:1090A800FDF7DFBBD4F8AC81B4F8A4A1744BCAF1C6
:1090B80020095FFA89F90AEB481E03EB8E0E5FEA76
:1090C800990301F0F185013318016E496E4A0EEBE0
:1090D800000C0EF1100313ED024A13ED035A13EDC1
:1090E800016A13ED047A51ED024A51ED035A51ED2C
:1090F800016A51ED047A64EE244A65EE255A66EE5B
:10910800266A67EE277A10339C4542ED024A42ED03
:10911800035A42ED016A42ED047A01F1100102F1AD
:109128001002D8D15949A0F11002964401EB020C63
:10913800224419F0030309D0BEEC017AFCEC017A51
:1091480067EE277A013BE2EC017AF5D1BAF1000F1C
:1091580041F0D481142F7DF484AB03F0E3FA069B2D
:10916800DFF85081D4F8A861C01AA8F80200FDF70A
:1091780078BBDFF83C914148D9F80820B9F80C10C1
:1091880022F03EF8424B1F78142F01F0A185D4F845
:10919800A8610136C4F8A86122E7D4F8AC913D4B28
:1091A8003D4ADFED3E7AD2ED008A3D4A4FEAC901D9
:1091B8000B44F8EE688A9B8809EE103A643BC82B8A
:1091C800A8BFC82368EEA78AF8EE497A782BB8BFFB
:1091D800782368EEA78A07EE903A4944B0EE680A09
:1091E80002EB8108B8EEE78A23F05CF9B8EEC99A79
:1091F800F0EE409AB0EE680A23F0B6F838EE097A35
:1092080079EE487A28EE098A67EE877AB7EE006A1F
:1092180088EE277A142FF8EE007A77EE076A60EE68
:10922800277A89EEA67A77EE065A36EE477AC6EEA0
:10923800256A67EEA67A27EE267AC8ED006A88EDD9
:10924800047AC8ED026AC8ED017AC8ED037A01F024
:109258009185144B0E4A09F1010983FB0938A8EBE3
:10926800E97808EB48080136A9EB08081778C4F82C
:10927800A861C4F8AC8117E7B86500206819002018
:109288005C3D0020EC3E002078190020DC3E0020E8
:10929800043200205C3F0020344D002027D4D23611
:1092A800C84C002056555555A02B0020603400208E
:1092B800443D002008320020DFF80494B9F800E0AB
:1092C800D9F804C04FEA5E084FEA880204EB8E061C
:1092D8005FEADE0E04EB020300F0A08010320EF10C
:1092E800010EEB4803EB0E1E324410330CF110074D
:1092F80006F1100151ED032A51ED043A10ED043A3C
:1093080010ED032A51ED026A11ED016A10ED020A0F
:1093180010ED018A12ED044A12ED035A53ED044A86
:1093280053ED035A13ED027A53ED017A52ED020A16
:1093380012ED011A73EE238A72EE221A40ED048AA6
:1093480040ED031A70EE268A78EE061A40ED028A7E
:1093580040ED011A74EE848A75EE851A43ED048A8D
:1093680043ED031A77EE208A77EE811A43ED028ADD
:1093780043ED011A73EE633A75EE655A17ED035A19
:1093880032EE623A74EE644A65EE631A17ED044AE7
:1093980023EE052A64EE652AE3EE041A10339E458F
:1093A80024EE843AA3EE842A00F1100007F1100796
:1093B800A5EE853A01F1100102F11002E4EE852ACA
:1093C80041ED071A01ED082A02ED073A42ED082A95
:1093D80057ED055A17ED065A70EE666A38EE466A7A
:1093E80030EEC77A71EE677A26EE253A65EEE63AF0
:1093F80025EE674A67EE054AE6EE053AA6EE853A97
:10940800A7EE254AE7EEA54A01ED063A41ED053AF1
:1094180002ED064A42ED054A7FF46CAF1FFA88F860
:10942800624641469B4821F059F84146D9F8042044
:10943800304621F053F8984B1B78142B7FF42EAE4E
:1094480024E6DFF8809299F80020900801F014854E
:10945800DFF874C200F101084FEA48180CEB080E57
:109468000CF12003ACF1700113ED076A53ED056AA6
:1094780013ED037A53ED017A53ED025A13ED084ABE
:1094880053ED064A13ED045A26EE066A66EEA66AFE
:1094980027EE077A67EEA77AA4EE046A20339E4582
:1094A800E4EEA46A01F11001A5EE057AE5EEA57ACD
:1094B800F1EEC65AB1EEE66AF1EEC76AB1EEE77AA6
:1094C80041ED085A01ED076A41ED066A01ED057A9A
:1094D800CAD1A8F12008C44404EB001012F0030319
:1094E80018BF0CF1080C0FD05CED017A1CED027A64
:1094F80067EEA77A013BE7EE077A0CF1080CB1EEAC
:10950800E77AA0EC017AEFD1142F01F05C840136E0
:10951800C4F8A861FDF70EB903F004F95E4B069094
:109528001F78142F05BFDFF8A481D4F8A861D4F8F8
:10953800A861A8F80060FDF7E2B876EE665AFFF772
:109548001ABB564A5649D2ED007A564A91ED007A2E
:109558001278C4ED7E7A84ED7F7A002A01F0978232
:1095680077EE676A5049C4ED7C7AC4ED7B6AFF22C6
:10957800D1ED006ADFED4D7A84F80022FDF713BCC7
:109588004B494B69002B3DF4E4AA4A484A4B0088F2
:1095980093FBF0F00B684FF0010E186081F811E0B2
:1095A800FDF7D7BA454EDFF8289196ED004A96EDBB
:1095B800057AD6ED014A96ED066AD6ED046A96ED6F
:1095C800035AD6ED025A67EE897A09EB8703A4EEAF
:1095D800277AA4EEA76A66EEC76AA5EE476AE5EEA3
:1095E800A76A20EE070A86ED056AC6ED066A83EDCE
:1095F800007A29EE088A22F009FF69EE288AD6ED5A
:109608000E5AD6ED176A96ED091AD6ED121A96ED8E
:109618000F5A96ED187A96ED0A2AD6ED132A96ED8A
:109628000D6AD6ED167A96ED0C3AD6ED0B3A96ED14
:10963800154AD6ED144AE1EE085A002209EB8703D1
:10964800E8EEA16A00B2C4F89421A2EE085AC4F860
:109658009821C4F89C21A8EEA27A26EE656A67EEE6
:10966800E67AA3EE655AA3EE886AA6EEC47AE8EE17
:10967800A47A86ED0E5AC3ED205A86ED0F6AC3ED23
:10968800406A86ED177AC6ED187AFEF783BC00BFEC
:10969800781900206819002004320020883400203E
:1096A800242C0020EC610020382C00200000000051
:1096B800D0580020E858002020A10700E03F0020F3
:1096C800443D00203E3D0020E819002008320020DB
:1096D8005C3D0020B3494A69002A3DF46BAA0A6838
:1096E80013604B74FDF766BAB5F93C306A6207EE51
:1096F800903A0122F8EEE77AEB66C5F88820002355
:10970800012FC5ED1F7AC5ED1E7AC5F8803001F02E
:10971800E681B7427DF434AFB5F93E302B6707EEEA
:10972800903A00220123F8EEE77AAA62C5F89C3045
:109738000023012FC5ED247AC5ED237AC5F89430AE
:1097480001F0D181B7427DF44BAFB5F940306B677A
:1097580007EE903A00220123F8EEE77AEA62C5F8AC
:10976800B0300023012FC5ED297AC5ED287AC5F858
:10977800A8307DF465AF9FED8C8AB9F1030F46D010
:10978800BAF1000F09D007EE90AAF8EEE77AF4EEE6
:10979800C87AF1EE10FA01F17483844A6B6F12688B
:1097A80094F8B011A8F8060003EB560393FBF6F6FD
:1097B8000023EE6293621363D36231B17C4B1B8842
:1097C80023F40063002B7DF43DAF7A4B1B6813F440
:1097D800003341F07C8178491A46C85C012803F1BE
:1097E8000C0300F00E850132152AF6D1FDF72ABFC9
:1097F800724B9B7B002B3EF4FDA9FDF7F3BFF7EE00
:10980800006AFEF745BDF7EE006AFEF7C5BCB0EE8C
:10981800480A22F0FBFD00B2B2E7B4F8489109F11A
:10982800FF390FFA89F9B9F1000FA4F848917EF7CA
:10983800E0AB634BFEF743B8B4F81A3103F57A731B
:109848009BB2FDF7E8BFDFF88C8198F80020013A59
:109858000D2A18D8DFE812F097006A011901FC00F8
:1098680017001700E5005501C00080006C0060007B
:1098780055000E001F20059320F050F8059B10B9E5
:10988800012288F80020012B00F01E86FA78002AB1
:109898003EF42CAD4B4A1278D00706D405930CF051
:1098A80027FD059B002841F07382474FD4F890119B
:1098B8003A68914201F2738298F80030012B3EF425
:1098C80015AD94F88C21002A3EF410AD0B2B0DD861
:1098D80001229A4040F6030112EA01090CD112F460
:1098E800C06F03D0093B012B41F26484374B3A68BF
:1098F8005A600B2388F80030002384F88C31FEF777
:10990800F5BC012B01F022830E23132088F80030C8
:1099180018F024F8BB78B6E7012B01D1F8F776FCEC
:109928000D23132088F8003018F018F8BB78AAE740
:10993800264A254952680968C8328A4204D322F067
:10994800B7FBBB7800289ED0032B01F01B830123B3
:1099580088F80030BB7896E71D4B1B78002B01F088
:1099680086821A201FF0DAFF002841F0808294F8DE
:109978008C31002B41F07B82092388F8003010F0ED
:1099880005FBBB787FE70F4B1B78DB0701F1E9820A
:109998001F201FF0C3FF0028BCD00C2388F800301C
:1099A800B8E700BFD058002000000000A83A002007
:1099B80080660020D429002060F50208005F00209E
:1099C8002C320020A4310020F0580020E43500207B
:1099D800A43600201D4200201A201FF09FFF0028F7
:1099E800CDD0994B1B88002BC9D1984B4520D3F873
:1099F800009021F07BFA0E2021F078FA484621F0F9
:109A08003FFBDDF82490484621F03AFB904A914B01
:109A180012681A6048460A2388F8003010F008F8DF
:109A2800ADE721F0B3F98C4B002105208DE8030048
:109A3800A3F108020291532010F0DEFF00287FF402
:109A480069AF864ABB781060082288F800201AE7B8
:109A580021F09CF9824A0292A2F10C03252101937C
:109A68000091A2F10A035021163A492010F0C4FFD0
:109A780000287FF44FAF794ABB7810604FF0FF3170
:109A88005160072288F80020FDE6DFF8D09121F028
:109A98007DF9744AD9F80430126864339342BFF4EC
:109AA80039AF402021F04AF900287FF433AFD9F8C4
:109AB80000306D49DFF8B4B14FF0400A11E005916C
:109AC80021F014FADBF80020D9F800300599013AA2
:109AD8000133BAF1010ACBF80020C9F8003001F0CF
:109AE8000683CB5C1846002BE9D100234FF0FF32E8
:109AF800C9F80030042388F80030C9F80420BB787E
:109B0800C1E621F043F910F07BFA00283FF402AFD8
:109B180022F0CEFA00283FF4FDAE4D4A4D4B1268B4
:109B28001A600A2388F80030BB78ACE64D4A4B49E6
:109B380012684A604D4800220A600321026088F8D2
:109B48000010A0E64A4ADFED4B7A92ED080A059329
:109B5800B4EEE70AF1EE10FA40F2CC8422F0ECFC05
:109B6800D4ED457A20EE270A22F050FCB0F5617F4B
:109B7800059B00F35C8607EE900AF8EEE76ADFEDD6
:109B88003E7A66EEA76A07EE903AB8EEE77AFDEEFF
:109B9800E67A17EE903A2033402B41F224819FED6C
:109BA800370A22F033FC00B207EE900AB8EEE77AE3
:109BB800334BD3ED037A77EE877AC3ED037AFDF75B
:109BC80019BE0A9B93F800E00EF0010EBEF1000FDB
:109BD8007DF4BAAEFDF780BC2A4BDFED2B7A1E6808
:109BE800C4ED707A16F0805640F0238310F4800696
:109BF80000F0B7810026B6EE007A67EE877AF4EEB9
:109C0800E75AF1EE10FA48BFF0EE675A40F11183B7
:109C1800C4ED815AFDF706BB02F084FD0646FDF748
:109C2800D3BD74EE677AB7EE007AF4EEC77AF1EE38
:109C380010FAC4ED707A40F33F8784EEA77A8DED71
:109C48000C7AFDF7E5BA00BF746800207068002040
:109C5800846800207C68002020EF0208E43500209A
:109C680072ED0208F05800200CED0208E0670020B1
:109C7800602900208FC2753CD06D393A0000000081
:109C88002C3200202034002000000080BAF1000FA0
:109C980000F0E78598ED007ADDED0C6ADFF81CC965
:109CA80025EE877AA6EE867AF0EE676AE7EE056A11
:109CB800BDEEE67A17EE106A17EE100A9E42A8BFAC
:109CC8001846B142C8BF084607EE100AB8EEC77A70
:109CD800012A8CED007A3DF437AE98ED047ADDED7B
:109CE8000D6A25EE877AA6EE867AF0EE676AE7EEC9
:109CF800056ABDEEE67A17EE106A17EE100A9E4264
:109D0800A8BF1846B142C8BF084607EE100AB8EE09
:109D1800C77A022A8CED017A3DF416AE98ED087ADE
:109D2800DDED0E6A25EE877AA6EE867AF0EE676A92
:109D3800E7EE056ABDEEE67A17EE106A17EE100A2E
:109D48009E42A8BF1846B142C8BF084607EE100A8F
:109D5800B8EEC77A032A8CED027A3DF4F5AD98ED9A
:109D68000C7ADDED0F6A25EE877AA6EE867AF0EE9C
:109D7800676AE7EE056ABDEEE67A17EE106A17EE37
:109D8800100A9E42A8BF1846B142C8BF084607EE4F
:109D9800100AB8EEC77A042A8CED037A3DF4D4ADE4
:109DA80098ED107ADDED106A25EE877AA6EE867AB0
:109DB800F0EE676AE7EE056ABDEEE67A17EE106A1E
:109DC80017EE100A9E42A8BF1846B142C8BF0846FF
:109DD80007EE100AB8EEC77A052A8CED047A3DF42E
:109DE800B3AD98ED147ADDED116A25EE877AA6EE0B
:109DF800867AF0EE676AE7EE056ABDEEE67A17EE58
:109E0800106A17EE100A9E42A8BF1846B142C8BF92
:109E1800084607EE100AB8EEC77A062A8CED057ACE
:109E28003DF492AD98ED187ADDED126A25EE877A49
:109E3800A6EE867AF0EE676AE7EE056ABDEEE67A88
:109E480017EE106A17EE100A9E42A8BF1846B142D4
:109E5800C8BF084607EE100AB8EEC77A072A8CED85
:109E6800067A3DF471AD98ED1C7ADDED136A65EE66
:109E7800875AE6EE265AE5EE257AFDEEE77A17EEE2
:109E8800902A9342A8BF13468A42A8BF194607EEF4
:109E9800901AF8EEE77ACCED077AFDF755BDD800B1
:109EA8003EF526ADFDF7ABBC012A40F3188607EE58
:109EB800101AB8EEC77AC7EE876AB1EEE68AB9F12A
:109EC800030F13D0BAF1000F09D007EE90AAF8EEED
:109ED800E77AF4EEC87AF1EE10FA00F1D287EB6E69
:109EE80003EB560393FBF6F36B6212E4B0EE480AF9
:109EF80022F08CFA00B2E5E7012A7FF73CAC07EEC6
:109F0800101AB8EEC77AC7EE876AB1EEE68A34E46B
:109F1800012A40F3E88507EE101AB8EEC77AC7EEB3
:109F2800876AB1EEE68AB9F1030F14D0BAF1000FCF
:109F380009D007EE90AAF8EEE77AF4EEC87AF1EEC7
:109F480010FA00F19E872B6F03EB560393FBF6F391
:109F5800AB62FFF7F7BBB0EE480A22F057FA00B23F
:109F6800E4E7B6EE007AF4EEC75AF1EE10FA3FF7DE
:109F780042AEFDF757B9D8ED004A9DED0C4ADFF81F
:109F88003CC665EEA44AFDEEC73AE4EE064AB0EEDA
:109F9800674AA4EE854A13EE901AF4EEC46AF1EE0D
:109FA80010FAF0EE444A88BFF0EE474AFDEEE44A64
:109FB80014EE900A14EE906A9842A8BF1E46814299
:109FC800C8BF0E4604EE906AF8EEE44A012ACCEDCA
:109FD800004A3DF47DAAD8ED044A9DED0D4A65EE90
:109FE800A44AE4EE064AB0EE674AA4EE854AF4EEC7
:109FF800C46AF1EE10FAF0EE444A88BFF0EE474A20
:10A00800FDEEE44A14EE900A14EE906A9842A8BF56
:10A018001E468842B8BF0E4604EE906AF8EEE44A3F
:10A02800022ACCED014A3DF453AAD8ED084A9DED29
:10A038000E4A65EEA44AE4EE064AB0EE674AA4EE7C
:10A04800854AF4EEC46AF1EE10FAF0EE444A88BF8D
:10A05800F0EE474AFDEEE44A14EE900A14EE906AD8
:10A068009842A8BF1E468842B8BF0E4604EE906AC2
:10A07800F8EEE44A032ACCED024A3DF429AAD8EDC9
:10A088000C4A9DED0F4A65EEA44AE4EE064AB0EE8E
:10A09800674AA4EE854AF4EEC46AF1EE10FAF0EECF
:10A0A800444A88BFF0EE474AFDEEE44A14EE900AAF
:10A0B80014EE906A9842A8BF1E468842B8BF0E4662
:10A0C80004EE906AF8EEE44A042ACCED034A3DF423
:10A0D800FFA9D8ED104A9DED104A65EEA44AE4EEBA
:10A0E800064AB0EE674AA4EE854AF4EEC46AF1EE79
:10A0F80010FAF0EE444A88BFF0EE474AFDEEE44A13
:10A1080014EE900A14EE906A9842A8BF1E46884240
:10A11800B8BF0E4604EE906AF8EEE44A052ACCED84
:10A12800044A3DF4D5A9D8ED144A9DED114A65EECF
:10A13800A44AE4EE064AB0EE674AA4EE854AF4EE75
:10A14800C46AF1EE10FAF0EE444A88BFF0EE474ACE
:10A15800FDEEE44A14EE900A14EE906A9842A8BF05
:10A168001E468842B8BF0E4604EE906AF8EEE44AEE
:10A17800062ACCED054A3DF4ABA9D8ED184A9DED69
:10A18800124A65EEA44AE4EE064AB0EE674AA4EE27
:10A19800854AF4EEC46AF1EE10FAF0EE444A88BF3C
:10A1A800F0EE474AFDEEE44A14EE900A14EE906A87
:10A1B8009842A8BF1E468842B8BF0E4604EE906A71
:10A1C800F8EEE44A072ACCED064A3DF481A9D8ED19
:10A1D8001C4A9DED134A65EEA45AE6EE045AE5EED4
:10A1E800257AF4EEE76AF1EE10FAC8BFF0EE477A86
:10A1F800FEF7D6BE8223FCF720BBDFEDEB7AFCF737
:10A20800E7BAD4F8B46153003EB1981801EB800066
:10A2180076784078B042BDF415AA134401EB830167
:10A228000023C4F8B411A4F80832C4F80C32FDF7BE
:10A2380009BAB7EE007A77EE677AF4EEE75AF1EEEC
:10A2480010FA88BFF0EE675AE2E4D8ED004A9DEDB7
:10A258000C4ADFF868C365EEA44AFDEEC73AE4EE9F
:10A26800064AB0EE674AA4EE854A13EE901AF4EE59
:10A27800C46AF1EE10FAF0EE444A88BFF0EE474A9D
:10A28800FDEEE44A14EE900A14EE906A9842A8BFD4
:10A298001E468142C8BF0E4604EE906AF8EEE44AB4
:10A2A800012ACCED004A3DF44AABD8ED044A9DEDB5
:10A2B8000D4A65EEA44AE4EE064AB0EE674AA4EEFB
:10A2C800854AF4EEC46AF1EE10FAF0EE444A88BF0B
:10A2D800F0EE474AFDEEE44A14EE900A14EE906A56
:10A2E8009842A8BF1E468842B8BF0E4604EE906A40
:10A2F800F8EEE44A022ACCED014A3DF420ABD8ED51
:10A30800084A9DED0E4A65EEA44AE4EE064AB0EE10
:10A31800674AA4EE854AF4EEC46AF1EE10FAF0EE4C
:10A32800444A88BFF0EE474AFDEEE44A14EE900A2C
:10A3380014EE906A9842A8BF1E468842B8BF0E46DF
:10A3480004EE906AF8EEE44A032ACCED024A3DF4A2
:10A35800F6AAD8ED0C4A9DED0F4A65EEA44AE4EE44
:10A36800064AB0EE674AA4EE854AF4EEC46AF1EEF6
:10A3780010FAF0EE444A88BFF0EE474AFDEEE44A90
:10A3880014EE900A14EE906A9842A8BF1E468842BE
:10A39800B8BF0E4604EE906AF8EEE44A042ACCED03
:10A3A800034A3DF4CCAAD8ED104A9DED104A65EE5B
:10A3B800A44AE4EE064AB0EE674AA4EE854AF4EEF3
:10A3C800C46AF1EE10FAF0EE444A88BFF0EE474A4C
:10A3D800FDEEE44A14EE900A14EE906A9842A8BF83
:10A3E8001E468842B8BF0E4604EE906AF8EEE44A6C
:10A3F800052ACCED044A3DF4A2AAD8ED144A9DEDF5
:10A40800114A65EEA44AE4EE064AB0EE674AA4EEA5
:10A41800854AF4EEC46AF1EE10FAF0EE444A88BFB9
:10A42800F0EE474AFDEEE44A14EE900A14EE906A04
:10A438009842A8BF1E468842B8BF0E4604EE906AEE
:10A44800F8EEE44A062ACCED054A3DF478AAD8EDA0
:10A45800184A9DED124A65EEA44AE4EE064AB0EEAB
:10A46800674AA4EE854AF4EEC46AF1EE10FAF0EEFB
:10A47800444A88BFF0EE474AFDEEE44A14EE900ADB
:10A4880014EE906A9842A8BF1E468842B8BF0E468E
:10A4980004EE906AF8EEE44A072ACCED064A3DF449
:10A4A8004EAAD8ED1C4A9DED134A65EEA45AE6EE75
:10A4B800045AE5EE257AF4EEE76AF1EE10FAC8BF21
:10A4C800F0EE477AFEF7D9B93849394A89681268EF
:10A4D80091423FF6DBA998F800200C3A022A7DF653
:10A4E80005AF94F88C2188F80030002A3DF4FEAEC0
:10A4F800FFF702BA9FED2F7AFFF75ABB2E4B4FEAB0
:10A50800890E5FEA9A0901EB0E0C03EBC818A64402
:10A5180000F0198509F101094FEA091908EB09004A
:10A5280008F110030CF110010EF1100213ED024AAC
:10A5380013ED035A13ED016A13ED047A51ED024A43
:10A5480051ED035A51ED016A51ED047A64EE244A43
:10A5580065EE255A66EE266A67EE277A103398422A
:10A5680042ED024A42ED035A42ED016A42ED047A95
:10A5780001F1100102F11002D8D1A9F11009C84463
:10A588000CEB0901CE441AF0030A3EF4E3ADB8EC33
:10A59800017AF1EC017A67EE277ABAF1010AEEEC5A
:10A5A800017AF4D1FEF7D6BD0000024378140020EA
:10A5B80038360020000000005C3D00206034002098
:10A5C800BAF1000F00F09083DFF85C869DED0C4A2D
:10A5D800D8ED004A65EEA44AE4EE064AB0EE674AB2
:10A5E800A4EE854AF0EE444AB9F1000F06D0F4EE25
:10A5F800446AF1EE10FAC8BFF0EE474ABDEEC77ADA
:10A6080017EE101ABDEEE47A04EE901A17EE100A4F
:10A61800814200F388849842A8BF184607EE100AC2
:10A62800B8EEC77ADFF804C6012A8CED007A3DF44B
:10A638008BA998ED047A9DED0D4A25EE877AA4EE54
:10A64800067AB0EE674AA7EE054AB0EE447AB9F149
:10A65800000F00F05784F4EEC46AF1EE10FA40F3EC
:10A66800518408469842A8BF184607EE100AB8EE6B
:10A67800C77A022A8CED017A3DF466A998ED087A2A
:10A688009DED0E4A25EE877AA4EE067AB0EE674A6B
:10A69800A7EE054AB0EE447AB9F1000F00F027841E
:10A6A800F4EEC46AF1EE10FA40F3218408469842A9
:10A6B800A8BF184607EE100AB8EEC77A032A8CED31
:10A6C800027A3DF441A998ED0C7A9DED0F4A25EEEA
:10A6D800877AA4EE067AB0EE674AA7EE054AB0EE8E
:10A6E800447AB9F1000F00F0F883F4EEC46AF1EE91
:10A6F80010FA40F3F28308469842A8BF184607EEBE
:10A70800100AB8EEC77A042A8CED037A3DF41CA926
:10A7180098ED107A9DED104A25EE877AA4EE067A18
:10A72800B0EE674AA7EE054AB0EE447AB9F1000FD9
:10A7380000F0C983F4EEC46AF1EE10FA40F3C38363
:10A7480008469842A8BF184607EE100AB8EEC77A1E
:10A75800052A8CED047A3DF4F7A898ED147A9DED5E
:10A76800114A25EE877AA4EE067AB0EE674AA7EE7C
:10A77800054AB0EE447AB9F1000F00F09A83F4EE7E
:10A78800C46AF1EE10FA40F3948308469842A8BFD1
:10A79800184607EE100AB8EEC77A062A8CED057A35
:10A7A8003DF4D2A898ED187A9DED124A25EE877AE5
:10A7B800A4EE067AB0EE674AA7EE054AB0EE447AF0
:10A7C800B9F1000F00F06B83F4EEC46AF1EE10FAF1
:10A7D80040F3658308469842A8BF184607EE100A5A
:10A7E800B8EEC77A072A8CED067A3DF4ADA898ED45
:10A7F8001C7A9DED134A65EE875AE4EE065AE5EE9B
:10A80800857AB9F1000F00F04283F4EEE67AF1EEB2
:10A8180010FA40F13C830A469A42A8BF1A4604EE51
:10A82800902AF8EEE44ACCED074AFDF78DB807EE1A
:10A83800903ADFEDED6AB8EEE77A66EEA65A9FED3C
:10A84800EB5A9FEDEB6ADFEDEB7AA5EE856A26EE13
:10A85800A55AE5EE867AE5EE276A26EE870AFFF71F
:10A86800A0B9D8ED006ADDED0C4A65EEA66AE4EE03
:10A87800866AF0EE674AE6EE854AFDEEE46A16EE71
:10A8880090EA714500F341819E45A8BF9E4606EEB9
:10A8980090EAF8EEE66A002E00F07B84DFF88CC3BD
:10A8A800012ACCED006A3DF44FA8D8ED046ADDED2D
:10A8B8000D4A65EEA66AE4EE866AF0EE674AE6EEB1
:10A8C800854AFDEEE46A16EE90EA714500F3FA81D6
:10A8D8009E45A8BF9E4606EE90EAF8EEE66A002E70
:10A8E80000F04C84022ACCED016A3DF42DA8D8ED85
:10A8F800086ADDED0E4A65EEA66AE4EE866AF0EEB9
:10A90800674AE6EE854AFDEEE46A16EE90EA71457E
:10A9180000F3D5819E45A8BF9E4606EE90EAF8EE64
:10A92800E66A002E00F0FA83032ACCED026A3DF4B1
:10A938000BA8D8ED0C6ADDED0F4A65EEA66AE4EEC9
:10A94800866AF0EE674AE6EE854AFDEEE46A16EEA0
:10A9580090EA714500F3B0819E45A8BF9E4606EE79
:10A9680090EAF8EEE66A002E00F0CE83042ACCEDD9
:10A97800036A3CF4E9AFD8ED106ADDED104A65EEE4
:10A98800A66AE4EE866AF0EE674AE6EE854AFDEED0
:10A99800E46A16EE90EA714500F38B819E45A8BFE4
:10A9A8009E4606EE90EAF8EEE66A002E00F09283E4
:10A9B800052ACCED046A3CF4C7AFD8ED146ADDED86
:10A9C800114A65EEA66AE4EE866AF0EE674AE6EE9C
:10A9D800854AFDEEE46A16EE90EA714500F375814A
:10A9E8009E45A8BF9E4606EE90EAF8EEE66A002E5F
:10A9F80000F0BA83062ACCED056A3CF4A5AFD8ED81
:10AA0800186ADDED124A65EEA66AE4EE866AF0EE93
:10AA1800674AE6EE854AFDEEE46A16EE90EA71456D
:10AA280000F33F819E45A8BF9E4606EE90EAF8EEE9
:10AA3800E66A002E00F0CC83072ACCED066A3CF4C7
:10AA480083AFD8ED1C6ADDED134A65EEA65AE4EE35
:10AA5800865AE5EE257AFDEEE77A17EE902A9142BE
:10AA680003DC9A42A8BF1A46114607EE901AF8EE80
:10AA7800E77A002E7FF40FAA069B002B7FF40BAA1F
:10AA8800059B5B45B8BFF0EE477AFFF704BA77EE4F
:10AA9800C76AF0EE477AFEF765BDBCF834309FED23
:10AAA800567A07EE903AF8EEE77A544B67EE877AD3
:10AAB800C3ED007AFCF7A3BE514B1E6816F0805612
:10AAC8007FF499A8FFF792B84E4BFCF7EFBE4E4BB8
:10AAD8001B78032B00F041820023FEF77CBE9FED1C
:10AAE8004B8AFFF7ECB99FED498AFFF71CBA9FED37
:10AAF800480ADFF83C8125EE800A21F087FCD4F86B
:10AB0800A861A8F80600FBF7ACBE06EE901AC0E6EE
:10AB180093ED000A05930791069221F077FCDFF880
:10AB280014E1DFF814C1DEF8ECE0DFF80481069ADE
:10AB3800A8F800008CFB0E3C4FEAEE7ECEEBAC1E74
:10AB480007EE90EAF8EEE77A059B0799FDEEE77ABB
:10AB580017EE900AA8F80200FCF7ADBE07EE907A4F
:10AB6800F8EEE78ADFED2B7A9FED340A84F88471DA
:10AB780068EEA78A38EE800AFDEEC07A17EE903AA2
:10AB88002033402B40F2C9819FED200A1B4BFDEE7C
:10AB9800E87A83ED010A17EE903A2033402B00F251
:10ABA800BF81DFED277AF4EEE78AF1EE10FA40F381
:10ABB800FB81DFED196ADFED197A01E0F0EE478AD3
:10ABC800F4EEE78AF1EE10FA38EEE67AF6DCDFED1D
:10ABD800147AB4EEE77AF1EE10FA40F175829FED3F
:10ABE8000E6ADFED106A35E084F9223F92E741B939
:10ABF8009730083C15A82ABE6F12833A78000020C7
:10AC0800203400202C3200208A3800200000000068
:10AC18000000C84235FA8E3CDB0FC940E4CB164130
:10AC2800DB0F49C0E4CB16C1A02B00206034002004
:10AC3800083200201C010020D34D6210DB0FC93FF1
:10AC4800DB0F494092E741B99730083C15A82ABE66
:10AC5800B0EE677AB4EEE67AF1EE10FA77EE067A9D
:10AC6800F6D41FED0A7AF4EEC77AF1EE10FA40F343
:10AC78005E811FED0D7A77EE677A27EEA76A5FEDA2
:10AC88000F5A5FED0F6A1FED0F7AE6EE256A67EE41
:10AC9800865AA6EE267AE5EE877AC4ED627AFDF743
:10ACA8009ABE06EE901AC2E6C149C24A8C46FEF721
:10ACB80040BA06EE901A76E606EE901A51E606EECF
:10ACC800901A2CE606EE901A07E606EE901A8CE625
:10ACD80001F028FDB84BDFF80C831F78069BC01ADB
:10ACE800A8F80200FEF753BAFDEEC74A0DF1300E80
:10ACF8009A46DFF8F4C2DFF8F48214EE901A0EEBED
:10AD080082024B4606E07245E8EC014A0CF1100C51
:10AD18003CF41AAEDCED004ABEEC014A65EEA44AEA
:10AD2800E6EE044AB0EE674AA5EE244AF0EE444A3D
:10AD380033B1F4EE446AF1EE10FAC8BFF0EE474AB8
:10AD4800FDEEE44A14EE909A494504EE901A04DCAC
:10AD5800D145A8BFD14604EE909AF8EEE44A002EF9
:10AD6800D1D106980028CED105985845B8BFF0EE45
:10AD7800474AC8E701F0D6FC069BDFF86882D4F89A
:10AD8800AC91D4F8A861C01AA8F80200FEF761BA1D
:10AD98008A4A126802F59C520832C4F8902198F841
:10ADA8000020012A7DF4A2AA94F88C21002A7DF4BF
:10ADB8009DAA032B00F0A18120F0A2FF012384F8B3
:10ADC8008C31FDF793BA01F0ADFC7B4BDFF81482B0
:10ADD8001F78069B99F80020D4F8A861C01AA8F833
:10ADE8000400FEF794BBDFED767AF4EEE76AF1EE45
:10ADF80010FA40F3DC81DFED735A9FED736A01E0CE
:10AE0800F0EE676AF4EEC66AF1EE10FA76EEE57ACD
:10AE1800F6DCDFED6E6AF4EEE67AF1EE10FA40F158
:10AE2800C381DFED685A9FED6A6A01E0F0EE667A49
:10AE3800F4EEC67AF1EE10FA77EEA56AF6D4DFEDF5
:10AE4800657AF4EEE76AF1EE10FA04DDDFED5C7A7C
:10AE580077EEE66AF1E4DFED607AF4EEE76AF1EEA8
:10AE680010FA44BFDFED597A77EEE66AE5E409980F
:10AE78000EF0DEFDFEF783BD4E4800F1800CFEF7B4
:10AE88002DBBA8F80600A5F8B460FCF7E3BBFDEEFF
:10AE9800E77A17EE902A8A42FFF6C3ACBCE4BDEE0F
:10AEA800C77A17EE100A8842BFF695AC07EE101A5B
:10AEB80096E4BDEEC77A17EE100A8842BFF666AC74
:10AEC80007EE101A67E4BDEEC77A17EE100A88423B
:10AED800BFF637AC07EE101A38E4BDEEC77A17EEA6
:10AEE800100A8842BFF608AC07EE101A09E4BDEE56
:10AEF800C77A17EE100A8842BFF6D9AB07EE101AC8
:10AF0800FFF7DABBBDEEC77A17EE100A8842BFF624
:10AF1800A9AB07EE101AFFF7AABBF6F7FBFE35E65A
:10AF2800DFED2E7AB9E607EE101AFFF779BB9FED31
:10AF38002A7AF4EEC77AF1EE10FA44BF9FED237A2D
:10AF480077EE677A99E66146FFF71DBBF6F7EEFFE5
:10AF580000283EF4DFACFEF7D7BC16F0E3FCFCF7A4
:10AF680071BB80201AF0F0FF08B106F01BFF20F03B
:10AF7800C7FEFEF70DBD94F8E031002B7BF4DAAE86
:10AF8800FBF7C5BEDFF86890D9F8000006F0DEFED2
:10AF9800134B1B780022022BC9F800207EF4D7AC93
:10AFA80006F036F9FEF7D3BCB0EE687A0FE600BFBC
:10AFB800DC3E00206819002004320020F0580020F0
:10AFC800DB0F4940DB0FC940E4CB1641DB0F49C01A
:10AFD800E4CB16C1DB0FC93FDB0FC9BF000000007F
:10AFE8003036002008320020A02B002060340020DA
:10AFF800E46700207B4A7C4B10681B689847089BD5
:10B008009BED007AD3ED007A784BD7ED006A83ED9B
:10B01800020A774B67EE277A2B4427EE8C7AD3ED1A
:10B02800007A744B67EE277AF0EE665AE7EE8D5A8F
:10B0380093ED006AB1EE467AB4EEE57AF1EE10FAD5
:10B0480008DCF4EEC65AF1EE10FA8CBFB0EE467A80
:10B05800B0EE657A684B1B78012B02D0192B7BF474
:10B06800E0ADDFED667AB4EEE7DAF1EE10FACCBFC8
:10B0780001230023FBF7E0BDDFED617AF4EEE7DAA8
:10B08800F1EE10FA23DCDFED5F7AF4EEE7DAF1EEA9
:10B0980010FA1CD45C4BD3ED007AB1EE677AB4EEAB
:10B0A800C7DAF1EE10FA1FD4B4EEE7DAF1EE10FACF
:10B0B80088BFB0EE67DA554BC7ED00BA1B689342FC
:10B0C800BBF670ADFCF78DBEF0EE477AC9E59FED93
:10B0D80050DAF0E7069800287FF46AAC05985845DE
:10B0E800B8BFF0EE476A63E4B0EE47DAE3E7CB5C5B
:10B0F800002B7EF40FACFEF7F8BC80201AF024FF7A
:10B1080000287DF4F3A857E6069800287FF42EACB3
:10B1180005985845B8BFF0EE476A27E40698002816
:10B128007FF402AC05985845B8BFF0EE476AFFF7C0
:10B13800FBBB132B05D1B0EE480A21F067F9AAF83A
:10B148000000B0EE480AD5F8143232489847324B1E
:10B158001B78132BB0EE408A7BF4C4AB21F056F970
:10B16800AAF80200FBF7BEBB069800287FF442ACA1
:10B1780005985845B8BFF0EE476A3BE406980028A2
:10B188007FF4B0AB05985845B8BFF0EE476AFFF7B3
:10B19800A9BB069800287FF481AB05985845B8BF2D
:10B1A800F0EE476AFFF77ABBF0EE676A47E6F0EE23
:10B1B800667A2EE645201FF099FEFF201FF096FEC6
:10B1C80016481FF007FE48461FF090FEFEF78EBB9C
:10B1D800069800287FF430AC05985845B8BFF0EEC3
:10B1E800476A29E4682800207C2800202C340020A5
:10B1F800082B0020702B00205026002000009642CB
:10B2080000C0F84400C0F8C46C2B0020502B00206C
:10B2180000000000C84C0020043200204414030839
:10B228000B4B002210B4027203F1B404012102E0B6
:10B23800072A09DC9979890702D5197981540132DD
:10B248009C4203F11403F3D15DF8044B704700BF2F
:10B258002C0D03081F230370704700BF012222230F
:10B2680002704370704700BF2C22022302704370A3
:10B27800704700BF436A8269D154436A0169426BCF
:10B2880001338B4228BF00234362002A2FD0EFF3FB
:10B298001181502383F31288436B1A68D2072CD488
:10B2A80070B45E686EB9456A826A954217D084693F
:10B2B8001444DC600ED9AA1A5A608562002280F80C
:10B2C80050201A6842F00102C9B21A6081F311884D
:10B2D80070BC70470469A21A5A608662EEE70123BF
:10B2E80080F85030C9B281F3118870BC7047C26CC5
:10B2F800136843F0800313607047C9B281F3118863
:10B30800704700BF026B10B462B1036CC268446935
:10B31800D11A013B615C5DF8044B08BF1346036416
:10B32800C8B27047016A4369C4685B5C0131A142D5
:10B3380028BF114601625DF8044BD8B2704700BFC0
:10B34800436B13B190F850007047836A406A181A2B
:10B35800B0FA80F040097047416A836A99420AD37B
:10B36800CB1A416B026961B14968501E0B44834294
:10B378000AD2C01A704702691144CB1A416B0029DE
:10B38800F2D1501EC01A704700207047036B43B1BA
:10B39800026C5B6893422FBF981AC0689B1AC0184A
:10B3A8007047C269036A9A422FBFD01AC0688018D2
:10B3B800C01A70470A4B30B503F1140493F9002002
:10B3C8005D78072AC8BF143A811804330D7313F83F
:10B3D800025C855413F8012C0A76A342EED130BDE5
:10B3E80040EF020803682DE9F041DF691FB13B46D1
:10B3F800BDE8F0411847002A164611DD04460D46FF
:10B408000E4400E023689B68204698470028F9D03E
:10B41800236815F8011B1B6820469847AE42F1D1F6
:10B42800BDE8F08100232322027043708370C3704B
:10B43800704700BF2DE9F0470569C3681D4028D053
:10B448000F4606464FF000484FF00009B5FA85F35D
:10B4580028FA03F2D2431B3B32611540042B16D85D
:10B46800DFE803F03129211903007B6A002B32D071
:10B4780003F1FF3A1FFA8AFAC7F824903C6A34B1FC
:10B4880023682046514698476468002CF8D1002D5F
:10B49800DCD1BDE8F0873868716B036889B29847DA
:10B4A800002DD3D1F5E77868B16B036889B2984766
:10B4B800002DCBD1EDE7B868F16B036889B29847E6
:10B4C800002DC3D1E5E7F868316C036889B2984765
:10B4D800002DBBD1DDE7F36A1FFA83FACEE700BF80
:10B4E80030B50446C06C61710368A26823F001039B
:10B4F800036087B0A379009213F004023DD04FF4A3
:10B50800805213F00203019244D102934FF48063F6
:10B518000022039311F00103059237D10493082305
:10B528008D07694648BF049316F098FE6079E36C6E
:10B53800A17900F00202002A15BF4FF440324FF4FF
:10B5480080324FF40034002410F0010F586808BF0F
:10B558002246CC074CBF024320EA02025A609A688E
:10B5680009074CBF42F0080222F008029A601A68E4
:10B5780042F001021A6007B030BD13F002030192D5
:10B588000BD04FF4005513460295C1E704230493EA
:10B598000C23C5E74FF40053B7E70293B8E700BFA1
:10B5A80010B50446C06CA160036823F00103036072
:10B5B800A37986B013F00402009141D04FF4805271
:10B5C80013F00203019244D102934FF4806362792D
:10B5D8000393D1074FF000030493059345BF042359
:10B5E800049308230C236946920748BF049316F076
:10B5F80035FE6079E36CA17900F00202002A15BFDC
:10B608004FF440324FF480324FF40034002410F0ED
:10B61800010F586808BF2246CC074CBF024320EAF6
:10B6280002025A609A6809074CBF42F0080222F0E9
:10B6380008029A601A6842F001021A6006B010BD4A
:10B6480013F00203019207D04FF400511346029100
:10B65800BDE74FF40053B7E70293B8E738B50C4C91
:10B668000C4DAC4206D2616820461434F5F78CFFC5
:10B67800AC42F8D3084A094B094C14600022094926
:10B688001A705A7008480860BDE838401DF058BC68
:10B69800D04403081C490308B8650020AC650020A5
:10B6A80004410020E8660020BC650020F0B50C29A4
:10B6B8002BD8DFE801F06F2A2A2A4C2A2A2A2B2ABB
:10B6C8002A2A0700046AB2F80CE097881668674DC2
:10B6D80024F480540462036A4468C16923F4005363
:10B6E80043EA0E3321F4E641A84243EA073341EA2C
:10B6F800062100F0B58005F50065A84200F0B0808D
:10B7080092684460C16102640362F0BD046A96896C
:10B718009588D2F800E0554F24F480740462036AD7
:10B728004468C16923F4007343EA062321F07301D6
:10B73800B84243EA052341EA0E017ED04C4DA842A7
:10B748007BD092684460C161C2630362F0BD046A41
:10B7580096899588D2F800E0444F24F010040462DA
:10B76800036A4468816923F0200321F0807143EA69
:10B77800061321F4E641B84243EA051341EA0E21D3
:10B7880048D03B4DA84245D09268446081618263AD
:10B798000362F0BD046A9389B2F804E01768334E77
:10B7A80024F001040462056A4468816943EA0E03CF
:10B7B80021F4803125F002059BB221F07301B042DB
:10B7C80043EA050341EA070114D0294DA84211D0E4
:10B7D80005F54065A8420DD005F58065A84209D059
:10B7E80005F58065A84205D092684460816142638E
:10B7F8000362F0BDD689158A578A23F008033343BC
:10B808003D43D68824F4407423F00403ADB2334397
:10B818002C43E9E7D589178AD68823F0800343EAC1
:10B82800051324F44064558A23F0400344EA87044E
:10B8380043EA061344EA8504A6E7D589178AD68819
:10B8480023F4006343EA052324F44054558A23F47F
:10B85800806344EA071443EA062344EA051470E7C0
:10B86800158A24F4804444EA851449E7002C0140F1
:10B87800003401402DE9F04FF022002183B07848D0
:10B88800784CDFF80492784D784E794FDFF8FC81D8
:10B8980022F0C7FE77487849DFF8F4E1DFF8F4C111
:10B8A80000221359834200F0C180B3F1804F00F0A9
:10B8B800C980AB4200F0C880B34200F0C780BB42E9
:10B8C80000F0C680734500F0C580634500F0C48071
:10B8D800434500F0C380DFF8C0A153457ED00AF588
:10B8E800806A534508BF092379D01432C82AD8D1B1
:10B8F8005C4C624D624E604F04F1C80802E014349B
:10B90800A04568D0A379002BF9D023794FEA131901
:10B9180009F1FF39B9F1050F03F00F03EFD835F836
:10B92800190040FA03F2D207E9D54FF0010A0AFAE2
:10B9380003F3013B184020F06DF916F8093051491E
:10B94800184411EBC002DAD051F83000DFF84CE1AE
:10B95800217A00F138439B0A1EF8033003F01F0ECA
:10B968005B09022B0AFA0EFA62D0032B65D0012B71
:10B9780003D17B694AEA03037B6193880093B3FA96
:10B9880083F3C3F11F039BB2DA0800EB820203F0D2
:10B998000703D2F820E09B004FF00F0C0CFA03FCD1
:10B9A8002EEA0C0EC2F820E0D2F820E001FA03F3E8
:10B9B80043EA0E03136269460023022214348DF809
:10B9C80004208DF805308DF806308DF807300DF01D
:10B9D80011FBA04596D103B0BDE8F08F082309EB11
:10B9E800C3034FF0010B93F818A00AF01F034FEAA6
:10B9F8005A1ABAF1020F0BFA03F30BD0BAF1030F7C
:10BA08000ED0DA457FF471AFD1F814A043EA0A03E7
:10BA18004B616AE7D1F818A043EA0A038B6164E72F
:10BA2800D1F81CA043EA0A03CB615EE70023D6E7FE
:10BA3800BB694AEA0303BB619FE7FB694AEA030360
:10BA4800FB619AE70123CAE70223C8E70323C6E795
:10BA58000423C4E70523C2E70623C0E70723BEE79C
:10BA6800D85D00202C0D03080004004000080040A9
:10BA780000100040002C0140001002401012030882
:10BA88001C120308D05F002040EF0208004001406C
:10BA9800001400400034014000440140240D030814
:10BAA80003682DE9F04F03F13845644EAD0A0124CF
:10BAB800755D05F01F066D09022D04FA06F400F005
:10BAC800A280032D00F0A480012D52D08088B0FA06
:10BAD80080F4C4F11F04A4B2E50803EB850504F063
:10BAE80007042E6AA4000F27A74026EA07062E623D
:10BAF8002E6A01F0030702FA04F47A1E3443012A7D
:10BB0800C1F3810CC1F300182C62C1F3411135D97E
:10BB1800C60700F19780850700F1A380440700F16C
:10BB2800B180020700F1BF80C60600F1CD8085060E
:10BB380000F1DB80440600F1E980020600F1F7809D
:10BB4800C60500F10581850500F11381440500F162
:10BB58002181020500F12F81C60400F13D81850491
:10BB680000F14B81440400F15981020455D4BDE829
:10BB7800F08F334D6E6934436C61A7E70024224689
:10BB88004FF0010E4FF0030904E00132102A04F1CE
:10BB98000204ECD00EFA02F636EA0005F5D1D3F825
:10BBA80008A009FA04F5ED430AEA050AC3F808A053
:10BBB800D3F808B00CFA04FA4AEA0B0AC3F808A04A
:10BBC800B3F804A01FFA8AFA2AEA06069E80B3F898
:10BBD80004A008FA02F646EA0A06B6B29E801E6873
:10BBE8002E401E60D3F800A007FA04F646EA0A06BB
:10BBF8001E60D3F80CA001FA04F605EA0A0A46EA20
:10BC08000A05DD60C1E70E4DAE693443AC615DE7FE
:10BC18000B4DEE693443EC6158E71A6822F0404254
:10BC28001A601A6842EA87771F60DA6822F0404291
:10BC380042EA8171D960BDE8F08F00BF240D030886
:10BC4800001002401A6822F003021A601A683A4388
:10BC58001A60DA6822F003020A438507DA607FF582
:10BC68005DAF1A6822F00C021A601A6842EA87026D
:10BC78001A60DA6822F00C0242EA81024407DA60AC
:10BC88007FF54FAF1A6822F030021A601A6842EA4C
:10BC980007121A60DA6822F0300242EA0112DA600A
:10BCA80002077FF541AF1A6822F0C0021A601A68CD
:10BCB80042EA87121A60DA6822F0C00242EA811268
:10BCC800C606DA607FF533AF1A6822F440721A604C
:10BCD8001A6842EA07221A60DA6822F4407242EAD5
:10BCE80001228506DA607FF525AF1A6822F44062E2
:10BCF8001A601A6842EA87221A60DA6822F44062F7
:10BD080042EA81224406DA607FF517AF1A6822F406
:10BD180040521A601A6842EA07321A60DA6822F456
:10BD2800405242EA0132DA6002067FF509AF1A682A
:10BD380022F440421A601A6842EA87321A60DA68C6
:10BD480022F4404242EA8132C605DA607FF5FBAE52
:10BD58001A6822F440321A601A6842EA07421A60E6
:10BD6800DA6822F4403242EA01428505DA607FF55A
:10BD7800EDAE1A6822F440221A601A6842EA874235
:10BD88001A60DA6822F4402242EA81424405DA6005
:10BD98007FF5DFAE1A6822F440121A601A6842EA88
:10BDA80007521A60DA6822F4401242EA0152DA6055
:10BDB80002057FF5D1AE1A6822F440021A601A68AB
:10BDC80042EA87521A60DA6822F4400242EA815253
:10BDD800C604DA607FF5C3AE1A6822F040721A60B2
:10BDE8001A6842EA07621A60DA6822F0407242EA88
:10BDF80001628504DA607FF5B5AE1A6822F0406208
:10BE08001A601A6842EA87621A60DA6822F04062A9
:10BE180042EA81624404DA607FF5A7AE1A6822F02C
:10BE280040521A601A6842EA07721A60DA6822F009
:10BE3800405242EA0172DA6097E600BF10B5040981
:10BE4800013C052C17D80D4B33F8142000F00F00D7
:10BE580042FA00F313F001030DD0012303FA00F0B6
:10BE6800013810401FF0D6FE054A064B125D1044FB
:10BE780003EBC00010BD002010BD00BF1012030866
:10BE88001C120308D05F002001490248FFF7D2BA0C
:10BE9800A05E00200048014001490248FFF7CABAE5
:10BEA800505E00200040014001490248FFF7C2BA35
:10BEB800285E00200004004002494FF08040FFF750
:10BEC800B9BA00BF005E002010B5064C06482146EE
:10BED800FFF7B0FA04F1A0010448BDE81040FFF7ED
:10BEE800A9BA00BFD85D0020002C014000440140E1
:10BEF80001490248FFF79EBAD85D0020002C014096
:10BF08002DE9F04104684E4DA30AAB427AD00AD914
:10BF18004C4DAB425FD00135AB4277D0023DAB42CE
:10BF28005DD0BDE8F081B3F5801F67D04A3DAB42D4
:10BF380059D14FF0700E022647794FEA970C002925
:10BF480068D0B000634685190227D4F80C809F405A
:10BF58000CEB4503BFB23C4D03F1040C47EA08075C
:10BF680045F8231045F82C20E760EFF311815022A3
:10BF780082F31288821905EBC2021369002B34D0B0
:10BF880013620433821905EBC202576917B11F60A7
:10BF980053690433821905EBC202976917B11F6010
:10BFA80093690433821905EBC202D76917B11F6080
:10BFB800D36904330027CAB21F6082F31188304462
:10BFC80005EBC000036A9BB9E3684FF6FE721340A5
:10BFD800E360BDE8F0814FF0C00E0426ACE74FF0F7
:10BFE800980E0326A8E7BDE8F08105EB0E03C9E724
:10BFF800E36843F00103E360BDE8F0814FF0480EC9
:10C00800012699E74FF0200E002695E74FF0E80E3D
:10C01800052691E7BF08022306FA03F0BB40DB437D
:10C02800E768094D9BB23B4087190CEB470CE3606E
:10C038000CF1040345F82C1045F8232095E700BFC0
:10C048004B00100051001000D85D002030B5036887
:10C058005C4D18885C4CB4FBF2F20139013AAB42F2
:10C0680094B283B089B282B266D05848834263D012
:10C07800B3F1804F60D0A0F5983083425CD000F5D2
:10C088008060834258D0524883425BD000F580607C
:10C0980083427CD022F4407200F58C3092B2834205
:10C0A8001A80D9621C850ED0484A93420BD002F5FB
:10C0B8004062934207D002F58062934203D002F5B2
:10C0C8008062934201D100221A8601225A611A889D
:10C0D8003C4992B242F001028B421A8061D0B3F11E
:10C0E800804F60D03B4A93425FD002F58062934212
:10C0F8005DD002F5006293425BD002F58062934204
:10C1080059D002F59032934257D002F540629342DB
:10C1180055D002F5806293421ED002F580629342A8
:10C1280008BF092219D002A84FF0012340F8043DA6
:10C1380016F0F0F803B030BD254822F070028342B3
:10C1480092B2A3D101201A80D9621C8558611A883D
:10C1580092B202431A80C5E708221F4B03EBC203C1
:10C1680001A85C7E8DF80440012300228DF805307B
:10C178008DF807308DF8062016F0CCF81B2CD9D195
:10C18800164B019301A816F0C5F803B030BD012085
:10C198001A80D9621C8558611A8892B202431A80A3
:10C1A8009DE70022D9E70122D7E70222D5E703223B
:10C1B800D3E70422D1E70522CFE70622CDE70722FD
:10C1C800CBE700BF002C014000A24A040034014024
:10C1D800001000400004004040EF0208190100016F
:10C1E8001F4B98422CD0B0F1804F2BD0A3F594333D
:10C1F800984229D003F58063984227D003F500635D
:10C20800984225D003F58063984223D003F59033F4
:10C21800984221D003F5406398421FD003F580630C
:10C22800984207D003F58063984208BF092202D0DC
:10C238000020704708220B4B03EBC203187E70479F
:10C248000022F8E70122F6E70222F4E70322F2E7E8
:10C258000422F0E70522EEE70622ECE70722EAE7E8
:10C26800002C014040EF02082DE9F04F013085B065
:10C27800C3B203938E4D8F4F8F4C904E0A23029377
:10C28800DFF840921DF0C4FE4FF4FA7A4FF0100C1C
:10C298004FF47A70D9F80430C3F30803002B40F048
:10C2A800C880EFF31183002B40F0C3802968A2688F
:10C2B80000BF2B689942F9D1D7F800E000FB0EF3D4
:10C2C8009B1AB3FBFEF300FB01314FF0010E019105
:10C2D800D9F80430C3F30803002B40F08E80EFF345
:10C2E8001183002B40F089802B68A16800BF2A6861
:10C2F8009342F9D1D7F800B000FB0BF2521AB2FB07
:10C30800FBF200FB0323019A9B1AB3F57A7FDFD374
:10C31800BAF1010ABED1039B002B40F0C4804FF450
:10C328007A7ADFF8A09150464FF0100CD9F8043013
:10C33800C3F30803002B40F09980EFF31183002B1F
:10C3480040F094802968A26800BF2B689942F9D10F
:10C35800D7F800E000FB0EF39B1AB3FBFEF300FBDB
:10C3680001314FF0010E0191D9F80430C3F30803ED
:10C378003BBBEFF3118323BB2B68A16800BF2A687E
:10C388009342F9D1D7F800B000FB0BF2521AB2FB76
:10C39800FBF200FB0323019A9B1AB3F57A7FE3D3E0
:10C3A800BAF1010AC2D1029B013B02937FF468AF44
:10C3B8004349444B4448454A0860DA6005B0BDE843
:10C3C800F08FEFF311888CF31288A1682368DB03E0
:10C3D80044BFC6F800E0A1682B6832685FFA88F8A5
:10C3E80088F31188D7F800801A4400FB08F35B1A19
:10C3F800B3FBF8F300FB0233CDE7EFF311888CF3BE
:10C408001288A1682368DB0344BFC6F800E0A1686E
:10C418002B6832685FFA88F888F31188D7F80080AB
:10C428001A4400FB08F35B1AB3FBF8F300FB023372
:10C4380069E7EFF311828CF31288D4F808E02368D7
:10C44800D90303D501233360D4F808E02B68316899
:10C45800D2B282F311883A68194400FB02F3A3EBC5
:10C468000E03B3FBF2F300FB01312EE7EFF3118269
:10C478008CF31288D4F808E02368D90303D5012384
:10C488003360D4F808E02B683168D2B282F311889F
:10C498003A68194400FB02F3A3EB0E03B3FBF2F373
:10C4A80000FB01315DE7184619F0F2F837E700BFE5
:10C4B800F0580020F458002010E000E0EC5800206C
:10C4C800FC9F002000ED00E0EFBEADDE0400FA05A1
:10C4D8002DE9F04F013085B0C3B203930B460291AA
:10C4E8008B4C8C4E002B00F099808B4D8B4FDFF8D6
:10C4F80030921DF08DFD4FF4FA7A4FF0100C4FF486
:10C508007A70D9F80430C3F30803002B40F0DE80BA
:10C51800EFF31183002B40F0D9802968A26800BF8F
:10C528002B689942F9D1D7F800E000FB0EF39B1A6B
:10C53800B3FBFEF300FB01314FF0010E0191D9F876
:10C548000430C3F30803002B40F08780EFF3118316
:10C55800002B40F082802B68A16800BF2A689342B4
:10C56800F9D1D7F800B000FB0BF2521AB2FBFBF27C
:10C5780000FB0323019A9B1AB3F57A7FDFD3BAF144
:10C58800010ABED1039B002B40F0BD804FF47A7A9C
:10C59800DFF88C9150464FF0100CD9F80430C3F3F3
:10C5A8000803002B75D1EFF31183002B71D1296893
:10C5B800A26800BF2B689942F9D1D7F800E000FBC8
:10C5C8000EF39B1AB3FBFEF300FB01314FF0010E93
:10C5D8000191D9F80430C3F3080313BBEFF31183B7
:10C5E800FBB92B68A16800BF2A689342F9D1D7F834
:10C5F80000B000FB0BF2521AB2FBFBF200FB032364
:10C60800019A9B1AB3F57A7FE3D3BAF1010AC4D130
:10C61800029B013B0293002B7FF467AF05B0BDE896
:10C62800F08FEFF311888CF31288A1682368DB037D
:10C6380044BFC6F800E0A1682B6832685FFA88F842
:10C6480088F31188D7F800801A4400FB08F35B1AB6
:10C65800B3FBF8F300FB0233D2E7EFF311888CF356
:10C668001288A1682368DB0344BFC6F800E0A1680C
:10C678002B6832685FFA88F888F31188D7F8008049
:10C688001A4400FB08F35B1AB3FBF8F300FB023310
:10C6980070E7EFF311828CF31288D4F808E023686E
:10C6A800D90303D501233360D4F808E02B68316837
:10C6B800D2B282F311883A68194400FB02F3A3EB63
:10C6C8000E03B3FBF2F300FB01317FE7EFF31182B6
:10C6D8008CF31288D4F808E02368D90303D5012322
:10C6E8003360D4F808E02B683168D2B282F311883D
:10C6F8003A68194400FB02F3A3EB0E03B3FBF2F311
:10C7080000FB013118E7184618F0C2FF3EE700BFEA
:10C7180010E000E0EC580020F0580020F458002009
:10C7280000ED00E0204B5B68C3F3080330B4BBB9ED
:10C73800EFF31183A3B91D4B1D4C1868A16800BF06
:10C748001A689042F9D11B4B1C684FF47A7202FBAD
:10C7580004F3591AB1FBF4F130BC02FB0010704726
:10C76800EFF31182102383F3128811498C680B6848
:10C7780013F4803F104B02D0012018608C680B49DD
:10C78800D2B20D68186882F311880A4B19684FF401
:10C798007A72284402FB01F31B1B30BCB3FBF1F394
:10C7A80002FB0030704700BF00ED00E0F0580020A9
:10C7B80010E000E0F4580020EC5800202DE9F84F74
:10C7C8008046FFF7AFFF254E2549DFF8A0E0254A50
:10C7D800254D844610274FF47A740120DEF8043082
:10C7E800C3F30803D3B9EFF31183BBB90B68D2F8CD
:10C7F80008A000BFD1F800904B45F7D1D6F800B09B
:10C8080004FB0BF9A9EB0A09B9FBFBF904FB039339
:10C81800A3EB0C034345E1D3BDE8F88FEFF3118A8E
:10C8280087F31288D2F808B01368DB0344BF286086
:10C83800D2F808B00B68D5F800905FFA8AFA8AF344
:10C848001188D6F800A0994404FB0AF3A3EB0B0364
:10C85800B3FBFAF304FB0933DAE700BFF45800200E
:10C86800F058002010E000E0EC58002000ED00E057
:10C878002DE9F04FDFF830C1474A4849484E494D45
:10C888008046102718F1FF38C0F08480DCF80430A7
:10C89800C3F30803002B5CD1EFF31183002B58D1AD
:10C8A8000B68946800BF08688342F9D1D6F80090F5
:10C8B8004FF47A7000FB09FEAEEB040EBEFBF9FEE6
:10C8C80000FB03EEDCF80430C3F308034FF47A747A
:10C8D8000120FBB9EFF31183E3B90B68D2F808A084
:10C8E80000BFD1F800904B45F7D1D6F800B004FB53
:10C8F8000BF9A9EB0A09B9FBFBF904FB0393A3EBBA
:10C908000E03B3F57A7FBDD2DCF80430C3F3080315
:10C91800002BDFD0EFF3118A87F31288D2F808B022
:10C928001368DB0344BF2860D2F808B00B68D5F859
:10C9380000905FFA8AFA8AF31188D6F800A0994421
:10C9480004FB0AF3A3EB0B03B3FBFAF304FB093371
:10C95800D5E7EFF3118487F31288D2F808901368AB
:10C96800D80303D501232B60D2F808900B682868F8
:10C97800E4B284F31188D6F800A04FF47A7400EB7F
:10C98800030E04FB0AF3A3EB0903B3FBFAF304FB5E
:10C998000E3E97E7BDE8F08F10E000E0F058002069
:10C9A800F4580020EC58002000ED00E030B4EFF31C
:10C9B8001183102282F312880649074C0A68074837
:10C9C800013200250A602560DBB2026883F3118812
:10C9D80030BC7047F0580020EC58002010E000E010
:10C9E8000F4B1B88014643B90E4B0F4A1B78106842
:10C9F8000BB981F00101F4F797BB0C4B5A691AB1D6
:10CA080018B91A68106058747047094A186811886C
:10CA1800084A92FBF1F2012102605974704700BF85
:10CA2800C8580020CA580020CC580020D0580020F0
:10CA3800E858002020A107001D4B70B59C68E36CE6
:10CA4800226BDD69C2B1636B2BB12B0702D5E36C96
:10CA580008221A6270BD2A06F7D5A26A616A8A425C
:10CA68001FD0511CA069A162825C2069E66C8142DA
:10CA78003285EAD3A362E8E7A906E4D5E26A1AB1E7
:10CA8800988C80B29047DEE7E1699B8C6069DBB2E5
:10CA98004E1CE6614354E169E368994228BFE261AC
:10CAA800D1E7E26C136823F080031360CDE700BF81
:10CAB800842400201D4B70B55C68E36C226BDD6933
:10CAC800C2B1636B2BB12B0702D5E36C08221A6243
:10CAD80070BD2A06F7D5A26A616A8A421FD0511C26
:10CAE800A069A162825C2069E66C81423285EAD342
:10CAF800A362E8E7A906E4D5E26A1AB1988C80B285
:10CB08009047DEE7E1699B8C6069DBB24E1CE66109
:10CB18004354E169E368994228BFE261D1E7E26CD6
:10CB2800136823F080031360CDE700BF842400203E
:10CB38001D4B70B51C68E36C226BDD69C2B1636B79
:10CB48002BB12B0702D5E36C08221A6270BD2A06A6
:10CB5800F7D5A26A616A8A421FD0511CA069A162F6
:10CB6800825C2069E66C81423285EAD3A362E8E7F9
:10CB7800A906E4D5E26A1AB1988C80B29047DEE73C
:10CB8800E1699B8C6069DBB24E1CE6614354E16944
:10CB9800E368994228BFE261D1E7E26C136823F0A9
:10CBA80080031360CDE700BF8424002070B4EFF346
:10CBB8001186502383F31288436B1A68D20720D456
:10CBC8005D686DB9446A826A944217D081691144DC
:10CBD800D9600ED9A21A5A608462002280F85020C7
:10CBE8001A6842F00102F1B21A6081F3118870BC30
:10CBF800704701698A1A5A608562EEE7012380F856
:10CC08005030F1B281F3118870BC704703685B6AD9
:10CC180003B11847704700BF03681B6A03B1184780
:10CC2800704700BF03682DE9F041DF691FB13B463B
:10CC3800BDE8F0411847002A164611DD04460D46A6
:10CC48000E4400E023689B68204698470028F9D0E6
:10CC5800236815F8011B1B6820469847AE42F1D19E
:10CC6800BDE8F08103689B69184700BF03685B69EA
:10CC7800184700BF0368DB68184700BF03689B6854
:10CC8800184700BF03685B68184700BF03681B6844
:10CC9800184700BF10B40B4B0B4A1C780123834084
:10CCA800234052F8200031B9B3FA83F149095DF8FD
:10CCB800044BF4F739BA191C18BF01215DF8044B6D
:10CCC800F4F732BABA580020BC580020054B53F884
:10CCD800203033B11A689B88918A0B4218BF1B0415
:10CCE80093617047BC580020036803F138422DE96E
:10CCF800F04F920A584DAA5C02F01F055209012410
:10CD0800022A04FA05F400F08C80032A00F08E80D1
:10CD1800012A3CD001F003077A1E012AC1F3810CD5
:10CD2800C1F300188088C1F3411135D9C60700F155
:10CD38009780850700F1A380440700F1B1800207BE
:10CD480000F1BF80C60600F1CD80850600F1DB80CA
:10CD5800440600F1E980020600F1F780C60500F1FB
:10CD68000581850500F11381440500F12181020543
:10CD780000F12F81C60400F13D81850400F14B814B
:10CD8800440400F15981020455D4BDE8F08F334AB8
:10CD980055692C435461BDE7002422464FF0010E2B
:10CDA8004FF0030904E00132102A04F10204ECD028
:10CDB8000EFA02F636EA0005F5D1D3F808A009FA0A
:10CDC80004F5ED430AEA050AC3F808A0D3F808B049
:10CDD8000CFA04FA4AEA0B0AC3F808A0B3F804A04C
:10CDE8001FFA8AFA2AEA06069E80B3F804A008FA0F
:10CDF80002F646EA0A06B6B29E801E682E401E60FB
:10CE0800D3F800A007FA04F646EA0A061E60D3F82B
:10CE18000CA001FA04F605EA0A0A46EA0A05DD60EA
:10CE2800C1E70E4A95692C43946173E70B4AD569AB
:10CE38002C43D4616EE71A6822F040421A601A68DF
:10CE480042EA87771F60DA6822F0404242EA81713D
:10CE5800D960BDE8F08F00BF240D03080010024020
:10CE68001A6822F003021A601A683A431A60DA68EC
:10CE780022F003020A438507DA607FF55DAF1A687E
:10CE880022F00C021A601A6842EA87021A60DA680D
:10CE980022F00C0242EA81024407DA607FF54FAFC4
:10CEA8001A6822F030021A601A6842EA07121A60F9
:10CEB800DA6822F0300242EA0112DA6002077FF5EE
:10CEC80041AF1A6822F0C0021A601A6842EA871253
:10CED8001A60DA6822F0C00242EA8112C606DA60F5
:10CEE8007FF533AF1A6822F440721A601A6842EA72
:10CEF80007221A60DA6822F4407242EA01228506A3
:10CF0800DA607FF525AF1A6822F440621A601A6861
:10CF180042EA87221A60DA6822F4406242EA8122F1
:10CF28004406DA607FF517AF1A6822F440521A6097
:10CF38001A6842EA07321A60DA6822F4405242EA72
:10CF48000132DA6002067FF509AF1A6822F440421E
:10CF58001A601A6842EA87321A60DA6822F4404294
:10CF680042EA8132C605DA607FF5FBAE1A6822F420
:10CF780040321A601A6842EA07421A60DA6822F4F4
:10CF8800403242EA01428505DA607FF5EDAE1A6863
:10CF980022F440221A601A6842EA87421A60DA6864
:10CFA80022F4402242EA81424405DA607FF5DFAE8E
:10CFB8001A6822F440121A601A6842EA07521A6084
:10CFC800DA6822F4401242EA0152DA6002057FF57B
:10CFD800D1AE1A6822F440021A601A6842EA8752EF
:10CFE8001A60DA6822F4400242EA8152C604DA6022
:10CFF8007FF5C3AE1A6822F040721A601A6842EAD6
:10D0080007621A60DA6822F0407242EA0162850417
:10D01800DA607FF5B5AE1A6822F040621A601A68C5
:10D0280042EA87621A60DA6822F0406242EA816264
:10D038004404DA607FF5A7AE1A6822F040521A60FD
:10D048001A6842EA07721A60DA6822F0405242EA25
:10D058000172DA6097E600BF2DE9F04F4A484B4B62
:10D068004B4C4FF090414FF0010A4FF002094FF03E
:10D0780004084FF0080C4FF0100E2027402680259A
:10D0880030F8022B12F0010F03D01960A3F804A0A6
:10D09800083312F0020F03D01960A3F80490083384
:10D0A80012F0040F03D01960A3F80480083312F0BB
:10D0B800080F03D01960A3F804C0083312F0100F4A
:10D0C80003D01960A3F804E0083312F0200F02D04F
:10D0D80019609F80083312F0400F02D019609E80BB
:10D0E800083312F0800F02D019609D80083312F4C3
:10D0F800807F05D04FF4807B1960A3F804B0083313
:10D1080012F4007F05D04FF4007B1960A3F804B037
:10D11800083312F4806F05D04FF4806B1960A3F8C0
:10D1280004B0083312F4006F05D04FF4006B196097
:10D13800A3F804B0083312F4805F05D04FF4805B85
:10D148001960A3F804B0083312F4005F05D04FF457
:10D15800005B1960A3F804B0083312F4804F05D0BF
:10D168004FF4804B1960A3F804B00833D20B04D0F5
:10D178004FF4004219609A80083301F58061A1429A
:10D188007FF47EAFBDE8F08F10120308D05F002057
:10D19800001800482DE9F04F2DED028B984B994A65
:10D1A8001C7893B000F59C412031814606911160AE
:10D1B800002C00F07686944A1268904240F28A80E9
:10D1C800924A93491768934DDFF888B20492013C5C
:10D1D80002911C7007F48057002F40F08880029B52
:10D1E8005B7D002B40F02786049B1B681E0401F121
:10D1F800FB80894B99459BF8023000F2F484002BA0
:10D2080040F0F584854B0593049B1F6817F48059FB
:10D2180040F0B585029BB5F906605B8B9E42B4BFB2
:10D22800002601267E4B1B6813F0805369D0059AAF
:10D23800127812F001026AD002987A49408C91ED76
:10D24800037A039107EE900AF8EEE77AB4EEE77AEC
:10D25800F1EE10FA81F27C81002E60D1724C94F8C4
:10D26800A01000295BD171487149006890F82D0021
:10D2780000240C604C608C606E49002850D1087006
:10D28800002A51D0F8064FD56B4A1278D1064BD4F4
:10D29800B9F1000F48D1002B46D17A0244D4674B2C
:10D2A8001B78002B01F0DB86654B9B78002E41F044
:10D2B80091873BB1634A644B12681B689B1A002B29
:10D2C800C1F294871020584C14F048FB012384F8CD
:10D2D800A13029E04D4B4E4A1F68049307F480574C
:10D2E80002924C4DDFF86CB1002F3FF478AF00216B
:10D2F8004B48F4F7E6FD00287FF471AF0FF092FB7E
:10D308006DE77C0293D4059A127802F00102464C2C
:10D31800002184F8A01043490391002EA3D0454969
:10D3280001200870002AADD1484B1A78002A50D144
:10D338000299B5F900E0488B898BB5F90240704530
:10D34800B4BF8027002747F040037145D8BF3B464C
:10D358009B0843F08007A042B8BF3B4643F0400714
:10D36800A142C8BF3B469B08B5F90440B5F9067011
:10D3780043F0800EA042B8BF734643F0400EA1426E
:10D38800C8BF73469B0843F0800E274C8742C8BF2E
:10D39800734643F0400E94F8A2C08F42B8BF73465C
:10D3A8009C4501F0BB82A4F8A42084F8A620234958
:10D3B80084F8A2300F78002F01F01B825F2B01F058
:10D3C80087826F2B01F02081059B1B78DE0741F1D6
:10D3D800E480049B1B6803F00403002B40F06E8676
:10D3E8000DF140081A4C0022C8F8042004F1500935
:10D3F800109240F6330A192740F283362FE000BF17
:10D40800E4400020983C0020E0400020444D0020EB
:10D41800D84E00201C5D0020404B4C00A431002059
:10D42800203400202C3200207C1B0020B86500200E
:10D4380038340020481B0020283400208A1400209B
:10D448002C360020F0580020B03A00204C42002032
:10D45800543600205C66002004344C4520D0A27865
:10D46800E3789A4217FB0261F6D26278043217FB1E
:10D47800036335F912205245A8BF5246B2F5617FC1
:10D48800B8BF4FF461728A42E6DD9A42E4DC217843
:10D498002429E1D840460434F4F704FD4C45DED194
:10D4A800624A634B177898E8030083E80300002F6B
:10D4B80000F066855F4B07935D480121F4F701FD95
:10D4C800002840F00E839BF80330002B40F00983BE
:10D4D800594B0693594C23881EB226F001061FFAB1
:10D4E80086F84345A4F8008000F0DD87544E4FF0DD
:10D4F80002090E2014274FF0FF0A86F80090777073
:10D5080086F802A014F02AFA49464948B4F800807F
:10D51800F4F7D7FC002841F0A78128F002039BB25A
:10D52800434523800BD0464B1421FF2202260E20B0
:10D538001E7059709A7014F011FAB4F80080414BBB
:10D54800414A19785068099318F0030F08BF81F011
:10D558000201C1F340010892F3F7E6FD24213448A3
:10D56800F4F7AFFC30B9059A13785E0744BF23F08F
:10D5780004031370069B1B6813F00A0F1AD00621C8
:10D588002B48F4F79EFC002800F0B0872388580643
:10D5980041F1AE8007212648F4F793FC50B12B4B9C
:10D5A8002B4AB3F904302B4982FB0302DB17C3EB88
:10D5B800A2030B800C211E48F4F783FC2288002864
:10D5C80000F0F28242F480739A42238009D01C4B07
:10D5D80002201421FF2218700E2059709A7014F03E
:10D5E800BDF91D4B1B78082B00F0EA820E2B00F0CA
:10D5F800E782049B1B68590561D5184B1B79002BE2
:10D6080000F0268114210A48F4F75BFC002840F05A
:10D6180024810EF0CFF8012014F0E2F800284ED053
:10D62800DFF83C9000264FF0CC0A1EE09165002000
:10D6380020340020E8660020E065002086380020BD
:10D64800482C0020BA580020BC5800202C66002026
:10D6580067666666AC3A0020503600201C3200200F
:10D66800A4590020DEB2022E29D80AFB06F8731C42
:10D6780059F80870002FF5D1C378BA4A90F902001A
:10D6880052F8233001970322009201213A4613F001
:10D698008DFC034606EB460000EB0010069353B1E1
:10D6A800394609EB8000CC2220F0BBFF069B49F8E5
:10D6B80008300136F6B219F08DF90028D3D1059B50
:10D6C8001E7816F0010600F0DB80A74B01221A70C5
:10D6D800079BB5F906101B68A4485A89012791428F
:10D6E800077080F24782A24B4FF07E521A60A14A1F
:10D6F800029BB5F900E01F8B92F90430107892F87C
:10D7080001C0002BAEEB070314BF01224FF0FF321C
:10D71800002BB8BF5B42B3F5FA7FA8BF4FF4FA738A
:10D72800984280F224821B1A07EE903AF8EEE77AC4
:10D73800039BBE45C3ED007A03DAF1EE677AC3EDC9
:10D74800007AB5F902E0AEEB0703002BB8BF5B42E5
:10D75800B3F5FA7FA8BF4FF4FA73984280F20482B7
:10D768001B1A07EE903AF8EEE77A039B7745C3ED6C
:10D77800017A03DDF1EE677AC3ED017AB5F90400A9
:10D78800C31B002BB8BF5B42B3F5FA7FA8BF4FF4A9
:10D79800FA736345CCBFA3EB0C03002302FB03F32E
:10D7A80007EE903A039A049BF8EEE77AB842C2ED86
:10D7B800027ABCBFF1EE677AC2ED027A1A6812F4F7
:10D7C800805200F0AE81B1F5FA6F6B4BA8BF4FF4F1
:10D7D800FA61B1F57A7F1878B8BF4FF47A71A1F57C
:10D7E8007A71002840F0B681644D654885FB013E9A
:10D7F800CB17C3EB6E1303F1010E6FF0630C30F916
:10D808001EE030F913000CFB0313AEEB000103FB21
:10D8180001F385FB0315DB17C3EB651303441BB248
:10D8280007EE903A039BB8EEE78A83ED038A002A55
:10D8380040F0798323885B0600F1B880002E40F021
:10D8480043811CF0C4FA13B0BDEC028BBDE8F08F25
:10D85800059B1B78DA077FF5DCAE3C2018F074FBDB
:10D8680000283FF42CAF04F09DFA3C2016F0EAFBA8
:10D878000028F8D1059B1E7816F001067FF425AF25
:10D88800394B1B780693002B7FF422AFDFF814A1E5
:10D89800DFF814911AF8030C99F800805146AAF1A0
:10D8A80003071CF011F8002800F01485069BB8F156
:10D8B800000F53D107F1080178791CF005F800280A
:10D8C80041F033832F49B87A1BF0FEFF002800F09F
:10D8D8001585B8F1020F41F02B832B49F87B1BF01B
:10D8E800F3FF002841F027832849387D1BF0ECFF1F
:10D8F800002800F01585B8F1040F41F01F83244972
:10D90800787E1BF0E1FF002841F01B832149B87F96
:10D918001BF0DAFF002800F01585B8F1060F41F07A
:10D9280013831D4997F823001BF0CEFF002841F010
:10D938008E801A4997F828001BF0C6FF002800F0CF
:10D948001585B8F1080F41F09380154997F82D0017
:10D958001BF0BAFF00283FF4BBAE09231A4601F0BA
:10D9680078B800BF1C060308A5310020801A0020E3
:10D97800241B002008360020F41C00201F85EB51D2
:10D98800EC660020D42A0020D92A0020DE2A0020B4
:10D99800E32A0020E82A0020ED2A0020F22A0020AD
:10D9A800F72A0020CA2A002080000020CB4BCC4A4E
:10D9B800B3F90430CB49DFEDCC6A09889FEDCB7A07
:10D9C80082FB0302DB17C3EBA2035B1A1BB207EE51
:10D9D800903AF8EEE77A67EEA67A77EE876ABDEEB8
:10D9E800E66A16EE103A2033402B40F28D86DFEDC2
:10D9F800C06ABDEEE77A17EE103A2033402B00F2EA
:10DA08007F869FEDBC7AF4EEC77AF1EE10FA41F307
:10DA18001A82DFEDB95A9FEDB96A01E0F0EE477A54
:10DA2800F4EEC67AF1EE10FA37EEE57AF6DCDFEDC1
:10DA3800B47AB4EEE77AF1EE10FA41F10882DFED3C
:10DA4800AE5A9FEDB06A01E0B0EE677AB4EEC67ADE
:10DA5800F1EE10FA77EE257AF6D49FEDA47AF4EE7B
:10DA6800C77AF1EE10FA00F38B859FEDA77AF4EEF2
:10DA7800C77AF1EE10FA44BF9FEDA17A77EE677A84
:10DA880067EEA75A9FEDA15A9FEDA16A9FEDA17A73
:10DA9800A5EE856A27EEA55AA5EE867AE5EE077A01
:10DAA800039A92ED016AD2ED005A27EEC67A65EE26
:10DAB800A77AA5EEA67AE6EE267A82ED007AC2ED7E
:10DAC800017A002E3FF4BDAE099B1978089B01F03E
:10DAD80001011868F3F728FB13B0BDEC028BBDE811
:10DAE800F08F8D4B06931B689F077FF5F3AC8B4C2B
:10DAF800B4F8008018F0010F7FF40FAD48F001036F
:10DB0800984523803FF409AD854B022214211A70F1
:10DB18000E20FF2259709A7013F020FFB4F800808D
:10DB2800FBE4029B588B8142C0F2D283B1F5FA6FB5
:10DB3800D4BFC0EB0101C0F5FA614FF47A7303FB5F
:10DB480001F1784B1D78C0F5FA60B1FBF0F1002DBA
:10DB58003FF44AAE5B78744801FB03F380FB030192
:10DB6800DB17C3EB61113FE6DFED617AFDE5DFED21
:10DB7800607ADDE5B1F5FA6F80F2A483187A8B1A22
:10DB880003FB00F3C2F5FA6293FBF2F3C3F16403FB
:10DB980007EE903AF8EEE77A9FED647A644B67EE09
:10DBA800877AC3ED007AA2E522F480739BB29A4289
:10DBB80023807FF40CAD5F4B1B78082B7FF416ADE8
:10DBC800228822F040039BB29A4223803FF411AD91
:10DBD800534B02201421FF2218700E2059709A709E
:10DBE80013F0BCFE05E513B901238BF80230524B44
:10DBF80005931B201F789BF821601BF08FFE012ED8
:10DC080007F00109824600F05F8607F002030393DC
:10DC18009BF82030DFF82C81484C052B00F2A280BD
:10DC2800DFE813F0920050000600E3000701C5008A
:10DC3800012E04BF05238BF82030B9F1000F00F046
:10DC48001B81029B3E4FB3F91810B8F80030002230
:10DC580061F30F0263F31F42002361F30F0361F3C3
:10DC68001F436A603968DBF814202B608A42C0F0D1
:10DC78005684012E41F0D28203229BF82030039271
:10DC8800CBE71BF077FE012808D12D4FB8F80230FA
:10DC98003A68642101FB0323CBF81030BAF1000F76
:10DCA80004D098F80630002B40F09680012E59D009
:10DCB800234FDBF810203B689A42C0F0808601238E
:10DCC8008BF82030012E72D098F80730012B00F025
:10DCD800DD8008F0F7FB9BF820309EE72C660020DB
:10DCE80067666666AC3A002035FA8E3CDB0FC93FA2
:10DCF80000000000DB0F4940DB0FC940E4CB1641B0
:10DD0800DB0F49C0E4CB16C1DB0FC9BF92E741B9AD
:10DD18009730083C15A82ABEE06500208638002008
:10DD2800482C0020F41C00201F85EB510AD7233C07
:10DD3800241B002050360020A431002080660020DB
:10DD4800F0580020402C0020B9F1000F99D14FF471
:10DD58008060BAF1000F00F0C68313F00FFF0023B4
:10DD6800CBF81030039B002B3FF44EAA039813F016
:10DD7800F5FD049B1F6817F480593FF44BAA1D2139
:10DD8800BB48F4F79EF800287FF444AAB94A029BDE
:10DD9800D2881B8BB5F90660991A8E4240F3048627
:10DDA80013449E42B4BF00260126FFF73BBAB24F88
:10DDB8003A68B8F80230642101FB03234FF480600D
:10DDC8000022CBF810308BF820208BF8032013F0BA
:10DDD800BDFE9BF8203020E708F074FB03224FF4C7
:10DDE8007A738BF82020CBF81C30A34F238843F09C
:10DDF800020323800EF016FE3A68DBF81C30134449
:10DE08000422CBF818308BF82020012E40F0CF8563
:10DE18003B68DBF818209A42A4D2984B187818B9B6
:10DE28001BF07CFD00289DD1238823F0020323806A
:10DE3800BEE7914FE9E7029A013BD27D35F91330ED
:10DE4800002A40F06783A3F57A73B3F57A7FA8BFF9
:10DE58004FF47A7323EAE37307EE903A9FED887ADA
:10DE6800F8EEE77A67EE877A864AFCEEE77A17EEED
:10DE7800903A1380FFF7BDB97F4F3B6847F23052A5
:10DE88000323CBF81C208BF82030AFE708F01AFBEF
:10DE9800032240F6B8338BF82020CBF81C30764F9D
:10DEA800A4E7794F3B78002B00F0DE87774BDFF84B
:10DEB800F881DFF8F8B1DFF8F8A1029345465E462D
:10DEC800039099460EE019F804109847032C28DCB3
:10DED80088B93B782AF8020F01349C4205F1040501
:10DEE80080F21081072CE1B23046DBF80430EADD1D
:10DEF800984700B2EDE738F824206B88801A4FF471
:10DF08007A719B1A01FB00F040F6CA0290FBF3F00D
:10DF18000844904240F2EE23A8BF10469842B8BF8A
:10DF2800184600B2D5E71D215148F3F7CAFF00286B
:10DF38003FF480AC9BF80330002B7FF47BACDFED23
:10DF4800547A544938EE678AC7F5FA63FDEEC87A01
:10DF58001BB2CDED027ABDF90820120381FB020144
:10DF6800D217C2EBA11203FB02F343F30F333B4476
:10DF780007EE903A039BF8EEE77AC3ED037A59E48B
:10DF8800DFF830A1DFF83081434C0AF15A064FF030
:10DF9800010951461AF8010C1BF096FCF8B19AF8E1
:10DFA80004009AF802309AF803E000EB400104EB11
:10DFB8008101013BD1F8B42003EB4303434493426E
:10DFC8000DD094F8E02081F8B0E009FA00F022EAD8
:10DFD8000000C1F8B430C1F8B87084F8E0000AF164
:10DFE800060AB245D5D12D4B07931946224A2C4B28
:10DFF8002C4C09681B78D2F8009008910693A4F17C
:10E00800B00A002663685BB31F784FB3A268A9EB18
:10E018000202002A0ADB9AF8E0200121B14022EA34
:10E02800010209F5FA718AF8E020A160069ABAB1EE
:10E03800227859780432D2B2002940F08F820299AE
:10E0480035F91220098B01F1C800824240F37E8421
:10E058009AF8E0109A7841FA06F3D90740F1F28469
:10E068000136042E04F10C04CCD1FFF725BA00BF09
:10E0780020340020282C0020F05800208A1400208A
:10E08800AAF1823F8438002000450020D84E0020A5
:10E0980000007A44D34D62107C1B0020E866002003
:10E0A800553800202C1C002018450020346600201C
:10E0B8007A1B0020E1290020A4EF0208B24C94F852
:10E0C800AA3053B1059B1B78D80706D5029BB5F932
:10E0D80006205B8B9A4200F38A841121AB48F3F740
:10E0E800F0FE002800F0228294F8AE302BB994F8A4
:10E0F800A83013B93223A4F8AC30012384F8AE3029
:10E10800FFF76EB9DDF80C90A14A04921146A14AB6
:10E11800096842F2010AA2FB092B11EA0A0A4FEA2E
:10E128009B1B00F0FF819C4D9C489D4C9D4A95F897
:10E1380000E0007884F800E01070BEF1000F04D011
:10E14800984A92F800E08EF0010E8F4C0F2084F868
:10E158002400002B00F05A83934B0B931B780A93EF
:10E168001E463B78029F914AB7F824C0DFF87082B8
:10E1780009903D46FF8C08973746A2FB0662520875
:10E188002D8B0E9502EB420294F825500C95BA1A85
:10E19800D2B201F48051079204F128060BF5967269
:10E1A8006746834DCDF80CE0A4465446DDF830A010
:10E1B8000F9100200592CDF834909E46039B002BCA
:10E1C80000F03B823CF910101FFA81F9B9454FEA7B
:10E1D800400203D3089B994540F2718258F82010F9
:10E1E8008B4580F03382A95E002C40F047820130D5
:10E1F8007045A95206F10606E0DB09986D4ADDF87C
:10E2080034908CF824000F28644651460CBF012135
:10E218000021734684F825A0117000F0FD82DFF814
:10E22800C4B1654E654F34883868DBF80810DBF8F0
:10E238000420CBF80C0044F00404401A9042574FD5
:10E248003480584C4FF0010188BF0022397021708A
:10E2580088BF8BF82120002B00F0F382049A0299E2
:10E268001768574EB1F824C0B1F818E0504817F4B1
:10E278008057344640F00A8339460EE0627802EB54
:10E28800820202EB820202F2EE2292B201318B424A
:10E2980020F8022B04F102040ED016F81120002AEF
:10E2A80000F01182022AE9D00131028820F8022BFD
:10E2B8008B4204F10204F0D10B9A137801331370E6
:10E2C800FEF78ABF1B7AC3F1640307EE903A61E454
:10E2D800114636E40AF1050178791BF0F5FA0028B1
:10E2E8003FF4F0AAB8F1010F40F01F8607F10D01C5
:10E2F800B87A1BF0E9FA002840F01A863149F87B11
:10E308001BF0E2FA00283FF4EFAAB8F1030F40F03F
:10E3180012862D49387D1BF0D7FA002840F00E866A
:10E328002A49787E1BF0D0FA00283FF4EFAAB8F10A
:10E33800050F40F006862649B87F1BF0C5FA00286D
:10E3480040F00286234997F823001BF0BDFA002805
:10E358003FF4EFAAB8F1070F40F079831E4997F808
:10E3680028001BF0B1FA002840F082831B4997F877
:10E378002D001BF0A9FA00283FF4AAA9B8F1090F4B
:10E388003FF4A6A9FFF7E9BA7C1B0020203400203F
:10E39800444D0020D34D6210743C0020C40400207A
:10E3A80055380020C5040020AD440020ABAAAAAA15
:10E3B8001C5D00209E66002080660020F05800202A
:10E3C8004C450020D92A0020DE2A0020E32A00201C
:10E3D800E82A0020ED2A0020F22A0020F72A00204F
:10E3E800B04400205C660020CD4CD4F88830A9EBFE
:10E3F8000303002BFEF6FDAECA4A94F88C30517C1C
:10E40800069AC4F888200133C74A029E32F81120C0
:10E41800B17D03F00F0384F88C30234492B292FB51
:10E42800F1F283F8902094F8901094F8912094F8E1
:10E43800923094F89C000A4494F89310134494F88A
:10E448009420194494F895300A4494F8961013448B
:10E4580094F89720194494F898300A4494F899103D
:10E46800134494F89A20194494F89B300A441344AE
:10E4780094F89D1094F89F20184494F89E30014415
:10E488000B441A4442F30B12642AF17DA8BF64229C
:10E4980013B209B1C2F1640307EE903A9FEDA37A73
:10E4A800F8EEE77ADEE40221A148F3F70AFD002836
:10E4B8003FF433A8268018F0020F7FF440A848F0F4
:10E4C8000203434523803FF43AA89A4B02221421C1
:10E4D8001A700E20FF2259709A7013F03FFAB4F8A0
:10E4E8000080FFF72CB813F031FB38E4228822F0C3
:10E4F80040039BB29A4223803FF44CA88D4B0220E4
:10E508001421FF2218700E2059709A7013F026FA01
:10E51800FFF740B8C3F53B6308331BB293E403230A
:10E528000393ABE4844A92F800E006E694F8A83036
:10E53800002B3EF455AF059B1B7813F001037EF4C6
:10E548004FAF012284F8A83084F8A920FEF748BF0D
:10E55800734C012184F8A010FEF7E1BE012900F0F8
:10E5680035849AF8E0200123B34001361343042E82
:10E578008AF8E03004F10C047FF444ADFEF79CBF48
:10E588009FED797A77EE677AFFF77ABA059B6B4A3F
:10E598001B781060DB0700F1388294F8A600002889
:10E5A8007EF417AFB4F9A430322B7EF712AF94F88B
:10E5B800A2200121572A84F8A61000F0A284049B07
:10E5C8001B6813F0040302D05A2A00F062855D2A02
:10E5D80000F0BD845B2A00F021855E2A00F02585C5
:10E5E800562A00F02D85972A00F04985A72A40F081
:10E5F800C5845349049B0A781B6842F004020A70D8
:10E6080003F00403FEF7E9BEB2F5FA7FFEF6E1AEC9
:10E6180094F8A620002A7EF4DCAE059B1B78012125
:10E62800DF0784F8A61000F1A1840DF041FD049BDA
:10E638001B6803F00403FEF7D0BE002F3DD058F846
:10E6480020108B454FEA4002FFF4CDAD3D4B995C5D
:10E6580003EB0209002900F0F980022946D199F854
:10E66800011001EB810101EB810101F2EE2189B278
:10E67800032832DD09B2002C3FF4B9AD079B26F818
:10E688001310BAF1000F03D10A9B022B7FF6AFAD2E
:10E69800B6F800A07188B6F804902B4B5144894411
:10E6A8000FFA89F983FB0931284BA1EBE97123F8AB
:10E6B800029009B24FF0010A99E539464200059BDC
:10E6C80048F8203090E5CAB2022A04D9032A7FF418
:10E6D800EBAD6246DAE57246D8E5012303FA00F9A4
:10E6E800099B23EA090309B209937DE5A95ABFE703
:10E6F80043F04002934222807FF400AFFEF74ABF06
:10E70800DFED137AFFF7CCB9F4EEC77AF1EE10FA21
:10E7180040F3AE83DFED115A9FED0E6A2EE000BF85
:10E728007C1B0020685800208458002014AE234128
:10E7380020340020482C002055380020B43A00200E
:10E74800283400204C45002056555555EC1B002018
:10E7580000000000E4CB1641DB0F49C0DB0FC940C5
:10E76800E4CB16C1DB0FC93FDB0F494092E741B943
:10E778009730083C15A82ABEF0EE476AF4EEC66A40
:10E78800F1EE10FA36EEE57AF6DC5FED0D6AB4EEDE
:10E79800E67AF1EE10FA40F198835FED105A1FED1A
:10E7A800106A01E0B0EE667AB4EEC67AF1EE10FABD
:10E7B80077EE256AF6D41FED157AF4EEC76AF1EE06
:10E7C80010FA40F39F801FED187A77EE666A66EEBE
:10E7D800A65A1FED1A5A1FED1A6A1FED1A7AA5EEEE
:10E7E800856A26EEA55AA5EE867AE5EE076AFFF752
:10E7F80000B93946C148F3F764FB00283FF4C6AEB8
:10E8080084F8A7700DF054FCFEF7DEBDBC49BD4A84
:10E818000B91BD4D012111701B21B8480393F3F7EB
:10E8280050FB039B00287FF4FAACDFF8FCB2B74F2B
:10E83800DBF80C203B68CBF808309B1AC82B00F299
:10E848001A83049B1F6807F4805735E5C1B2022973
:10E8580040F2BA8203297FF449AF0E9B19460F9BF9
:10E86800002B08BF394603E728F0010292B242455F
:10E8780022803FF420AE0E2086F80090777086F84C
:10E8880002A013F06BF8B4F8008014E600210FE042
:10E89800627802EB820202EB820202F2EE2292B26C
:10E8A8000131994220F8022B04F102043FF404AD2F
:10E8B80016F811201AB1022AEAD00288F0E7CAB283
:10E8C800032AFAD87246EBE700230393FFF7A0B9AF
:10E8D800B2F5FA7FFEF67DAD94F8A630002B7EF4F3
:10E8E80078AD059B1B78012113EA010084F8A61076
:10E8F80000F0CF820EF096F8049B1B6803F0040327
:10E90800FEF76BBD9FED827AF4EEC76AF1EE10FA5E
:10E9180044BF9FED807A77EE666A58E77E4A7F4962
:10E928001068B4F9A420C76981FB07018911FF1792
:10E93800781A00F5FF407F3082423EF738ADC91B98
:10E948000A4412B2A4F8A420FEF731BDC8398A429D
:10E9580040DA9AF8E0109A7841FA06F3DB073FF5B7
:10E968007FAB52420120099213F0D8F87B1E099A16
:10E97800162B00F2BF80DFE813F076018C015D01F1
:10E98800B501A2011F010A01F801E1010D024601CA
:10E99800BD00B50124021F010A01F801DC01920043
:10E9A8007E00F300DB00A8000126FEF73BBC3A68B6
:10E9B800DBF81C301344CBF81830FFF7D3B907F055
:10E9C80081FD032240F6B8338BF82020CBF81C30A9
:10E9D800FFF70CBA9AF8E0300122B24023EA0203AA
:10E9E80009F5FA728AF8E030A260FFF739BB002116
:10E9F8004248F3F766FA00287FF46FAB322384F8B5
:10EA0800AA00A4F8AC30FFF768BB454B1B78002B75
:10EA18003EF4DFAC9BF80330002B7EF4DAAC94F8BC
:10EA2800A7300133DBB2032B84F8A7307EF6D1ACD4
:10EA38003C4B5B7813B9002E7EF4CBAC0DF0F2FFA3
:10EA4800FEF7C2BC002A0CBF012002208BE7072377
:10EA58001A4602EB8202174489F80030B9787878B0
:10EA680009F066FA059B1E7806F00106FEF730BE2F
:10EA780008231A46EDE7DAF8E400DFF8B080817879
:10EA88001144C829A8BFC82121EAE171817098F80A
:10EA98000230002B40F0698306F050FE61E5DAF899
:10EAA800E400DFF8888041781144C829A8BFC8214C
:10EAB80021EAE171417098F80230002BECD0132064
:10EAC8001AF08AFFDAF8E400E6E7DAF8E400DFF89B
:10EAD8005C8090F8361098F8023011446429A8BF79
:10EAE800642121EAE17180F83610002BD4D0172078
:10EAF8001AF072FFDAF8E400CEE700BF20340020F5
:10EB0800AD4400209E6600201C5D0020F0580020C7
:10EB1800DB0FC9BFDB0F49C0A83A0020D34D6210F4
:10EB2800553800202C3600205C660020204200204A
:10EB3800DAF8E400DFF8988690F8371098F8023091
:10EB48001144FE29A8BFFE2121EAE17180F837109F
:10EB5800002BA1D016201AF03FFFDAF8E4009BE75B
:10EB68000898DFF86C8641781144B1F5967FA8BF04
:10EB78004FF4967121EAE171417098F80230002B48
:10EB8800B8D015201AF028FFDAF8E40084E7DAF89C
:10EB9800E400DFF83C86017998F802301144C8296E
:10EBA800A8BFC82121EAE1710171002B40F0CF8292
:10EBB800102F7FF478AF6FE7DAF8E400DFF81086FB
:10EBC800C17898F802301144C829A8BFC82121EAA1
:10EBD800E171C170002B40F011830F2F3FF45CAF3F
:10EBE80001781144C829A8BFC82121EAE171017040
:10EBF80098F80230002B3FF44FAF12201AF0ECFEC9
:10EC0800DAF8E40048E7DAF8E400DFF8C485017AC6
:10EC180098F802301144C829A8BFC82121EAE17137
:10EC28000172002B3FF438AF0B201AF0D5FEDAF84A
:10EC3800E40031E70899DFF898850F791744642FC5
:10EC4800A8BF642727EAE7770F711AF0DFFE98F864
:10EC58000230002B3FF44EAF032039461AF0BCFEB9
:10EC6800DAF8E40018E70898DFF8648501781144B9
:10EC7800FA29A8BFFA2121EAE171017098F8023057
:10EC8800002B3FF437AF01201AF0A6FEDAF8E400B3
:10EC980002E70898DFF83885817811446429A8BF0D
:10ECA800642121EAE171817098F80230002B3FF469
:10ECB80021AF02201AF090FEDAF8E400ECE608989A
:10ECC800DFF80C85C17998F80230114481F3080106
:10ECD800C171002B3FF40EAF05201AF07DFEDAF863
:10ECE800E400D9E6089BDFF8E884997998F80200EF
:10ECF80011446429A8BF642121EAE17199710028AF
:10ED080040F02D820D2F3FF4F5AE089898F80230A8
:10ED1800417911446429A8BF642121EAE171417154
:10ED2800002B3FF4E7AE0E201AF056FEDAF8E400A6
:10ED3800B2E6DAF8E400DFF8988451E7DAF8E4009C
:10ED4800DFF88C84817998F802301144C829A8BF6B
:10ED5800C82121EAE1718171002B3FF49DAE0920A1
:10ED68001AF03AFEDAF8E40096E6DAF8E400DFF89A
:10ED78006084417998F802301144C829A8BFC82195
:10ED880021EAE1714171002B40F04082112F7FF49C
:10ED980076AE81E6DAF8E400DFF83484C17998F8D1
:10EDA80002301144C829A8BFC82121EAE171C17104
:10EDB800002B3FF471AE0A201AF00EFEDAF8E400D8
:10EDC8006AE6DFF80C84A0E70E9951E435F91220C1
:10EDD8009978B2F5617F4FF4966393FBF1F33ADBD0
:10EDE80040F633019142A8BF11460C2FA1F561717D
:10EDF80091FBF3F100F0FB80182F7FF4B2ABC9B29E
:10EE0800C8290B46A8BFC823DAF8E400C27DDFB2E0
:10EE180097423FF4A6AB9A1ADFF8B483C77548BF88
:10EE28000732D71098F802300137FFB23BB9002FEC
:10EE38003FF497AB384612F071FEFFF792BB1820EB
:10EE48001AF0CAFDF3E7B0EE677AFEF7F0BDF0EE10
:10EE5800477AFEF702BE0C2F00F0E480182F7FF4EB
:10EE680080AB00210B46CFE7C54A0292FFF74CB9A9
:10EE7800B0EE667A89E4C34A049B1F68138823F0BE
:10EE880004031380012307F480578BF82130FFF720
:10EE980013BABD4B1B6813F4003340F0CA80184600
:10EEA800BA490E5C0F2E00F10C0011D00133152B5E
:10EEB800F7D1049B1B68FA3A0021A4F8A42003F0B8
:10EEC800040384F8A610FEF788BAF0EE476A72E4E5
:10EED800AF4FD7F800E05800BEF1000F07D0C618B2
:10EEE80001EB86069EF801E076787645E1D2184473
:10EEF800A84EA94B01EB80010020396030801860D2
:10EF0800D7E7A64BA6491A684FF47A73B3FBF2F316
:10EF1800C3EB431203EB8202049B1B68D200A1F8E7
:10EF2800B42003F00403FEF758BA01231A4690E50B
:10EF380002231A468DE503231A468AE504231A4656
:10EF480087E505231A4684E506231A4681E5954B8D
:10EF5800002201209449954C0B60227012F0DEFDCE
:10EF6800049B1B6803F00403FEF737BA049B90491F
:10EF78001B680A6003F00403FEF72FBA0021BB2ABE
:10EF8800109100F0B780B72A00F0B080BE2A00F0D8
:10EF9800AB80BD2A00F09180792A00F0D1807A2ACE
:10EFA80000F0C7809E2A00F0BE809D2A00F0B48041
:10EFB800AE2A00F05C81AD2A00F05281EF2A00F001
:10EFC8004981FD2A00F04081FB2A00F03781FE2AA2
:10EFD80000F02E81F72A00F025817B2A7EF4F9A91A
:10EFE8004FF4FA61022019F05BFAFEF7F2B9CFB2DA
:10EFF8006E4B09915B78BB423FF4B3AADFF8D0812E
:10F00800384619F019FB98F8023009991BB1C9B2B2
:10F018000C201AF0E1FC0137FFB208E7654B01222A
:10F02800022097E700273946E2E7634B02220320D4
:10F0380090E7624B1B78032B00F09D8003462FE777
:10F048000FF092FCF2F714FB0FF076FC01F0F4F9E4
:10F05800012012F063FD94F8A220FFF7C4BA002E35
:10F068003EF430A9564C94F8A130002B3EF45CA92C
:10F0780012F058FC002384F8A130FEF755B9049B20
:10F08800504A1B684FF4C871118003F00403FEF75F
:10F09800A4B994F8A820002A38D194F8AA3083F0AB
:10F0A800010384F8AA3043BB0C2012F057FC049BE0
:10F0B8001B6803F00403FEF790B94FF6FE73424A4B
:10F0C800D0899689014433449381D1810FF04CFC57
:10F0D800F2F7CEFA0FF030FC01F0AEF9012012F091
:10F0E8001DFDB4F8A420E4E60223E8E70B464FF63A
:10F0F800FE71E4E70B460221E1E70B2012F02EFC3B
:10F10800049B1B6803F00403FEF767B984F8A800A2
:10F1180084F8A910FEF761B90021FF201CF0CAFD90
:10F1280094F8A22044E701201CF0C4FD94F8A22022
:10F138003BE7264A137A43F001031372FEF749B9F5
:10F14800224A137A23F001031372FEF742B9102002
:10F1580009921AF041FCDAF8E400099A28E50D2032
:10F1680009921AF039FC099ACCE514201AF034FCFB
:10F17800DAF8E40090E412F0D5FBB4F9A42098E69C
:10F18800D84E002080660020D429002060F50208AF
:10F198001C1B0020701B0020741B0020344D002015
:10F1A800B04A002004410020B8650020AC6500206A
:10F1B800B43A002052410020A04100208A380020A3
:10F1C8007C1B002006670020103600208466002083
:10F1D80020420020002B3FF445AF2849284A0968FF
:10F1E8004FF47A7000FB031313603BE7254C0DF0D6
:10F1F80019FC002384F8A130FEF796B80F20099275
:10F208001AF0EAFBDAF8E400099AE6E41120099218
:10F218001AF0E2FBDAF8E400099AB7E5032303934E
:10F22800FEF7A4BD0021042019F03AF9FEF7D1B881
:10F238000021032019F034F9FEF7CBB80021022091
:10F2480019F02EF9FEF7C5B80021012019F028F9A8
:10F25800FEF7BFB80021084619F022F9FEF7B9B841
:10F26800FF2100201CF026FD94F8A220A6E601212B
:10F2780000201CF01FFD94F8A2209CE6F058002006
:10F28800B03A00207C1B002038B50B4C23688BB1AA
:10F298005A68821A002A054604DA0CE05A68AA1A43
:10F2A800002A07DB9A68226018461A689047236884
:10F2B800002BF3D138BD38BDB43C002008B506F0AA
:10F2C800F3FB024B024ADA60FEE700BF00ED00E004
:10F2D8000400FA05024A034B1278197808F048BE70
:10F2E80064190020651900202DE9F04F2DED028BDF
:10F2F800A0F10A0389B00C46E72B00F25D86DFE82F
:10F3080013F01C015B065B065B065B065B065B068F
:10F318005B065B065B065B065B065B065B065B06DD
:10F328005B065B065B065B065B065B065B065B06CD
:10F338005B0679055B065B065B0669055B065B0693
:10F348005B0654065B06C6055B06AD055B06A105B4
:10F358005B0698055B062E065B061A065B065B06CF
:10F368005B0613060B065B0641035B065B063A0366
:10F378005B0612035B065B065B06F6025B065B0632
:10F388005B065B06D7025B06FC005B063D046E016C
:10F398005B065B065B065B065B065B065B062D0190
:10F3A8005B060F045B06DB035B0662035B064E032A
:10F3B8005B065B065B065B061C05E104DA04A90430
:10F3C800E8005B065B065B0236025B06FF01E301B1
:10F3D8005B065B065B065B06D8015B065B06B7014E
:10F3E8005B065B065B06A8019101C30281025B060E
:10F3F8005B065B0672025B065B0689045B065B06BE
:10F408005B065B065B065B065B065B065B065B06EC
:10F418005B065B065B065B065B061C055B065B061C
:10F428005B065B065B065B065B065B065B065B06CC
:10F438005B065B065B065B065B065B065B065B06BC
:10F448005B065B065B065B065B065B065B065B06AC
:10F458005B065B065B065B065B065B065B065B069C
:10F468005B065B065B065B065B065B065B065B068C
:10F478005B065B065B065B065B065B065B065B067C
:10F488005B065B065B065B065B065B065B065B066C
:10F498005B065B065B065B065B065B065B065B065C
:10F4A8005B065B065B065B065B065B065B065B064C
:10F4B8005B065B065B065B065B065B065B065B063C
:10F4C8005B065B065B065B065B065B065B067E040B
:10F4D8005404AC4E337853B1AB4F002537F8021FB4
:10F4E8002046F2F70AFB33780135AB42F6DC0120FF
:10F4F80009B0BDEC028BBDE8F08FA24E3378002B2B
:10F50800F5D0A24F0025B846236817F81520591CD6
:10F5180021601A7098F8011001EB810101EB81015B
:10F5280001F2EE2189B22046F2F7E7FA3378013585
:10F53800AB4208F10208E7DCD9E7954D28461BF0F5
:10F54800BFFE0028D3DD2B460544226813F8011BB3
:10F55800501C9D4220601170F7D1C8E708F0FCFCF0
:10F56800FF28064600F01E8608A9002501F8125D4E
:10F578000DF10D008DF80D5008F0CEFC08A800F82C
:10F58800115D08F0BDFC08A800F8105D08F0ACFC9F
:10F5980008A820F8085D08F09BFC23685A1C226024
:10F5A8001E7023689DF80D20591C21601A7023686D
:10F5B8009DF80E20591C21601A7023689DF80F20B1
:10F5C800591C21601A7023689DF81020591C21606D
:10F5D8001A702046BDF81810F2F78FFA87E70B6803
:10F5E8006C4E01255A1C0A601D700B68B2785919B7
:10F5F80021601A701BF0EEFD2368674A67495F199E
:10F6080027601870B1F90010B2F90000F2F7EEFBAC
:10F6180023685A192260187031882046F2F76DFA6B
:10F62800284665E70A685E4B5E491878551C2560D0
:10F63800107022685878551C2560107022689B78D5
:10F64800501C206013702046C988F2F756FA012032
:10F658004EE7544D08462988F2F74FFA6988204644
:10F66800F2F74BFA2046A988F2F747FA01203FE75C
:10F678004D4D05F16006A9882046F2F73EFAE98863
:10F688002046F2F73AFA29892046F2F736FA236833
:10F69800AA7A591C21601A702368EA7A591C2160D9
:10F6A8001A7055F80C1B2046F2F710FAB542E2D151
:10F6B8001DE73E4952232268501C2060137011F840
:10F6C800013F002BF7D112E739480023226805686B
:10F6D80003EB4301561C6D5C2660157002682568B3
:10F6E8000A446E1C527826602A70026825680A440B
:10F6F80001339278691C0A2B21602A70E6D1F6E65C
:10F708002C4D0B682A68591C127821601A702B68D6
:10F7180022689978531C2360002311702A68216895
:10F728001A4401335279481C032B20600A70F5D122
:10F7380023682A68591C127A21601A7023682A687B
:10F74800591CD27821601A7023682A68591C1279CA
:10F7580021601A702B6820465989F2F7CEF92A6879
:10F768002368527A591C21601A702A6810E1002116
:10F778002046F2F7ABF920460021F2F7BEF9012046
:10F78800B6E600BF346600201A5D00204C45002014
:10F79800EC3500202042002080680020826800208C
:10F7A80008360020282C002054260020ECEF020800
:10F7B800B8650020E8660020AD4D08462988F2F7B4
:10F7C8009CF969882046F2F798F9B5F90430A94AF6
:10F7D800D91782FB0323C1EBA301204689B2F2F7B4
:10F7E8008CF9012084E6A44D0846298AF2F785F9A8
:10F7F800698A2046F2F781F92046A98AF2F77DF94D
:10F80800012075E6DFF8ACE20027FEB2714600235E
:10F818002268501C206016702268501C20601370EB
:10F82800226811F8010F0133551C062B2560107052
:10F83800EED10137062F0EF1060EE6D18F490023CF
:10F848002268501C206017702268501C20601370BA
:10F85800226811F8010F0133551C0B2B256010701D
:10F86800EED12368864A581C072120601970236846
:10F878000021581C20601970236892F8F020591C48
:10F88800216001201A7033E60B687E4A7E491078A1
:10F898007E4A5D1C2560187023688978581C206092
:10F8A800197023689278591C216001201A701FE68C
:10F8B8000B68774D591C2A7921601A7023686A7978
:10F8C800591C21601A7029882046F2F716F9236816
:10F8D800AA79591C21601A7069882046F2F70DF937
:10F8E8002368EA79591C216001201A7000E6F2F7B2
:10F8F8001DFB2368674D002803F101010CBF02229C
:10F90800032221601A7029882046F2F7DFF8A968D7
:10F918002046F2F7DBF8F2F7E1FA01462046F2F763
:10F92800D5F80120E4E50B685B4A5C4D11785C4A28
:10F93800581C2060197011682046F2F7C7F8236830
:10F94800584A591C127A21601A7029882046F2F701
:10F95800D4F8A9882046F2F7D0F829892046F2F78A
:10F96800CCF800212046F2F7C8F820460021F2F72B
:10F97800C4F80120BCE5084608224A49F2F78FF886
:10F988000120B5E50B68484A581C91782060197029
:10F9980023685278591C216001201A70A8E50B6869
:10F9A800394A4249D078394A5D1C25601870236865
:10F9B8004979581C206019702368D278591C216035
:10F9C80001201A7094E500212046F2F796F80021EC
:10F9D8002046F2F792F800212046F2F78EF82368C5
:10F9E800334D00265A1C22601E7023682A68591C51
:10F9F80092F82C2021601A7023682A68591C92F802
:10FA0800362021601A7023682A68591C92F837201A
:10FA180021601A7023685A1C22601E7023685A1CC1
:10FA280022601E7023685A1C22601E702B682046B4
:10FA3800598FF2F762F82B682046198FF2F75DF8B4
:10FA480023682A68591C92F82E2021601A702368AE
:10FA58005A1C22601E702B682046598EF2F74DF80A
:10FA68002B682046998EF2F748F8012040E500BF40
:10FA78002C66002067666666C86100203B38002057
:10FA8800583700209C4A00201036002020360020DD
:10FA9800402C00207814002050360020B424002088
:10FAA80028420020D84E00202C360020943A00200E
:10FAB800B865002017380020B14E0B687279B14D37
:10FAC800591C21601A702B682046198CF2F715F81A
:10FAD8002B682046D98BF2F710F871892046F2F787
:10FAE8000CF8B1892046F2F708F82B682046598CA3
:10FAF800F2F703F82B682046998CF1F7FEFFF1899D
:10FB08002046F1F7FAFF318A2046F1F7F6FF2A6816
:10FB1800236892F82620591C216001201A70E7E416
:10FB2800974EF378002B00F031830B680822591C9C
:10FB380021601A7023680122991821601A702368BD
:10FB4800914D591C2A7921601A702368AA78591C8A
:10FB580021601A7029882046F1F7CFFFE9892046ED
:10FB6800F1F7CBFF2368F279591C21601A702368DA
:10FB7800EA78591C216001201A70B9E40B68002545
:10FB88005A1C0A601D700B685A1C0A601D700B68AD
:10FB98005A1C0A60204629461D70F1F797FF204637
:10FBA8002946F1F793FF0120A2E4784B03F1700591
:10FBB80022681978501C2060117022685978501CEE
:10FBC8002060117022689978501C2060117022689A
:10FBD800D978501C2060117022681979501C206057
:10FBE800117022685979501C206011702268997927
:10FBF8000733501C9D4220601170D9D177E4644DC1
:10FC08000846E989F1F779FF2046A989F1F775FFD8
:10FC180001206DE40B685F4F591C3A7821601A7017
:10FC28003B78002B3FF463AC0025EEB2304609F078
:10FC380054FA23684278591C216030461A7009F03A
:10FC48004CFA01892046F1F758FF3B780135AB4261
:10FC5800EBDC4CE4504D514E9FED518ADFF8688142
:10FC6800DFED508A05F120070EE0FCEEE77ACDEDD6
:10FC7800017ABDF8041020460435F1F73EFFAF4283
:10FC880006F118063FF433AC717C0029F3D0464BDB
:10FC9800D5ED007A1B78012BE7D1444B1B68DB04B8
:10FCA80040F16A82F5EE407AF1EE10FA40F08E8269
:10FCB80040F2DC51DFE7084610223D49F1F7EFFE3C
:10FCC800012015E43B4B9B8AB3F5006F00F25C8280
:10FCD800B3F5806F00F27882B3F5007F34BF012757
:10FCE8000227354D05F10C0655F8041B91FBF7F179
:10FCF800204689B2F1F701FFAE42F5D12F4D304FC2
:10FD080005F10C06B5EC010AD7ED087A80EE270A52
:10FD18001CF07CFB81B22046F1F7EFFEAE42F1D138
:10FD2800284D05F10C0655F8041B204689B2F1F759
:10FD3800E4FEAE42F7D1FFF7DABB00258146DFF8D3
:10FD48008C80DFF88CB00595049506950795012100
:10FD58004FF6FF7A05E001350B2D00F04D8118F9BB
:10FD6800011F4F1C4AFA05F3F5D0DE07F3D5BBF89F
:10FD780000302B41D807EED506A8F2F793F8EAE74A
:10FD88009C4A0020B8650020C86100204827002050
:10FD980010360020B23100206034002008610020B5
:10FDA8000000404200E08244EC610020444D002005
:10FDB80050340020E46500201C660020384D0020E7
:10FDC800B04A00209C2C0020DB9B91411CF00208CB
:10FDD80086380020AA4D08462988F1F78EFEA988A2
:10FDE8002046F1F78AFE20462989F1F786FE012090
:10FDF800FFF77EBBA34D05F15006287815F068F88B
:10FE08002368027A591C21601A7023686A78591C81
:10FE180021601A702368AA78591C21601A70236817
:10FE2800EA780435591CAE4221601A70E5D1FFF713
:10FE38005EBB0B68944A591C527D216001201A70E0
:10FE4800FFF756BB914D05F1800655F8041F204673
:10FE5800F1F73CFEAE42F8D1FFF749BB8C4D05F1F6
:10FE68004006B5F880102046F1F747FE236895F85C
:10FE78008220591C21601A70236895F88320043564
:10FE8800591CAE4221601A70EBD1FFF730BB7E4D92
:10FE98000B682A7A591C21601A70A98B2046F1F741
:10FEA8002CFE298B2046F1F728FE698B2046F1F7B6
:10FEB80024FE2368EA7C591C21601A70A98C20460C
:10FEC800F1F71BFEE98C2046F1F717FE2368AA7F9D
:10FED800591C21601A70236895F82020591C21604C
:10FEE8001A70698C2046F1F708FE2368EA7A591CD3
:10FEF80021601A70E9682046F1F7E8FD23682A7C3A
:10FF0800591C21601A70236895F82120591C21601A
:10FF180001201A70FFF7ECBA0B68012299182160CA
:10FF280010461A70FFF7E4BA08460021F1F7CEFD33
:10FF38000120FFF7DDBA574D574E05F1300795F907
:10FF48000210564B93F906208A4203F1080336D073
:10FF58009E42F7D10835BD42F1D1FFF7C8BA504BE0
:10FF680003F15A0522685979501C206011702268E3
:10FF78001978501C2060117022685978501C206034
:10FF8800117022689978501C206011702268D97805
:10FF9800501C20601170226819790633501C9D424C
:10FFA80020601170DED1FFF7A2BA0B683D4A581CD9
:10FFB800117820601970EBE40020FFF799BA2368E4
:10FFC8005A1C2260197029882046F1F796FD23688B
:10FFD800EA78591C21601A7023682A79591C216013
:10FFE8001A702368AA79591C21601A7023686A79E3
:08FFF800591C21601A70ADE7ED
:020000040801F1
:10000000DFF8B4A000254FF008080135C5F1200243
:1000100008FA02F2A5F120032AFA05F6164328FA97
:1000200003F31E43252D06F001024FF000030BD011
:100030001343EAD0E8B219F075FC0028E5D0294650
:1000400006A8F1F733FFE0E7194B1A4E1B78DA07E1
:1000500048BF069B4FF0000544BF43F001030693E1
:100060002F4602E00135252D28D029463046F1F7EC
:100070002CFF0028F6D0294606A8F1F726FF002815
:1000800079D10137EEE700BFB424002054360020B8
:10009000D84E00205437002058370020CC5E002076
:1000A000B44E0020844E0020E0290020503600206D
:1000B000A43100206058002090E33FF4634B644D6E
:1000C000B3F850102046F1F71CFD624B198820460A
:1000D00089B2F1F716FD604B19684B0103F020025D
:1000E000C1F340031343C1F3800243EA4203C1F367
:1000F000C00243EA8203C1F3401243EAC20301F0A3
:10010000100119432046F1F7FCFC04A90422204603
:10011000F1F7C9FC23682978504A581C20601970EF
:1001200011886429A8BF64212046F1F7EAFCB9F1DF
:10013000960F42D000212046F1F7E3FC2168B7F189
:10014000190348BFA7F11203A3F3C4034A1C22609A
:1001500020461A460B7005A9F1F7A5FC2368404A12
:10016000581C10212060197020461188F1F7B2FC4C
:100170000120FFF7C1B9394604A8F1F797FE80E7DF
:10018000F4EEC87AF1EE10FA40DA4FF47A7176E5BF
:100190000827AAE50B68B178324A581C206019700C
:1001A00023681278591C21601A70CCE423685A1C09
:1001B000226001201E70FFF79FB923680322591C9B
:1001C00021601A7023686A78591C21601A70B5E79B
:1001D00004278AE5F4EEC87AF1EE10FA3FF56CAD2B
:1001E000F4EEE87AFDEEE77AF1EE10FA17EE901AE7
:1001F0001ED86FF4F973303903FB01F140F2E73395
:1002000091FBF3F101F2DB5189B238E5FDEEE77ABB
:1002100040F2E73217EE903A303B02FB03F388FBE3
:100220000312D917C1EB622101F2E93189B226E547
:1002300040F2F313A1F5836103FB01F140F2E733D0
:1002400091FBF3F101F2DD5189B218E51C010020A8
:10025000AC650020B8580020E0650020AE2C0020DE
:10026000806600200436002008B501210220FCF73A
:1002700015FD094B1B7803F00503052B08D0002161
:100280000120FCF70BFD00210846FCF707FDFEE707
:1002900005F0A0FCF3E700BF80240020022828BF5F
:1002A000022010B4084C094B207000EB8002C0EB18
:1002B000C20207495DF8044B013003EB4203C0B2B0
:1002C0000B6011F02FBC00BFAC6500200441002082
:1002D000B865002008B5FBF7C5F90EF049FBF1F74A
:1002E000CBF9BDE808400EF02BBB00BF08B50EF0FF
:1002F0003FFBF1F7C1F9BDE808400EF021BB00BF9C
:1003000038B5444B5A899989914224BF00225A81B9
:10031000198ADA89914224BF0022DA81DA7892B30D
:10032000072A30D03C493D4D91F857000124002167
:100330000A282C709C70D9713ED00C2866D0DFED55
:10034000387A002A31D1374C9FED370AA27800293C
:1003500018BFF0EE407A062A9EBF344901EB8201B5
:1003600091ED0F0A217959B3013A032A4DD8F7EEDE
:10037000007A87EE800A1CF04DF82388984228BF47
:100380001846208038BDD97921B198780428B8BFA3
:1003900004209870204890F857000A280CD00C28A8
:1003A000CDD1DFED237A002ACDD0072ACBD00A2881
:1003B0002CD1DFED207AC6E70A20DFED1F7AC0E7F7
:1003C0009B78164A07EE103A1178B8EEC77A27EEF6
:1003D000277A07EE901AF8EEE77A67EE877AB4EE9E
:1003E000E70AF1EE10FA10DDC0EE077AFDEEE77ACB
:1003F00017EE903A102BA8BF1023012BB8BF012392
:10040000DBB28B4238BF0B46137038BDDFED0B7A81
:1004100099E700BF9C4A0020B04A00200436002023
:100420006F120339C86100206F120338ECEF020825
:100430000AD7A3390F506E3A5304E9386F12833A42
:100440002DE9F047B14FB24E0EF092FABE421ED2E5
:10045000DFF84483DFF844934446258862197DB170
:100460004A450DD2052D0BD933886188C3F30B03A0
:10047000994200F0FA80144625886219002DEFD1C8
:10048000716830461436F1F783F8BE42E4D3A14ACE
:100490001378A3F1170102290FD99F4911F83300EE
:1004A000002840F00481D8000144497829B19B49D3
:1004B00011F83330002B00F02281994C6378022B25
:1004C00084BF002363702378022B84BF0023237032
:1004D000944B9A78042A00F0098132B91A88B2F54F
:1004E000F07F84BF4FF4F0721A808F4D8F4A2B68D3
:1004F0001A40002A00F00681D80700F1F280590462
:1005000000F1EA801A0700F1E2809B0400F1D88034
:10051000874D2B685A8C998C914224BF00225A84B3
:10052000FFF7EEFE12F06AFF10B9824810F0F0FCFF
:100530008020F1F763F84FF40070F1F75FF84FF4A3
:100540008020F1F75BF84FF40010F1F757F84FF007
:100550000070F1F753F84FF08060F1F74FF84FF06B
:100560000060F1F74BF86378022B06D8724A7349A2
:1005700003EB430302EB83030B602378022B07D8C2
:1005800003EB83016E4AC3EBC10302EB43032B6011
:1005900019F040FA002130226A481EF046F8286817
:1005A00004F058FF684B2E6803F1500102E0043359
:1005B00099427AD01A78002AF9D19C78D878844266
:1005C000F5D26249624B91F804E06248624D5C6B7F
:1005D000624B2860C827642111FB0E71DFF8C0E16F
:1005E00059605F4F30F8061C5E4DAEF800100021D8
:1005F0009960D960196159619961D96183F82010B6
:1006000083F821103A702E600CB10EF003F8564BAF
:100610009FED565A1B88564A9FED566A5579564C9F
:1006200056495748086006EE903AF8EEE66A138895
:10063000C5EE265A07EE103A53881279C4ED005AD7
:1006400007EE903AB8EEC77A4E4BF8EEE77A1D7295
:100650005A7227EE067A67EE867ABDE8F04783ED98
:10066000017AC3ED007A0EF06BB963799B077FF4D2
:1006700002AF716894F804A03046F0F789FF338820
:10068000BAEB133F04D01436BE42FFF4E5AEFEE6EB
:1006900073887068AA1FC3F30B039A4204F1060122
:1006A000A8BF1A461BF042FDEDE7012289E7D800FA
:1006B0000C186468002C7FF4F7AE17241470F3E66E
:1006C0003148F0F79BFF4020F0F798FF20E72F48D4
:1006D000F0F794FF2B6818E72D48F0F78FFF2B6891
:1006E00010E72C48F0F78AFF2B6808E79A8AB2F5E2
:1006F0007A7FBFF4FAAE4FF47A729A82F5E6182345
:100700001370DAE643F008032B60F5E61C49030892
:10071000D044030850360020F40D030888F1020885
:10072000AC650020C861002028420020096000025A
:10073000B8650020CC5E0020BC650020E866002083
:10074000044100202C1C002054360020402C0020A6
:10075000E465002016360020385800205C66002032
:100760008A140020601C0020781A0020C0C9FB48B1
:10077000641C002017B7D1387C1A0020AC29002057
:100780003661023D88290020094000020160000214
:10079000092000020860000202F0030800000408BB
:1007A0007040002008B50EF0E3F8F0F765FF0EF09A
:1007B000C7F8FFF745FE0120BDE8084011F0B2B9C7
:1007C00030B4034600F12405064C07CC0C3343F843
:1007D0000C0C43F8081C43F8042CAB42F4D130BC99
:1007E000704700BF44F00208034B33F80C2F02801F
:1007F0009B788370704700BF44F00208084B19686B
:1008000061B130B45D68074C642202FB05F2B2FBB3
:10081000F1F2228030BC002018605860704700BFA1
:10082000741C0020AE2C0020704700BF624B1B7868
:10083000002B3AD02DE9F041604B614D9B79AC68BB
:10084000A860013B82B0041B032B00F28380DFE829
:1008500003F03102292919F091F8002800F0828074
:10086000584B59491B78B5F84220D1ED037AEA6418
:10087000DB0700F1848002FB04F007EE900ADFED55
:10088000536A534BB8EEE77AD5ED127A5A60E7EE29
:10089000267A1A60BDEEE77AC5ED127A85ED117AF7
:1008A00083ED027A02B0BDE8F081494A13605360DB
:1008B00093607047474A484BD279DFF8308133F86C
:1008C0001220B8F902304548B8F9001092B207EE8C
:1008D000902A40F6E44707FB02F6C3EB1633B8EE66
:1008E000670A4FF47A7606FB03F393FBF1F3AB61EF
:1008F000EFF7AAFDD5F818E0D5ED047ADFED336AFD
:10090000B8F90220324BB8F900C0C3F804E00EFB7E
:1009100004F007EE100AB8EEC77ABCEEC06AE7EE44
:10092000267A8DED016ABDF80410C5ED047ABDEE9E
:10093000E77A07FB01F7C2EB173706FB07F683EDF3
:10094000027A96FBFCF685ED037A6E611E6002B0BA
:10095000BDE8F0811E4B00221A605A609A6002B016
:10096000BDE8F0811E4B1B68DE067FF579AF154BA5
:10097000B5F842201B78EA64D9070FD47BE7FDEE77
:10098000E77A184E17EE900AA0F57A7101FB01F391
:1009900086FB0306D817C0EB26100844B5F94010B3
:1009A000114B00FB01F083FB0013C017C0EBA31039
:1009B0000244EA645FE700BF2A3200204C66002050
:1009C000741C0020A43100202C3200202FE33E3183
:1009D000443700206858002084580020901C0020D4
:1009E000444D00201F85EB51D34D6210003600208E
:1009F000F0B5244B5B79012B83B00ED02249002344
:100A00000B804B80214B1B78022B04D1204B488854
:100A10000A8818805A8003B0F0BD1E4A1E4B927897
:100A20001E4D33F81240A4B207EE904A05F154006F
:100A3000B8EE670AEFF708FD194A1349107896785F
:100A40005378FCEEC07A00EB4010CDED017ABDF892
:100A5000042044F6FB77C3EB033300FB027200FB78
:100A60000474B2FBF3F2B4FBF3F3B2FBF6F2B3FBA4
:100A7000F6F392B29BB2A5F85020A5F852300A8046
:100A80004B80BFE74C660020143200200432002067
:100A9000083200206858002084580020741C002070
:100AA000EF400020F8B5254D25496879254C264BA7
:100AB000264E042264270A7001284FF0000184F8B2
:100AC000782084F88170A4F87A10A4F87C1084F857
:100AD0008010C4F8841031701980598020D0A97911
:100AE0001B4A00230129136084F888305360936007
:100AF00007D0022904D1174A636453609360F8BD9C
:100B0000F8BD154AE36053609360D3609FED130A0C
:100B100002F110004CF25031BDE8F840F1F778B91D
:100B2000282204F150001DF080FD4CF250319FED61
:100B30000C0A04F15400F1F76BF9D0E74C66002081
:100B40008A380020741C0020143200202A32002031
:100B500044370020B81C0020801C0020CDCCCC3EA7
:100B6000CDCCCC3D2DE9F0432F4DD5F88C3083B062
:100B70001BB195F89030022B02D003B0BDE8F08392
:100B80004FF020084046294C05F1940901265527CD
:100B900018F0C8FEA0B199F800300BB9217891B9CE
:100BA00008F101085FFA88F8B8F1230F04F1010495
:100BB00009F10109E1D0404618F0B4FE0028EAD15D
:100BC00089F80000ECE7D5F88C0050B30DF1080E61
:100BD000AA220EF8052D8DF802108DF800708DF800
:100BE00001608DF80430694655225340082213F005
:100BF000800F02F1FF324FEA430318BF83F0310345
:100C000012F0FF02DBB2F2D1714502D011F8012FD0
:100C1000EBE7AA2269468DF803308DF8042013F023
:100C2000B1F989F80060BBE7741C002054F0020899
:100C30001F4B1878002839D01E4A1389FBB11E4A71
:100C40009FED1E6AD2ED026A07EE903AF8EEE66A70
:100C5000F8EE677A07EE103A77EEE66AB8EEC77AF2
:100C600066EE866AC6EE877AFDEEE77A17EE900AA0
:100C70006428A8BF642020EAE070C0B2704710B4B6
:100C80000F4B54781B88117804FB1032091B642326
:100C900000FB01F003FB02F3B3FBF0F06428A8BFF4
:100CA00064205DF8044B20EAE070C0B2704700BFDA
:100CB0002A3200204C660020443700200000C84241
:100CC000143200202DE9F04F794D81B0FBF72EFD55
:100CD000D5F89C400022C5F89820002C00F0A58093
:100CE000237D052B074617D9216A23690B44C31AB4
:100CF0009342B8BF05F19C010ADBD5E0137D052BBB
:100D00000AD9136A12691344FB1A002B80F2CC80B3
:100D100051F8042F002AF1D14FF0010B0023B946FE
:100D20001E46C5F8983098469A46274623E07A6AC8
:100D300039693B7DA9EB0204B4FBF1F40134A4B2A0
:100D400013FB04F3013301369BB2B6B23C83FB8242
:100D5000984506D2BBF1000F01D1012C5FD998460E
:100D6000BA46D5F89830013305EB8302C5F89830C0
:100D7000D2F89C7047B3BB68C3B1FC8A002CD6D1B3
:100D8000396A4846A9EB01019847D0B195F8E83097
:100D9000002B52D13B7DC7F82490013601334FF030
:100DA0000102B6B23A83FB820124D1E73B6A3A6979
:100DB000A9EB0304B4FBF2F4A4B23C8334BBFB8A7A
:100DC000C6E73C83FB8AC3E72B686A68394901336D
:100DD00016443C4685E848004F46C1F800A0BAF1E9
:100DE000000F27D0DAF8203095F8E820AAF816404E
:100DF000FB1ACAF81C30CAF82090002A35D1DAF85C
:100E00000C30484601B0BDE8F04F18473B7D13FB5E
:100E100004F3013301369BB2B6B2FB8298E73A7D08
:100E2000062A04BF9846BA469BE72B68214A01333D
:100E30002B60146001B0BDE8F08FFBF777FC1E4B10
:100E40001E4A1F4C11681A68A0EB090002EB000E45
:100E50002268C3F800E09042A1EB5111014438BF71
:100E60001046164A2060116094E7FBF75FFCDAF841
:100E70000C3004469847FBF759FCDAF82C20DAF8D6
:100E80002830DAF83010001B9042A3EB53130344D0
:100E9000014438BF1046CAF82830CAF83010CAF8E2
:100EA0002C0001B0BDE8F08F4FF0000B36E700BF1B
:100EB000741C0020A83A0020B02C0020B42C002084
:100EC000B82C0020F0B43423184F194A03FB00F368
:100ED000D2F8EC60FC58FD18002E6B684B600C607B
:100EE0000DDDD2F89C309D421DD09C32002303E0E2
:100EF00052F8044FA54216D00133B342F8D1002274
:100F0000342303FB00700A720369CB60037D4B72CC
:100F1000836AC56A046BC2690A615B094D618C61B1
:100F2000CB61F0BC70470122EAE700BF1C01002042
:100F3000741C00202DE9F0414E4ED6F8EC40112CE7
:100F40007ADC002C40F39380D6F89C30984273D022
:100F5000012C5DD0D6F8A03098426DD0022C57D02D
:100F6000D6F8A430984267D0032C51D0D6F8A830D8
:100F7000984261D0042C4BD0D6F8AC3098425BD06C
:100F8000052C45D0D6F8B030984255D0062C3FD02D
:100F9000D6F8B43098424FD0072C39D0D6F8B830B4
:100FA000984249D0082C33D0D6F8BC30984243D070
:100FB000092C2DD0D6F8C03098423DD00A2C27D02D
:100FC000D6F8C430984237D00B2C21D0D6F8C83090
:100FD000984231D00C2C1BD0D6F8CC3098422BD074
:100FE0000D2C15D0D6F8D030984225D00E2C0FD02D
:100FF000D6F8D43098421FD00F2C09D0D6F8D8306C
:10100000984219D0112C03D1D6F8DC30984213D075
:10101000D6F89C504DB32B7D017D8B420FD3164FDC
:1010200000253A4605E052F8043F53B11B7D8B4240
:1010300007D30135AC42F6DA0020BDE8F0810E4F4F
:1010400000256B1C9B00191F621B06EB8505804663
:101050003944F818920001341DF0CDFAC5F89C808F
:10106000C6F8EC400120BDE8F081034FE9E7CFD09E
:10107000E2E700BF741C0020101D0020132830D0B0
:10108000112807D8184B342202FB003019B1C3686D
:101090000BB14FE7704770B5144DD5F8EC40002CFC
:1010A0000FDDD5F89C3098420CD005F19C063346F4
:1010B000002203E053F8041F884206D00132A24206
:1010C000F8D170BD002205F19C069000011DA21A06
:1010D000920031443044013C1DF08DFAC5F8EC40DB
:1010E00070BD034B1868D1E71C010020741C002060
:1010F000A83A002010B54FF4804082B010F074FB85
:1011000000B30022032390F90200009301924FF4F0
:10111000E1334FF480410FF04DFF0C4BC3F88C00CE
:1011200070B1012402221120214683F8944083F8F3
:10113000954083F8964083F89020FFF79FFF204664
:1011400002B010BD014BD3F88C00E9E7741C0020FD
:10115000F0B50D4685B006460068FBF761FD95E8E1
:101160001800E41A0023039324238DF808304D233C
:101170008DF80930B5F90A30FF2C2246A8BFFF22AE
:1011800001333DD02B7B002B0CBF3E233C238DF83D
:101190000A30FE2C2B898DF80B208DF80C3031DDB8
:1011A00023128DF80D408DF80E3007273A4602A91C
:1011B0003068FBF73BFD02ABDA190DF10B010023A0
:1011C0008A4221D1002C8DF807300CDD2246296897
:1011D0003068FBF72BFD2B689DF807201919994201
:1011E00016D18DF8072001220DF107013068FBF7B9
:1011F0001DFD3068FBF70EFD04F1090005B0F0BDE0
:101200002123C4E70527D1E711F8010B4340D7E7B5
:1012100013F8010B4240E2E72DE9F347012010F0FB
:10122000E3FA174EDFF85CA00024CC2708B1022CAB
:1012300002D902B0BDE8F08707FB04F856F8085061
:1012400015B10134E4B2F1E7C37890F902005AF81D
:10125000233001950322009201212A460FF0AAFEB5
:10126000814648B104FB0760CC2229461DF0DDF918
:10127000013446F80890E4B215F0B0FBD6E700BFA1
:10128000A45900201C0603082DE9F04F2DED088B12
:10129000C04CC14BC4F8043887B00023C4F80838E8
:1012A000F1F794F8FBF7DCFEF0F7B0F908B9FFF7B7
:1012B00011F8FFF7C5F80522B849B9481DF000FA42
:1012C00008B1FFF707F894F80C38B64D43F0010366
:1012D00084F80C38B44B9A78B44B1A70B44B1B6832
:1012E0002B6012F09DFC01210220FBF7D7FCF0F7E8
:1012F00003F82B681F070BD5AE4B1A7A0A2A07D8BA
:101300000123934040F20342134201D012F012FB3A
:101310006420A94EFBF7B0FAFAF7B0FAA74ADFF853
:10132000C4E20023B146985D03F10F0103F11307F6
:10133000314437440EEB000A11F8018FB8F1000F69
:1013400005D09AF80CC0C44508BF82F858C091F87F
:101350000480B8F1000F05D01EF800C0C44508BFD6
:1013600082F859C08F42E7D1B2F8581041B104EB6E
:10137000800009EB03015165C0F8102802F51772CF
:101380002033602BCFD12868C0F3801011F0BAFF52
:101390002B68DE0740F19F8311F044FFB4F8286802
:1013A000874B94F824081E80002E40F09A83FAF7A9
:1013B00049FD844A8449106094F82528003218BFFA
:1013C00001220A7058B194F82638C671002B4FF0EC
:1013D0002402827114BF11210121EFF732FC002099
:1013E000FBF702FB794B7A4803F1300C4FF0000811
:1013F00053F8057C77B313F9092CA11800EB0216FA
:1014000091F82AE891F82D9891F830A8991E11F8D2
:1014100001BFF34591F802B008BF86F804E0CB4560
:1014200091F804B008BF86F80590D34508BF86F848
:1014300006A09942EBD111014218167956B156799E
:1014400046B1967936B147505979D171997911726F
:1014500082F80C8010336345CAD11420EFF794FF53
:101460002C20EFF791FF0020EFF79BFF0120EFF713
:1014700098FFDFF87491DFF8748159F8063C029305
:10148000002B3AD019F90A6C142303FB06871A467D
:10149000002138461DF0C9F8A219A9F1030A92F8F3
:1014A000333892F835B803931AF8011F039B994219
:1014B00003D11846FAF7C6FCB8609AF803105945EC
:1014C00003D15846FAF7BEFCF860CA45ECD11423A4
:1014D00003FB06F108EB0102906870B1D06860B1BF
:1014E0002644A9F10A0048F8010096F83718029B33
:1014F000117496F8391853605174364B09F110097C
:101500004B45BAD113F07CFF1420FAF79BFCC4F8CA
:101510003C0818B12A2383710023C3712E4FEFF7C3
:10152000BAFDD4F83C0813F00FFD97F80890B9F114
:10153000000F5FD04846FAF785FC284E8046706061
:1015400018B12F2383710023C3713F78002F40F01F
:10155000CC82484614F040F8074600284AD0B8F13B
:10156000000F04D0027A02214046FAF79DFADFF814
:1015700080801B4A00230193009339468023404614
:1015800016F0F0FDB268802333611360012308F880
:10159000083C2FE0741C00206B080008221503088B
:1015A000B1650020444D0020AC65002004320020CD
:1015B00028420020D84E002058F00208641D002068
:1015C000C8580020CC580020CA580020C1F002089A
:1015D0005C67002012F10208706500205C65002045
:1015E00000A24A04B44E0020F2F002088C580020F9
:1015F00064650020DB49DC4A4B795E1E734273410F
:1016000013708B795F1E7B427B4113712B68190429
:1016100000F19B8213F0007305D0D44BDB7AA3F169
:10162000080043424341937013F0EAFCD4F8403879
:101630003BB9D4F8442822B9D4F84828002A00F04D
:101640009F801BB208EE103A9FEDC9BADFEDC98A40
:10165000C94AB8EEC88A002128EE0B8A117038EE0C
:10166000280AFDEEC07A17EE903A2033402B00F2A4
:101670006E82F0F753FBF0EE409AFDEEC87A17EE5B
:10168000903A2033402B00F26582B0EE480AF0F722
:1016900045FBB0EE40AAB4F9443809EE103AB8EE72
:1016A000C99A29EE0B9A39EE280AFDEEC07A17EE98
:1016B000903A2033402B00F25082F0F72FFBF0EEEF
:1016C00040AAFDEEC97A17EE903A2033402B00F283
:1016D0004782B0EE490AF0F721FBB0EE409AB4F928
:1016E000483808EE103AB8EEC88A28EE0B8A38EE71
:1016F000280AFDEEC07A17EE903A2033402B00F214
:101700003282F0F70BFBF0EE408AFDEEC87A17EE5E
:10171000903A2033402B00F22982B0EE480AF0F7CD
:10172000FDFA69EE806A68EE8A7AF0EE665AE7EEB4
:10173000895A924B28EEA96A20EE0A7AC3ED035A21
:10174000F0EE465AE7EE495AE6EE897AA6EE497A75
:1017500068EEAA8A2AEEC00A2AEE6AAA69EEAA9A56
:10176000C3ED008A83ED010A83ED029AC3ED045AAA
:1017700083ED05AA83ED067AC3ED077AC3ED089AD7
:101780000CF0CCFC002800F0F4817D4B18680DF0C3
:1017900031F894F80C387B4F012143F002030846DE
:1017A00084F80C38FBF77AFA00210846FBF776FA42
:1017B00000210220FBF772FA0A260120FBF78AFAC1
:1017C0000020FBF787FA1920FBF756F83B68D9038E
:1017D00002D40120FBF708F91920FBF74DF800208F
:1017E000FBF702F9013EE8D131463046FBF756FAE5
:1017F00031460120FBF752FAFEF782FD624B634F40
:10180000186803F027FE624B18880CF07BFF614BD1
:101810003A781A7004F0C4FC2A685F4BD2049E8A9E
:1018200048BF5E4A9B7848BF9688042B04D14FF48A
:101830008050EFF7E3FE002604F0D4FA584B304610
:10184000197815F011FB94F80C3843F0040384F870
:101850000C3801F053FB01F00BFB524B1B680BB132
:1018600015F016F900F012FF04F0A6FD13F050FA7F
:101870004FF4197200214C48DFF84C91DFF84C818D
:101880001CF0D3FEFFF7C8FC484B00261E809E705C
:101890000EF086FC464BC8F800604FF0FF3AC3F8E4
:1018A00000A04846434BC4F84C3816F0D3FF424AD8
:1018B00084F85A68012384F85838537884F859A872
:1018C0000D3384F8543813781E3384F85538D8F81B
:1018D0000030042B464605D05A1CC8F80020374A71
:1018E00042F823902B68364C13F4003F00F09380AD
:1018F00094F86838DFF8D880DFF8D890013B84F896
:10190000603894F8693884F86138C82004F65C03BC
:10191000C8F80030FAF7B0FFD8F8000006F0B0FFC2
:1019200089F80000C820FAF7A7FFD8F80030C4F8FB
:10193000703804F66C08234BC4F86C38404616F037
:101940001FFF012384F87838002384F87A38FF23B6
:1019500084F87938082384F87438152384F87538A6
:101960003AE000BF4C6600207C580020D84E002092
:1019700035FA8E3CDB0FC93FD80400204C400020D4
:10198000344D0020D4290020B865002050360020B6
:101990001036002050260020C8610020282C00208E
:1019A000B2310020B8270020A45900205C66002036
:1019B000FC04002008F102088C650020544200203D
:1019C000741C002034F10208C02400205042002082
:1019D000A86500209D6600206B4BC3F8008099F835
:1019E00000303BB13368042B04D05A1C3260674A84
:1019F00042F82380664E1022002130461CF015FE6E
:101A0000002017F03BFBFAF791FE804617F050FBE1
:101A1000604B4344F360604E002333702B68D8035F
:101A200008D517F091FA012333705C4B93F8F1005D
:101A300006F024FE2B68590501D50AF089F8584BA9
:101A40001B880BB914F0F2FDF0F736FC19F07EFBA1
:101A50003B78052B03D1534B4FF4C8721A80524B7D
:101A60001A684FF47A73B3FBF2F3C3EB431203EB40
:101A700082034E4ADB00A2F8B4304D4B4D4A1A6047
:101A80004D4A137843F008031370FFF70BF84B4BE4
:101A90001A68920306D53E4A07215172117A41F025
:101AA00001011172464A12681A6016F01FFB454A7E
:101AB000138843F08003138010F07CF8FFF71AFBC3
:101AC00094F80C3863F07F0384F80C3807B0BDEC51
:101AD000088BBDE8F08F98047FF560AC11F04CFBEB
:101AE0005CE4314616F0D4FC7CE4012F7FF482AD37
:101AF000404613F029FA7068EFF7CDFA4FF4E0731F
:101B0000336137703623002604A88DF810308DF825
:101B100011708DF812608DF8137010F023FC3723CC
:101B200005A88DF814308DF815708DF816608DF8B5
:101B3000177010F017FC244AD36943F03003D361C7
:101B4000224B1E85A3F8286454E501236BE5DFEDE5
:101B5000209A92E59FED1EAA9DE5DFED1DAAB0E556
:101B60009FED1B9ABBE5DFED1A8ACEE59FED180AC3
:101B7000D7E502210120FAF7AFFC124A138843F09F
:101B80000103138005E600BF946600205442002044
:101B900084660020404B4C005A3800205837002003
:101BA0007814002006670020344D0020B04A002041
:101BB000142E00208800002028340020444D0020EE
:101BC00028420020806600200010024000100040E3
:101BD0000000000008B50E4B1978012913D00DD371
:101BE000022902D10020FBF775F8FAF79FFD094B97
:101BF00000F5F42000F59070186008BD002108463B
